:100000000C9495090C94E4090C94E4090C94E4090B
:100010000C94E4090C94E4090C94E4090C94E409AC
:100020000C94E4090C94161D0C94E4090C94E40956
:100030000C9475380C94E4090C94E4090C94E409CC
:100040000C94E4090C94E4090C944A190C94E40906
:100050000C94780F0C94E4090C94420F0C94E4096E
:100060000C9406200C94E4090C94FB330C94E409E2
:100070000C9411960C94E4090C94088C0C94E409EB
:100080000C94E4090C94E4090C94E4092D2032202A
:100090003720402057206E207E208E20C9205823F4
:1000A0006E20E521F621252243226022BA22152363
:1000B000E725AA265C27D3270B28AE28B52A1F2BB5
:1000C000992BE22B2C2C5A2C872CEA2C342D7E2DAC
:1000D000772E1A344E349134013519355A3511368C
:1000E000D836D836D836D836D836D836D836D836A0
:1000F000D836D836D8368D368F369436AC36AE36BE
:10010000A66D656EEA6E196E406F706FDA6D486E9F
:10011000977D357EBA7E1C7F707FD97F39875A8064
:100120008C808C808C808C808C808C808C808C806F
:100130008C80BA803581CA81EF8132828A821583B0
:10014000FE836584658465846584658465846584CF
:10015000658465849D84BB84E0843C857885E785DF
:100160001486B486398714871487148714871487F4
:100170001487148714874F945294529452945B942A
:100180005E946194739470940A0D3D3D3D3D3D3DF8
:100190003D3D3D3D3D3D3D3D3D3D3D3D3D3D3D3D8F
:1001A0003D3D3D3D3D3D3D3D3D3D3D3D3D000A0D1F
:1001B000426174743A002025642043656C6C73209E
:1001C00000204C6F77207761726E696E673A202548
:1001D000642E2564000A0D466F756E6420424C2D16
:1001E0004374726C3A20002564000A0D0A0D212127
:1001F000204D495353494E4720424C2D4354524CB5
:100200003A202564202121000A0D43616C69627245
:100210006174696E6720707265737375726520739F
:10022000656E736F722E2E004F4B0A0D000A0D463D
:100230006C696768742D74696D65202575206D691A
:100240006E20546F74616C3A2575206D696E0041A3
:100250006E676C654E69636B202020202020204152
:100260006E676C65526F6C6C20202020202020412E
:1002700063634E69636B20202020202020202041D2
:100280006363526F6C6C2020202020202020205996
:1002900061774779726F2020202020202020204184
:1002A0006C746974756465205B302E316D5D20411E
:1002B00063635A2020202020202020202020204757
:1002C0006173202020202020202020202020204377
:1002D0006F6D706173732056616C756520202056B8
:1002E0006F6C74616765205B302E31565D20205243
:1002F00065636569766572204C6576656C2020477C
:1003000079726F20436F6D70617373202020204DD0
:100310006F746F7220312020202020202020204D5B
:100320006F746F7220322020202020202020204D4A
:100330006F746F7220332020202020202020204D39
:100340006F746F7220342020202020202020203144
:100350003620202020202020202020202020203176
:100360003720202020202020202020202020203165
:100370003820202020202020202020202020203154
:100380003920202020202020202020202020205321
:100390006572766F202020202020202020202048F9
:1003A0006F76657267617320202020202020204313
:1003B000757272656E74205B302E31415D20204372
:1003C00061706163697479205B6D41685D202048CC
:1003D000656967687420536574706F696E74203244
:1003E00035202020202020202020202020202032E6
:1003F00036202020202020202020202020202043C4
:100400006F6D7061737320536574706F696E74499A
:1004100032432D4572726F7220202020202020420E
:100420004C204C696D69742020202020202020471A
:1004300050535F4E69636B202020202020202047EE
:1004400050535F526F6C6C202020202020202021F0
:10045000212120494E434F4D50415449424C4520A3
:10046000212121002A002E000A0D20444143206F43
:100470007220493243204552524F52212043686531
:10048000636B204932432C2033567265662C20441E
:10049000414320616E6420424C2D4374726C005BBA
:1004A00025695D005B25695D002B204D696B726FCE
:1004B0004B6F70746572202B0048573A5625642E96
:1004C00025642053573A25642E256425632056342D
:1004D0000053657474696E673A2564202573004D76
:1004E00069786572204572726F72210045525225FB
:1004F00032643A00486172647761726520457272B5
:100500006F7220313A2564202121004D697373698F
:100510006E6720424C2D4374726C3A256421210091
:10052000493243204552524F5221212100486569EA
:100530006768743A202025356900536574706F69C7
:100540006E743A2535690050726573737572653A39
:10055000253569004F66667365743A202025356934
:10056000002841290048656967687420636F6E74CC
:10057000726F6C0044495341424C454400616374BE
:100580002E2062656172696E67004E69636B3A2066
:10059000202020202025356900526F6C6C3A2020E5
:1005A0002020202025356900436F6D706173733AF8
:1005B000202020253569004B25693A253469202003
:1005C0004B25693A25346920004E693A2534692063
:1005D00020526F3A253469200047733A2534692048
:1005E0002047693A253469200050313A2534692082
:1005F0002050323A253469200050333A253469209E
:100600002050343A25346920004779726F202D201C
:1006100053656E736F72004E69636B2534692028D1
:100620002533692E25692900526F6C6C25346920A9
:10063000282533692E2569290047696572253469A3
:10064000202825336929004E69636B2025346920F1
:10065000282533692E25782900526F6C6C202534AB
:100660006920282533692E257829005961772020B3
:10067000253469202825336929004E69636B2025BC
:100680003469202825336929282533692900526FC8
:100690006C6C202534692028253369292825336985
:1006A00029005961772020253469202825336929BC
:1006B000282533692900414343202D2053656E735B
:1006C0006F72004E69636B202534692028253369D9
:1006D0002900526F6C6C2025346920282533692944
:1006E000005A20202020253469202825336929003C
:1006F000566F6C746167653A2020202533692E257A
:100700003169560043757272656E743A2020202557
:1007100033692E2531694100506F7765723A202088
:10072000202020253469570044697363686172672B
:10073000653A202535696D416800526563656976C3
:1007400065720052432D525353493A2020202025F0
:1007500034690052432D5175616C6974793A2025D2
:1007600034690052432D4368616E6E656C733A259F
:10077000346900436F6D70617373004D61676E651E
:10078000743A202020253569004779726F3A20207D
:1007900020202025356900536574706F696E743AA6
:1007A0002025356900506F746925693A202025336A
:1007B0006900506F746925693A2020253369005318
:1007C0006572766F202000536574706F696E7420B7
:1007D0002025336900506F736974696F6E3A202564
:1007E00033690052616E67653A2533692D25336997
:1007F00000424C2D4374726C204572726F727320EC
:100800000025336420253364202533642025336498
:100810002000424C2054656D70657261747572657C
:100820000025336420253364202533642025336478
:100830002000424C2D4374726C20666F756E6420EC
:1008400000202563202020256320202025632020F0
:1008500020256320002025632020202563202020E0
:100860002563202020256320002025632020202DC3
:100870002020202D2020202D20003130003131007B
:10088000313200466C696768742D54696D652020AB
:1008900000546F74616C3A2535756D696E00416363
:1008A000743A20202535756D696E00287265736570
:1008B0007429000A0D47656E65726174696E672060
:1008C00064656661756C7420506172616D657465F4
:1008D0007220536574202564000A0D5573696E6794
:1008E00020506172616D65746572205365742025B6
:1008F00064000A0D47656E65726174696E672064F5
:10090000656661756C74204D69786572205461620A
:100910006C65000A0D4D697865722D436F6E6669CE
:10092000673A202725732720282575204D6F746F7F
:10093000727329000A0D414343206E6F7420636176
:100940006C69627261746564210D0A0000008F0099
:100950001E01AD013B02CA025803E60374040205FE
:100960008F051B06A7063307BE074808D2085B0998
:10097000E3096B0AF20A780BFD0B810C040D860D5E
:10098000070E870E060F840F00107B10F5106E11F6
:10099000E5115B12CF124213B31323149214FE1409
:1009A0006A15D3153B16A11605176717C817271820
:1009B0008318DE1837198E19E319361A871AD61AD2
:1009C000231B6E1BB61BFD1B411C831CC31C001D7F
:1009D0003C1D751DAB1DE01D121E421E6F1E9A1E92
:1009E000C31EE91E0D1F2E1F4D1F691F841F9B1F55
:1009F000B01FC31FD31FE11FEC1FF51FFB1FFF1FFD
:100A0000002004010000DF740002010108760103E8
:100A100002029C7602040303447703000404F9767F
:100A20002532692E2531695600253364256320253A
:100A30003033646D256300537461747573004552DF
:100A4000524F523A20253264200025346920253245
:100A5000693A25303269002534696D2563002533F4
:100A60006920253369202533692025336900253322
:100A700069202533692025336920253369005465B1
:100A80006D70657261747572657320202020002579
:100A900063432020202020002532692E253169560D
:100AA000202533692E2531694100253469572025D9
:100AB00036696D4168004D61676E65743A2533692A
:100AC000252520253369256300496E636C692E3A1C
:100AD0002533692563202825692920002532756D75
:100AE0002F73205361743A25642000202033440082
:100AF0004E6F4678004447505300486F6D653A2565
:100B000033646D202533642563202563004E6F20F8
:100B10004E6176694374726C210000000500050087
:100B20000401060108000601020004000400070099
:100B30000700070007000700070007000301030183
:100B4000050017010F01060009010A01190105013D
:100B5000050119011A010F0100004E6F2045727244
:100B60006F722020202020202020004E6F742063F0
:100B70006F6D70617469626C652020004D4B334D60
:100B80006167206E6F7420636F6D7061004E6F201F
:100B9000464320636F6D6D756E6963617400436FCA
:100BA0006D7061737320636F6D6D756E696300475F
:100BB000505320636F6D6D756E69636174696F006A
:100BC000636F6D706173732076616C756520202092
:100BD000005243205369676E616C206C6F73742000
:100BE0002000464320737069207278206572726F0E
:100BF0007220004E6F204E4320636F6D6D756E69DD
:100C0000636174004643204E69636B204779726FBD
:100C10002020202000464320526F6C6C20477972C0
:100C20006F202020200046432059617720477972A9
:100C30006F2020202020004643204E69636B204116
:100C40004343202020202000464320526F6C6C201C
:100C50004143432020202020004643205A2D414379
:100C600043202020202020202000507265737375BF
:100C700072652073656E736F72200049324320469F
:100C8000432D3E424C2D4374726C2000426C204D2B
:100C9000697373696E67202020202020004D6978D9
:100CA0006572204572726F722020202020004361FF
:100CB000726566726565204572726F72202000470A
:100CC000505320466978206C6F73742020202000D8
:100CD0004D61676E6574204572726F72202020200E
:100CE000004D6F746F72207265737461727420208E
:100CF0002000424C204C696D69746174696F6E20EC
:100D00002020004750532052616E6765202020202C
:100D1000202020004E6F2053442D43617264202018
:100D2000202020200053442D4C6F6767696E672098
:100D30006572726F7200466C79696E672072616EBF
:100D4000676521202020004D617820416C74697412
:100D500075646521202020004E6F20475053206687
:100D6000697820202020202000636F6D70617373EC
:100D7000206E6F742063616C2E00202121204C694D
:100D8000506F20766F6C74616765202121202000F0
:100D900020202020204D696B726F4B6F707465723C
:100DA0002020202020002020202020202020202063
:100DB000202020202020202020202000202025323C
:100DC000692E2531695620200020202532692E25E4
:100DD000316956202000414C543A2534696D202554
:100DE0006300414C543A2534696D202000414C5435
:100DF0003A2D2D2D2D200020202532693A25303224
:100E00006920200020202532693A253032692020CF
:100E1000004449523A2025336425630043002000F2
:100E2000202025356920200020202535692020003C
:100E3000493A2532692E2531694120003A003A00AD
:100E40003A002D2D2D2D2D2D2D2D2D2B2D2D2D2DF4
:100E50002D2D2D2D2D2D2D002D2D2D2D2D2D2D2DEF
:100E60002D2D2D2D2D2D2D2D2D2D2D2D2D003A00FF
:100E70005341543A2532642000444953543A2533AF
:100E8000646D004420003344002121004D41473A65
:100E900025337525252000484D3A253364256320E8
:100EA000256300696E636C3A253264256328253218
:100EB000692900202020202532756D2F733A2020CB
:100EC000484D3A2533642563202563004552523A44
:100ED000202532642021004552523A200021212051
:100EE0004C69506F20766F6C74616765202121001A
:100EF000207777772E4D696B726F4B6F70746572C8
:100F00002E6465202000202532693A253032692080
:100F1000202532692E25316956202534696D4168B6
:100F200000202532693A2530326920202532692E89
:100F300025316956202534696D4168004449523A8B
:100F4000253364256300414C543A2534696D0041D2
:100F50004C543A2534696D00414C543A2D2D2D2DB9
:100F60002000256300484D3A253364256320204442
:100F70004953543A2533646D202563005057523A43
:100F80002532692E253169412028256957292000FD
:100F90004346002020004750533A2532756D2F7389
:100FA000205341543A256420002020334420004E31
:100FB0004F464958004447505320002020204E6F90
:100FC000204E6176694374726C20202020202020FE
:100FD000002532692E2569202532692E25692025B4
:100FE00032692E2569202532692E25694100253375
:100FF000692025336920253369202533692563431A
:10100000002532692E2569202532692E2569410087
:101010002532692E2569202532692E256920253241
:10102000692E2569202532692E25694100253369FD
:101030002025336925634320202020202020200004
:101040002533692025336920253369202533692517
:101050006343004552523A20253264202100455214
:10106000523A20002121204C69506F20766F6C7419
:1010700061676520212100207777772E4D696B729B
:101080006F4B6F707465722E646520200053657419
:1010900074696E673A257520257320004D696E3A94
:1010A0002532692E253169562025732000414C5484
:1010B0003A00504F54493A2533752000284F4E29A5
:1010C000202000284F46462920004C494D49540015
:1010D000564152494F0044495341424C4544004314
:1010E000463A0044495341424C45440020284F4E63
:1010F00029200020284F46462900205445414348D6
:10110000004750533A0044495341424C454400285B
:1011100046524545290028484F4D45290028414958
:101120004429200028484F4C4429002046533A25A2
:101130007573656B2000484F4D4520414C543A0073
:1011400025756D00484F4C4420004E693A2534699E
:1011500020526F3A25346920433A2533690047739A
:101160003A2534692059613A253469200050313AD2
:101170002534692050323A25346920333A253369C1
:101180000050343A2534692050353A2534692036E8
:101190003A25336900434F55504C494E47204F463E
:1011A000462120004C4F4F50494E472120004848CF
:1011B000212000434F4D50415353204F464621209C
:1011C00000004F505152535453565748005859003D
:1011D0005A5545464748410049424A4A00000000E6
:1011E00000000000000000444C4D00000000004ED4
:1011F0000000004B00430A0D7777772E4D696B7224
:101200006F4B6F707465722E6465202863292048C7
:101210006953797374656D7320476D6248000A0DD8
:1012200074686520757365206F6620746869732023
:10123000736F667477617265206973206F6E6C7965
:10124000207065726D6974746564200A0D6F6E207C
:101250006F726967696E616C204D696B726F4B6F5D
:10126000707465722D4861726477617265005573A0
:10127000657200486F545420563400414354204452
:10128000534C004A657469005370656B7472756DD8
:101290000050504D000A0D52656365697665723ADB
:1012A0002000532E42757300756E6B6E6F776E2E35
:1012B000205573696E672050504D2E2E2E006E6F94
:1012C0007420737570706F72746564206279206821
:1012D0006172647761726521000A0D466C69676806
:1012E00074436F6E74726F6C0A0D4861726477613B
:1012F00072653A25642E25640A0D536F6674776112
:1013000072653A5625642E2564256320000A0D2057
:101310002D204C4942204E4F5420434F4D504154B4
:1013200049424C4520212121210011241FBECFEF2D
:10133000D0E4DEBFCDBF12E0A0E0B1E0E2EFF2E327
:1013400001E00BBF02C007900D92A83DB107D9F78D
:101350001BE0A8EDB2E001C01D92AE38B107E1F785
:101360007AEAE2E0F0E081E280935700D4907E01D7
:101370000894E11CF11C20EF37EF41E050E08701B9
:101380006FE0DA01C9012F5F3F4F4F4F5F4FABBF97
:10139000FC018791F80181938F01615067FFF1CFC4
:1013A000F7016EE0819178277095615067FFFACF61
:1013B0008889781729F0F7E9DF1611F40000FECFCD
:1013C0000E94B00A0C9478990C94000088E891E08F
:1013D0009F938F938EE296E19F938F93E091F40415
:1013E000F091F50409950F900F900F900F900895CC
:1013F00080913F07E82FFF27EE0FFF1FEE58F74FB2
:10140000808191818D5E9F4F14F010920201808146
:1014100091818A5B9F4FCCF4809102018823A9F4CB
:1014200081E080930201809128058F5F80932805D9
:10143000853038F088EE93E090930D0380930C0391
:10144000089566E970E00E94633A08951F93CF9370
:10145000DF93182F882389F08EEA91E09F938F9372
:101460008EE296E19F938F93E091F404F091F5045E
:1014700009950F900F900F900F9080916207823323
:1014800008F044C084EF91E00E942C1AEC01112373
:1014900029F0CE010E94351A8823D9F3C2E0D0E0AA
:1014A00026E530E080911F0190912001821793077B
:1014B00030F02196255D3F4FC730D10598F38091DC
:1014C00062079927C89F9001C99F300DD89F300DA2
:1014D0001124209300011123D9F068EC70E08C2FC7
:1014E0000E94633ADF93CF9386EB91E09F938F93B3
:1014F0008EE296E19F938F93E091F404F091F504CE
:1015000009958DB79EB706968DBF02C080930001E6
:10151000112311F1809100016AE00E94CB98892F7C
:1015200099279F938F93809100010E94CB989927D0
:101530009F938F9381EC91E09F938F938EE296E13E
:101540009F938F93E091F404F091F50409952DB7E2
:101550003EB7285F3F4F2DBFDF91CF911F91089578
:10156000CFEFD0E4DEBFCDBF8824992414B815B8DE
:101570008AE08AB98FE58BB9B7EEEB2EB3E0FB2E8C
:101580002EEC3FEFE20EF31EF7FEFACF199B08C0D8
:101590004C9B04C085E18093010108C086E101C035
:1015A00087E18093010181E08093670381E190E00E
:1015B0000E94F23090910101981789F081E190E04A
:1015C0000E94F2308F3F29F060E081E090E00E94BD
:1015D000FA306091010181E190E00E94FA3081E8E7
:1015E00087B93E9A8FEF88B98BE184B981E085B9DC
:1015F000469A84B7877F84BF80916000886180931A
:1016000060001092600084EC99E090930D03809349
:101610000C031092B4031092B30310927708109247
:1016200076081092B6031092B5031092B803109288
:10163000B70320910101243128F084EC94E0A0E06C
:10164000B0E004C08BE095E0A0E0B0E080933C0106
:1016500090933D01A0933E01B0933F012A3011F0D9
:10166000243110F0289801C0289A2C3010F027312E
:1016700011F4299A01C029980E94951A0E94661AAD
:101680000E9436160E944C380E94971E81E00E94EC
:10169000AF330E94386C0E943C7882E00E94C7946D
:1016A000809101018C3010F0873111F4299A01C02A
:1016B000299878940E94CE3280915603826080935C
:1016C0005603109259030E94274684EF91E00E942E
:1016D0002C1A7C018091560380FD05C0C7010E9431
:1016E000351A8823B9F385ED91E09F938F93AEE28D
:1016F000AA2EA6E1BA2EBF92AF92E091F404F09127
:10170000F504099580EA9FE00E942C1A7C01C0E054
:10171000D0E00F900F900F900F9004E118E0F8ECDC
:10172000CF2EF7E0DF2E0E9427468091560380FDE2
:1017300005C0C7010E94351A8823B9F3F6018081DC
:101740001816ACF40BC00E9427468091560380FD0A
:1017500005C0C7010E94351A8823B9F3C7010E944A
:10176000351A882321F4F8018081882364F7F80171
:10177000808187FF19C02196DF93CF93219787EE51
:1017800091E09F938F93BF92AF92E091F404F09118
:10179000F50409958091D9028F5F8093D9022DB706
:1017A0003EB72A5F3F4F2DBF219684E090E0C80EE0
:1017B000D91E085F1F4FCC30D10508F4B4CFC0E06C
:1017C000D0E001E118E0E8ECEE2EE7E0FE2EF801B3
:1017D000838187FD1DC0F70180811816CCF4219606
:1017E000DF93CF9321978AEE91E09F938F938EE2C0
:1017F00096E19F938F93E091F404F091F50409959D
:1018000082E080930A032DB73EB72A5F3F4F2DBF7A
:10181000F801838180788383219624E030E0E20E12
:10182000F31E085F1F4FCC30D10588F20E94E609F5
:1018300090913D078091D902981728F480910E0568
:10184000806180930E0588E092E09F938F93CEE2B3
:10185000D6E1DF93CF93E091F404F091F50409957C
:1018600088EE93E00E942C1A7C010E949D1E0F902E
:101870000F900F900F90C7010E94351A8823D9F35B
:1018800088E292E09F938F93DF93CF93E091F404EB
:10189000F091F504099580E00E94473B8091010199
:1018A0000F900F900F900F908A3011F0843110F04C
:1018B000289801C0289A80ED97E090930D038093BB
:1018C0000C0385E580932A058EE090E00E94F230BB
:1018D0009927182F00278FE090E00E94F230080F20
:1018E000111D1093DF020093DE028AE090E00E9457
:1018F000F2309927182F00278BE090E00E94F230F9
:10190000080F111D1093DD020093DC020F5F1F4FC3
:1019100039F08091DE029091DF028F5F9F4F41F49A
:101920001092DF021092DE021092DD021092DC02B1
:101930008091DC029091DD029F938F938091DE0273
:101940009091DF029F938F938DE292E09F938F930C
:10195000DF93CF93E091F404F091F50409950E9490
:10196000592588E893E19093370180933601C1E0CF
:10197000C09329058C2F0E94260A809165070E943A
:1019800013940E94E60980ED97E00E942C1A7C01D6
:101990008AEF90E00E942C1A83E0809397061092C1
:1019A000D8028091AC072DB73EB7285F3F4F2DBFBF
:1019B00084FF02C0C093E0028091E202882311F00C
:1019C0004798FECF80911003882309F453C2809179
:1019D0001101882309F44EC210921003809128054A
:1019E000882319F00E94F80902C00E9485490E94CC
:1019F0002746209101012A3011F0243110F0289857
:101A000001C0289A8091A703882331F08091A70311
:101A100081508093A7030EC080916F0080628093F5
:101A20006F00109273081092720880910E05886002
:101A300080930E0580913601909137010197909324
:101A40003701809336018091360190913701892BBF
:101A500021F0809157038823C9F18091360190913C
:101A60003701892BD9F40E94D93385E090E0909317
:101A70003701809336018091D1069091D20601966C
:101A80009093D2068093D10680910E058160809359
:101A90000E058091980682608093980680910901D6
:101AA00090910A018F5F9F4FC1F48091A603882314
:101AB000A1F088EA91E690930D0380930C0380E8EF
:101AC00090E090930A018093090107C02A3011F039
:101AD000243110F0289801C0289A0E949495809192
:101AE0001003882309F0C6C18091C104882319F02E
:101AF0000E94B987BFC180910F01882311F00E9415
:101B0000EE1A0E947A160E94C811C7010E94351A67
:101B1000882309F4ABC184E190E0E80EF91E0E942D
:101B2000AC1A80916507863019F40E945B7D04C071
:101B3000843011F40E94898880915703882349F0EA
:101B400080910E05826080930E05809198068260D8
:101B50000FC080910C0390910D03892B59F4809153
:101B6000360190913701079728F0809198068D7F74
:101B7000809398068091E002882361F08091A7030A
:101B8000873940F01092E00288E893E190930D03CA
:101B900080930C0380910401882321F0815080936D
:101BA00004012EC08093340510927B0310927A03B7
:101BB00010927903109278031092770310927603B3
:101BC0008091A7038823E1F48091090190910A0193
:101BD0008F5F9F4FA9F42091E002223089F088E9BD
:101BE0009AE390930D0380930C0380E09CE0909324
:101BF0000A0180930901222319F082E08093E00218
:101C000080919901893C48F081508093990180919D
:101C10000E058B7F80930E053FC080915509882368
:101C2000F9F080910E05846080930E0589E0809321
:101C300085048091090190910A018F5F9F4F81F483
:101C40008091A603882361F088E99AE390930D03BD
:101C500080930C0380E098EA90930A018093090135
:101C60001092770410927604109275041092740406
:101C700010927304109248091092870910928609F5
:101C800010928909109288098FEF9FEF9093850930
:101C9000809384091092990180910001282F3327A5
:101CA00080911F019091200182179307CCF48091BD
:101CB0006F03806280936F038091090190910A0104
:101CC0008F5F9F4FC1F480E797E190930D0380935E
:101CD0000C0380E093E090930A01809309010BC00C
:101CE00080910C0390910D03892B29F480916F034F
:101CF0008F7D80936F030E942F7184E080930B038C
:101D00008091E1028F5F8093E102813309F065C029
:101D10001092E10280916F0381FF0AC08091DA0284
:101D20009091DB0201969093DB028093DA0204C06B
:101D30005AEA852E55E0952E80917003909171039B
:101D40008050944008F049C02091E0063091E106AF
:101D50004091E2065091E30680911701909118019D
:101D6000A0911901B0911A01281739074A075B079A
:101D700064F48091E0069091E106A091E206B091B2
:101D8000E3060596A11DB11D20C02091E00630910B
:101D9000E1064091E2065091E3068091170190918F
:101DA0001801A0911901B0911A0182179307A40795
:101DB000B5079CF48091E0069091E106A091E206BF
:101DC000B091E3060597A109B1098093E0069093CD
:101DD000E106A093E206B093E3060894811C911CEF
:101DE00082E788168BE0980609F040C08824992481
:101DF0002091DE023091DF022F5F3F4F3093DF02F0
:101E00002093DE028091DC029091DD020196909396
:101E1000DD028093DC02832F9927682F8EE090E00B
:101E20000E94FA308091DE029091DF029070682F5C
:101E30008FE090E00E94FA308091DC029091DD0208
:101E4000892F9927682F8AE090E00E94FA308091CC
:101E5000DC029091DD029070682F8BE090E00E9490
:101E6000FA3084E190E00E942C1A7C010E947F717C
:101E70000E94537880910B03882309F09DCD0E9426
:101E8000596C9ACD1F920F920FB60F9211248F9317
:101E90009F93EF93FF93809106018823E1F4809153
:101EA000FC029091FD0201969093FD028093FC024A
:101EB000FC01E851FA4FE081ED3019F08F3A9105BD
:101EC00039F41092FD021092FC0281E08093060129
:101ED000E093C60004C01092FD021092FC02FF9134
:101EE000EF919F918F910F900FBE0F901F901895BB
:101EF0001F920F920FB60F9211242F933F934F937F
:101F00005F936F937F938F939F93AF93BF93CF9381
:101F1000EF93FF9390E08091E202813029F4809169
:101F2000C6008093CE00CCC08091E202823029F4BA
:101F30008091C60080933705C3C08091C60080930E
:101F4000F402509102035F3A10F0909303038091E2
:101F5000F4028D3009F065C080910303823009F0EE
:101F600060C090930303852F9927895C9A4FFC01E9
:101F7000329740812091FE023091FF02241B3109EB
:101F8000DC0111978C91281B3109C9019F70909336
:101F9000FF028093FE0246E0969587954A95E1F709
:101FA000982F935C909300032F733070235C2093E1
:101FB00001038081981729F48C91281711F491E07E
:101FC00006C090E08091F1028F5F8093F102C09192
:101FD000F302CC2309F074C0992309F471C081E0A5
:101FE0008093F302580F5093F0025150E52FFF27D2
:101FF000E95CFA4F8DE0808380913905823509F0E4
:102000005FC00E94592588E190E02CE00FB6F8945B
:10201000A895809360000FBE20936000C0930A03D0
:102020004FC020910303822F992781309105F9F049
:10203000823091051CF4892B21F040C0029711F1E8
:102040003DC08091F402833239F48091F3028823F9
:1020500019F481E0809303038091F40280933705A3
:1020600081E0809302038091F402992722C02F5FC0
:1020700020930303E52FFF27E95CFA4F8091F402D8
:10208000808309C0E52FFF27E95CFA4F8091F402B5
:1020900080835F3A20F45F5F5093020302C0109286
:1020A00003032091F4028091FE029091FF02820FBF
:1020B000911D9093FF028093FE0202C010920303D1
:1020C000FF91EF91CF91BF91AF919F918F917F91B0
:1020D0006F915F914F913F912F910F900FBE0F9095
:1020E0001F901895AC01A0E0B0E09D01A817B907BA
:1020F00048F4E8EEF5E08191280F311D1196A41700
:10210000B507C8F33F70FD01E851FA4FC90156E029
:10211000969587955A95E1F7835C80831196FD012A
:10212000E851FA4F2F733070822F835C8083A75160
:10213000BA4F8DE08C93109206018091E805809350
:10214000C6000895A0E0B0E0E8EAF0E10C944499FC
:102150002C859D850E85BB2483E28093E8059F59DD
:102160009093E9052093EA0533E0E32EF12C002358
:1021700009F49EC0CF84D888BE016D5E7F4FA989C7
:10218000BA890150109709F493C01097B9F0F6017D
:10219000EB0DF11DB3949081119791F4002349F157
:1021A000FB016E5F7F4FDB01C080D1806E5F7F4F90
:1021B0000D90BC91A02DBB24015002C090E019C02D
:1021C0001097B9F0F601EB0DF11DB3944081119712
:1021D00091F4002341F1FB016E5F7F4FDB01C08072
:1021E000D1806E5F7F4F0D90BC91A02DBB2401501C
:1021F00002C040E018C01097B1F0F601EB0DF11DE0
:10220000B3941081119781F4002371F0FB01329691
:10221000DB01CD90DC90BF016E5F7F4FA081B1816B
:10222000BB24015001C010E0F701E851FA4F892F9B
:1022300086958695835C80830894E11CF11CF701E8
:10224000E851FA4F892F99278370907024E0880F06
:10225000991F2A95E1F755279A0194E0369527951D
:102260009A95E1F7822B835C80830894E11CF11C32
:10227000F701E851FA4F4F705070440F551F440F4B
:10228000551F812F992726E0969587952A95E1F786
:10229000842B835C80830894E11CF11CF701E851D6
:1022A000FA4F1F73135C10830894E11CF11C6ACF72
:1022B000C7010E947210E9E00C946099A3E07A2FA4
:1022C0004091F0024650442309F458C0E72FFF27FD
:1022D000E95CFA4F80818D537F5FE72FFF27E95C30
:1022E000FA4F20812D537F5FE72FFF27E95CFA4FDC
:1022F00030813D537F5FE72FFF27E95CFA4F608114
:102300006D537F5F9927880F991F880F991F522F50
:1023100052955F70582B822F99278F709070F4E040
:10232000880F991FFA95E1F7232F26952695282BDC
:10233000832F992783709070E6E0880F991FEA95A4
:10234000E1F7682B41504F3FC9F0EA2FFF27E95CC6
:10235000FA4F5083AF5F41504F3F81F0EA2FFF2784
:10236000E95CFA4F2083AF5F41504F3F39F0EA2FCD
:10237000FF27E95CFA4F6083AF5FA5CF8AE395E062
:102380009093EF028093EE02A350A093ED02089584
:10239000A2E0B0E0EEECF1E10C944A998091F302F6
:1023A000882309F457C40E945E1180913805823653
:1023B00009F023C38091390599278037910509F4E5
:1023C000AFC081379105C4F48A36910509F480C203
:1023D0008B36910544F48B34910571F18636910565
:1023E00009F45FC10AC38D36910509F469C08E36C0
:1023F000910509F44DC001C38437910541F185373A
:1024000091054CF48137910509F491C0833791050A
:1024100009F4DFC0F2C28737910509F41BC288377F
:1024200091052CF48537910509F4D7C1E6C28937A7
:10243000910509F46DC1E1C2E091EE02F091EF0265
:102440008081918190938B0180938A01D6C2809183
:10245000F002A091EE02B091EF02853140F080E1F0
:10246000E2E1F5E00D9001928A95E1F70DC08D91C2
:102470009D910D90BC91A02D809312059093130512
:10248000A0931405B093150580EF8093EB024BC029
:10249000809106018823E1F38DE490E09F938F9370
:1024A0008BEB97E09F938F9381E08F938F938EE4D4
:1024B0008F930E94A2108DB79EB707968DBF9DC2C5
:1024C000A091EE02B091EF021C91113081F48DE4E5
:1024D000EBEBF7E00D9001928A95E1F70E940B3249
:1024E000198380910E058F7E80930E0501C019829D
:1024F000809106018823E1F381E090E09F938F9320
:10250000CE0101969F938F9381E08F938F938DE4FB
:102510008F930E94A210ADB7BEB71796ADBF6DC224
:1025200081E08093F6028FEF8093040166C2E09110
:10253000EE02F091EF02E0818E2F8A508A3058F43B
:102540008983882311F481E003C0863010F085E090
:10255000898361E00EC08E2F84518A3070F48983A4
:10256000882311F481E003C0863010F085E0898370
:1025700060E089810E948B3212C0E983EF3F19F439
:102580000E946E3289838981882311F481E003C01F
:10259000863010F085E0898389810E941031809116
:1025A00006018823E1F38CE790E09F938F938EE3FD
:1025B00097E09F938F9381E090E09F938F93CE015C
:1025C00001969F938F9382E08F9381E08F9381E5B3
:1025D00077C12091EE023091EF02D9018C918150A8
:1025E000853008F045C0F90181818D3509F040C082
:1025F0008091A6038823E1F52F5F3F4F8CE7EEE340
:10260000F7E0D9010D9001928A95E1F7F9018291E5
:102610000E947B3180917F079927AA27BB27BC01A5
:10262000CD0124EC39E040E050E00E94AC98DC01A0
:10263000CB018093820190938301A0938401B09396
:102640008501809180079927AA27BB27BC01CD016E
:102650000E94AC98DC01CB0180937E0190937F01B6
:10266000A0938001B09381010E946E32898301C0E2
:102670001982809106018823E1F381E090E09F9325
:102680008F93CE0101969F938F9381E08F938F93C9
:1026900083E58F930E94A2108DB79EB707968DBFDA
:1026A00026C0E091EE02F091EF02E0818E2F815082
:1026B000853018F48E2F0E9410310E946E3289836B
:1026C000809106018823E1F381E090E09F938F934E
:1026D000CE0101969F938F9381E08F938F9386E431
:1026E0008F930E94A210ADB7BEB71796ADBF809171
:1026F000A603882329F46EE670E089810E94633A7C
:1027000080E00E94260A809165070E94139475C19B
:10271000E091EE02F091EF028081992787FD90957C
:1027200090938D0880938C088181992787FD9095DF
:1027300090938F0880938E088281992787FD9095CA
:1027400090939108809390088381992787FD9095B5
:1027500090939308809392088481992787FD9095A0
:1027600090939508809394088581992787FD90958B
:1027700090939708809396088681992787FD909576
:1027800090939908809398088781992787FD909561
:1027900090939B0880939A088085992787FD909550
:1027A00090939D0880939C088185992787FD90953B
:1027B00090939F0880939E088285992787FD909526
:1027C0009093A1088093A0088385992787FD909511
:1027D0009093A3088093A20810C1E091EE02F091BB
:1027E000EF0280810E94A5378A83882319F481E053
:1027F000898301C01982809106018823E1F388E072
:1028000090E09F938F9389E098E09F938F9321E0CE
:1028100030E03F932F938091EE029091EF029F93CF
:102820008F933F932F93CE0102969F938F933F9365
:102830002F93CE01820F931F9F938F9384E08F93EA
:1028400081E08F9385E58F930E94A210EDB7FEB7CC
:1028500073963CC08091ED02893008F4CEC020917F
:10286000EE023091EF022F5F3F4F88E0A9E0B8E021
:10287000F90101900D928A95E1F7D9018E910E949C
:10288000FB368A83882319F481E0898301C0198289
:10289000809106018823E1F321E030E03F932F93FC
:1028A000CE0102969F938F933F932F93CE01820F79
:1028B000931F9F938F9382E08F9381E08F9387E59F
:1028C0008F930E94A210EDB7FEB73B96EDBF95C067
:1028D0008091A603882309F090C00E94CA9389833F
:1028E000823019F0843009F088C020E430E0F89498
:1028F0008091C1008F738093C1008091C9008F7354
:102900008093C9008091C100877E8093C10080912F
:10291000C900877E8093C9008091C80087FF03C0EB
:102920008091CE00F9CF8091C00087FF03C08091D5
:10293000C600F9CFE091EE02F091EF02E081E130C4
:1029400021F482E08093E2022EC0E43611F421E803
:1029500030E081E08093E202832F99278093CD00BD
:102960002093CC008091CD008093C5008091CC0055
:102970008093C4008091CA008F7D8093CA008091AB
:10298000CA008F7E8093CA008091C9008B7F80939C
:10299000C9008091CA0084608093CA008091CA00F7
:1029A00082608093CA008091CA00877F8093CA00AA
:1029B0008091C200877F8093C2008091C9008E7F82
:1029C0008093C9008091C10088618093C10080918B
:1029D000C90088618093C9008091C100806880939C
:1029E000C1008091C90080688093C90010926E0078
:1029F00010926F0010927000789480913905992799
:102A00008436910509F4BBC085369105ACF4813656
:102A1000910509F46FC0823691052CF48B34910531
:102A200009F45DC00FC18236910509F470C0833688
:102A3000910509F47FC006C18C36910509F4EDC0FB
:102A40008D3691054CF48736910509F4F8C0883627
:102A5000910509F4B2C0F6C08437910529F0863794
:102A6000910509F4E8C0EEC08091F002A091EE0259
:102A7000B091EF02803140F080E1E2E1F5E00D90AD
:102A800001928A95E1F70DC08D919D910D90BC91B9
:102A9000A02D8093120590931305A0931405B09375
:102AA0001505809106018823E1F31F9280910301AF
:102AB0008F9384E58F930E94A2108AEF8093EB029C
:102AC0008FEF8093040180EA9FE00E942C1A90937C
:102AD000E4028093E3020F900F900F90B3C0E09157
:102AE000EE02F091EF028081918190938B018093AF
:102AF0008A01A8C0E091EE02F091EF0280818093FC
:102B00000501803298F08FE1809305010FC0A091FC
:102B1000EE02B091EF028BE0EAE2F5E00D90019257
:102B20008A95E1F7809133058093D9068FEF8093E2
:102B3000040188C08091E7029091E802892B89F412
:102B4000E091EE02F091EF02E081EE2351F08AE095
:102B5000E89FC00111240E942C1A909305058093D0
:102B60000405E091EE02F091EF0290818AE0989FD7
:102B7000C00111249093E8028093E70215C08FEF03
:102B800080930401E091EE02F091EF0290818AE0DF
:102B9000989FC00111249093EA028093E902892B47
:102BA00019F081E08093F80280EA9FE00E942C1ADD
:102BB0009093E4028093E30245C08FEF8093040179
:102BC000E091EE02F091EF02908197FD08C082E063
:102BD0008093F5021092E6021092E5021AC09095D9
:102BE00080914F03892B80934F0391818AE0989FB6
:102BF000C00111249093E6028093E50284E0809363
:102C0000F50280EA9FE00E942C1A9093E4028093E0
:102C1000E30281E08093F90215C08FEF80930401F5
:102C2000E091EE02F091EF0280818093500381E009
:102C30008093FA0207C081E08093F70203C081E02D
:102C40008093FB021092F3021092EF021092EE02B8
:102C50001092ED02E3E0CE5F0C946699982F80917C
:102C6000C00085FFFCCF9093C60008950F931F937B
:102C700088E18093C1008091C00082608093C00091
:102C80008091C10080688093C1008091C100806400
:102C90008093C10000E010E00093C5008AE290E05C
:102CA0008093C4008091E9029091EA020E942C1A5C
:102CB00090930705809306058CED90E00E942C1AF6
:102CC0009093360580933505109208058AE5809328
:102CD000090586E080930C058BE080930A0510922D
:102CE0000B051093EF020093EE021092ED021F917C
:102CF0000F910895A0E1B0E0E0E8F6E10C94479967
:102D000080910601882309F4C1C28091E302909169
:102D1000E4020E94351A882361F01092E6021092B4
:102D2000E5021092EA021092E9021092E802109273
:102D3000E7028091E5029091E602892B41F08091B3
:102D4000E6059091E7050E94351A882329F48091C1
:102D5000F902882309F460C080910601882309F4F0
:102D60005BC08091F5020DEE16E08430A8F00E9461
:102D70006F2580E590E09F938F931F930F9381E0E1
:102D80008F938F9388E48F930E94A2102DB73EB744
:102D9000295F3F4F2DBF34C0109251038FE494E060
:102DA0009F938F9382E695E29F938F93E091F40433
:102DB000F091F504099584E190E09F938F931F9320
:102DC0000F9381E090E09F938F9385EF92E09F9324
:102DD0008F9382E08F9381E08F9388E48F930E949A
:102DE000A2108091F502982F8F5F8093F5022DB786
:102DF0003EB7215F3F4F2DBF943010F01092F50287
:102E00008091E5029091E6020E942C1A9093E705CA
:102E10008093E6051092F9028091FA02882351F11D
:102E200080910601882331F10E946F2580E590E0B2
:102E30009F938F938DEE96E09F938F9321E030E0E8
:102E40003F932F9381E291E09F938F933F932F9332
:102E500080E593E09F938F9383E08F9381E08F933E
:102E60008CE48F930E94A2101092FA028DB79EB745
:102E70000F968DBF8091F7028823D1F080910601D3
:102E80008823B1F08AE090E09F938F9388E095E0EB
:102E90009F938F9381E08F938F9386E58F930E940A
:102EA000A2101092F7022DB73EB7295F3F4F2DBFFA
:102EB0008091FB028823D9F0809106018823B9F024
:102EC0008BE090E09F938F938AE295E09F938F939E
:102ED00081E08F93809103018F9387E48F930E9409
:102EE000A2101092FB028DB79EB707968DBF8091FE
:102EF0003505909136050E94351A882309F461C082
:102F000080910601882309F45CC080915A079927B3
:102F1000880F991F880F991F7C010027F7FC0095E7
:102F2000102F8091010490910204A0910304B091AC
:102F30000404BC01CD01A80197010E94209930939F
:102F40002305209322058091F9039091FA03A09123
:102F5000FB03B091FC03BC01CD01A80197010E94C5
:102F60002099309325052093240580918403809334
:102F70002605809183038093270588E090E09F9346
:102F80008F9382E295E09F938F9381E08F9383E00C
:102F90008F938BE68F930E94A210809128052DB706
:102FA0003EB7295F3F4F2DBF853018F086E08093F4
:102FB000280583E690E00E942C1A909336058093B2
:102FC00035058091E9029091EA02892B41F08091C8
:102FD0000605909107050E94351A882321F48091F7
:102FE000F802882339F180910601882319F10E94A3
:102FF0004D3982E490E09F938F9387E996E09F9309
:103000008F9381E08F938F9384E48F930E94A2101B
:103010001092F8028DB79EB707968DBF8091E90296
:103020009091EA02009731F00E942C1A90930705C4
:10303000809306058091E7029091E802892B09F4BC
:10304000B8C080910405909105050E94351A882327
:1030500009F4AFC080910601882309F4AAC08091C9
:103060005A079927880F991F880F991F7C010027FD
:10307000F7FC0095102F8091010490910204A0911B
:103080000304B0910404BC01CD01A80197010E9482
:1030900020993093F7042093F6048091F9039091DE
:1030A000FA03A091FB03B091FC03BC01CD01A80180
:1030B00097010E9420993093F9042093F8042091FD
:1030C0003D0930913E0940913F0950914009DA0194
:1030D000C90163E0880F991FAA1FBB1F6A95D1F72A
:1030E000820F931FA41FB51F820F931FA41FB51F2C
:1030F00020913C0130913D0140913E0150913F01B2
:10310000BC01CD010E9420993093FB042093FA0466
:103110008091C9039091CA03A091CB03B091CC03D5
:1031200049E0B595A795979587954A95D1F78093EE
:10313000FC048091C5039091C603A091C703B09190
:10314000C80339E0B595A795979587953A95D1F736
:103150008093FD048091D1039091D203A091D30379
:10316000B091D40329E0B595A795979587952A95B1
:10317000D1F78093FE048EE090E09F938F9386EFCB
:1031800094E09F938F9381E08F938F9383E48F9349
:103190000E94A2108091E7029091E8020E942C1AEE
:1031A00090930505809304052DB73EB7295F3F4FE7
:1031B0002DBF809105018F3F71F1992704E0880FA1
:1031C000991F0A95E1F7815B9D4F40E150E0BC01FA
:1031D000CE0101960E94F69680E190E09F938F9336
:1031E000CE0101969F938F9381E090E09F938F9300
:1031F00085E091E09F938F9382E08F9381E08F939E
:1032000081E48F930E94A2108FEF809305018DB708
:103210009EB70B968DBF8091D9068823D1F08091FF
:1032200006018823B1F081E090E09F938F9389EDB0
:1032300096E09F938F9381E08F938F9382E48F9397
:103240000E94A2101092D9062DB73EB7295F3F4FBA
:103250002DBF8091F6028823C9F080910601882352
:10326000A9F084E390E09F938F9382E798E09F9387
:103270008F9381E08F938F9380E58F930E94A210AC
:103280001092F6028DB79EB707968DBFE6E0C05F3D
:103290000C9463991F920F920FB60F9211242F93E3
:1032A0003F935F936F937F938F939F93AF93BF935E
:1032B000EF93FF9380910B03882329F080910B03F8
:1032C000815080930B0380919704882319F08150DB
:1032D00080939704809113038150809313038F3F51
:1032E00009F04BC089E08093130380911103909102
:1032F00012030196909312038093110380911001A1
:103300008F5F817080931001882319F481E080938E
:103310001003349903C081E08093140380910C035F
:1033200090910D03892B11F180910C0390910D0365
:103330000B9750F080910C0390910D030A97909396
:103340000D0380930C0304C010920D0310920C0324
:1033500080910C0390910D032091090130910A0195
:1033600082239323892B41F0479A07C08FEF9FEF69
:1033700090930A0180930901479880911403882350
:1033800009F45AC020919901222309F055C0809177
:103390002D0983FF51C086B19927FC01E071F070BF
:1033A00084FF13C080910E0390910F0301969093B8
:1033B0000F0380930E0380910E0390910F03895E9B
:1033C0009340D0F12093140337C080910E03909165
:1033D0000F03892B69F180910E0390910F038A5698
:1033E000914030F580910E0390910F0369E270E0F7
:1033F0000E94D79880910E0390910F03860F971F1C
:1034000090930F0380930E0380910E0390910F030E
:103410000B9750F080910E0390910F030A979093B1
:103420008B0180938A0104C0F0938B01E0938A01A1
:1034300010920F0310920E03FF91EF91BF91AF9185
:103440009F918F917F916F915F913F912F910F90FD
:103450000FBE0F901F901895209111033091120309
:10346000280F391FC9010196089520911103309149
:103470001203821B930B892F992786958074907075
:103480000895CF93DF930E942C1AEC01CE010E9485
:10349000351A8823D9F3DF91CF910895CF93DF9325
:1034A0000E942C1AEC0109C080911101882329F097
:1034B000909311018FEC80937A00CE010E94351A0F
:1034C000982F882389F3DF91CF9108959FB7F894BF
:1034D0005F983E9A469A8091B0008F708093B000BA
:1034E0008091B00083608093B0008091B1008B73B5
:1034F0008093B1008091B1008B608093B1001092F5
:10350000B2008FEF8093B3008091B0008068809309
:10351000B000809170008A7F80937000809170006D
:103520008260809370009FBF08958AE090E00E94BF
:103530002C1A9093DB068093DA0682E085BD83EA3D
:1035400084BD17BC84EB88BD86E086BD80916E008B
:10355000816080936E0008958091AB07209169018E
:1035600082FF30C090916E078CE3989FB0011124C8
:1035700090916D0780E5989FA0011124922F90589B
:1035800097FD9D5F9595959586E09802C001112461
:103590002091070130910801281B390B3093080155
:1035A00020930701421753072CF0509308014093D2
:1035B000070108952617370784F070930801609378
:1035C00007010895822F992736E0880F991F3A95B1
:1035D000E1F790930801809307010895A0E0B0E01F
:1035E000E4EFFAE10C94469980917507E82FFF27E4
:1035F000EE5BFE4F9681D08080910F01A92FBB27F3
:10360000A7FDB095CB2FDB2F813009F017C120919A
:103610000104309102044091030450910404BD015F
:10362000CE010E94AC9897FF04C061587F4F8F4F26
:103630009F4F7B018C01C7E015950795F794E794A0
:10364000CA95D1F78D2D992787FD9095A92FB92F70
:103650002091F9033091FA034091FB035091FC0350
:10366000BC01CD010E94AC9897FF04C061587F4F08
:103670008F4F9F4FB7E09595879577956795BA954A
:10368000D1F7F801E701C61BD70BE80BF90B209126
:103690007E0430917F04C901A3E0880F991FAA9589
:1036A000E1F7821B930BAA2797FDA095BA2FC81BA1
:1036B000D90BEA0BFB0B809167019927AA27BB273F
:1036C000BC01CD019E01AF010E94AC9897FF04C0E0
:1036D00061507E4F8F4F9F4FFC01EB0179E0F595D4
:1036E000E795D795C7957A95D1F71091AB0760917B
:1036F00007017091080112FF05C070930E016093DD
:103700000D0118C040910D0150910E018091740778
:10371000282F3327CB01841B950BB9010E94EB980E
:1037200080910D0190910E01860F971F90930E01CD
:1037300080930D0110FF14C080910D0190910E0136
:1037400097FD0F9664E0959587956A95E1F7AA270E
:1037500097FDA095BA2FC80FD91FEA1FFB1F15C0F0
:1037600080910D0190910E0197FD0F9654E0959573
:1037700087955A95E1F7AA2797FDA095BA2F8C1B3C
:103780009D0BAE0BBF0BFD01EC012091A80722237E
:1037900021F133278091060390910703829FA001B6
:1037A000839F500D929F500D1124CA01AA2797FDA7
:1037B000A095BA2F8C0F9D1FAE1FBF1F2F5F3F4FCD
:1037C000442737FD4095542FBC01CD010E9420991C
:1037D000309307032093060304C0D0930703C093DC
:1037E000060380916D07282F3327220F331F220FE6
:1037F000331F8091060390910703821793077CF093
:1038000080916E07282F3327220F331F220F331F7B
:1038100080910603909107032817390724F4309309
:1038200007032093060380910101843108F4F7C057
:1038300080910F018F5F80930F01F3C02091F903F6
:103840003091FA034091FB035091FC03BD01CE017E
:103850000E94AC9897FF04C061587F4F8F4F9F4FD5
:103860007B018C0187E015950795F794E7948A957D
:10387000D1F78D2D992787FD9095A92FB92F2091EC
:103880000104309102044091030450910404BC01EE
:10389000CD010E94AC989B01AC0197FF04C0215858
:1038A0003F4F4F4F5F4FC7E0559547953795279549
:1038B000CA95D1F72E0D3F1D401F511F8091660103
:1038C0009927AA27BB27BC01CD010E94AC9897FF7E
:1038D00004C061507E4F8F4F9F4FFC01EB01B9E058
:1038E000F595E795D795C795BA95D1F78091680179
:1038F0009927A6E0880F991FAA95E1F740910B013F
:1039000050910C01209174073327841B950BB9014A
:103910000E94EB9880910B0190910C01860F971FEC
:1039200090930C0180930B018091AB0781FF14C031
:1039300080910B0190910C0197FD0F9674E0959585
:1039400087957A95E1F7AA2797FDA095BA2FC80F1A
:10395000D91FEA1FFB1F15C080910B0190910C012C
:1039600097FD0F9664E0959587956A95E1F7AA27EC
:1039700097FDA095BA2F8C1B9D0BAE0BBF0BFD01C5
:10398000EC012091A907222321F133278091040320
:1039900090910503829FA001839F500D929F500D2F
:1039A0001124CA01AA2797FDA095BA2F8C0F9D1F3D
:1039B000AE1FBF1F2F5F3F4F442737FD4095542F49
:1039C000BC01CD010E94209930930503209304038C
:1039D00004C0D0930503C093040380917107282F7E
:1039E0003327220F331F220F331F8091040390913E
:1039F0000503821793077CF080917207282F3327E5
:103A0000220F331F220F331F80910403909105036F
:103A10002817390724F430930503209304031092E8
:103A20000F01E7E0CDB7DEB70C9462991F920F92B9
:103A30000FB60F9211242F933F934F935F938F9361
:103A40009F93EF93FF93809101019091150384312F
:103A500008F04CC0992309F029C18091B00086FF7D
:103A600024C08091B0008F7B8093B00080910603CA
:103A70009091070387559E4F909309038093080305
:103A800025E08D3D920718F08CED95E005C0875735
:103A9000914030F487E791E0909309038093080305
:103AA0008091080390910903C2C08091B0008064A6
:103AB0008093B00080917307282F33278DED96E017
:103AC000289FA001299F500D389F500D1124CA0135
:103AD0002091160330911703821B930B90930903D7
:103AE0008093080381E080930F01DDC0992309F0E2
:103AF000DDC08091B00086FF9FC08091B0008F7BB9
:103B00008093B000E091180320917307EE23D9F45D
:103B100033278DED96E0289FA001299F500D389FF7
:103B2000500D1124CA012091160330911703821BF6
:103B3000930B90930903809308031092170310923C
:103B40001603469AB0C02E1738F48AE090E090939E
:103B5000090380930803A7C089EA93E090930903BF
:103B6000809308038E2F992783309105D9F08430F4
:103B7000910534F48130910549F0029761F020C03D
:103B80008430910591F0059799F01AC08091060351
:103B90009091070304C08091040390910503875519
:103BA0009E4F1DC08091090905C08091E00802C0A8
:103BB000809112099927880F991F880F991FEFCFBD
:103BC000FF27EE0FFF1FEE58F74F20813181220FA4
:103BD000331F8091080390910903820F931F9093E4
:103BE000090380930803809108039091090355E02D
:103BF0008D3D950718F08CED95E005C087579140F5
:103C000030F487E791E090930903809308032091B3
:103C10000803309109032C5B304030930903209353
:103C200008038091160390911703820F931F9093BE
:103C300017038093160337C08091B000806480938F
:103C4000B0008CEB90E0909309038093080380917F
:103C500016039091170384549F4F909317038093FA
:103C6000160380910A03882321F08091A7038823FB
:103C700021F480910A03823011F4469801C0469ADB
:103C8000809118038F5F80931803282F332780912A
:103C9000730799270196821793072CF481E080938C
:103CA0000F011092180381E08093150320910803FF
:103CB0003091090341E02F37340730F08FEF8093C4
:103CC000B3002F5F30400FC02F3F3105C9F0C0F067
:103CD000A9014F5F50404F37510550F480E8809361
:103CE000B30020583040309309032093080312C0DA
:103CF0008FEF8093B30050930903409308030AC0E9
:103D0000809108038093B300109209031092080376
:103D100010921503FF91EF919F918F915F914F91B9
:103D20003F912F910F900FBE0F901F9018951092FA
:103D30007C008FEC80937A000895CF93DF931092EC
:103D4000210386E987BD83E090E00E94F230C82F0E
:103D5000863E08F4C65FC8BD84E690E00E944E1A15
:103D600080911501909116018152934010F0C0EF9F
:103D700002C0C530F8F0C8BD82E390E00E944E1A40
:103D800084E694E09F938F938EE296E19F938F93C6
:103D9000E091F404F091F50409958091150190915A
:103DA00016010F900F900F900F908152934010F4D6
:103DB000C550DFCF6C2F83E090E00E94FA30CF3007
:103DC00018F0CCE8D0E002C0C0E0D0E0CA3FD10596
:103DD000F8F4C7BD82E390E00E944E1A86E694E0B4
:103DE0009F938F938EE296E19F938F93E091F404DB
:103DF000F091F504099580911501909116010F90AD
:103E00000F900F900F908052934010F02196DECFCC
:103E1000C093EA0680914B0780FF09C08C2F8A501F
:103E20008B3E28F080910D05806480930D05C7BD01
:103E30008CE291E00E944E1ADF91CF910895EF92AB
:103E4000FF921F93CF9310E080ED97E00E942C1A11
:103E50007C01CCE8133019F4CB3008F0C9E010E055
:103E600080913003909131038C5F934024F48091D2
:103E7000140181500AC08091300390913103875022
:103E8000944034F0809114018F5F8093140101C03D
:103E900011E080912E0390912F038C5F934024F4C6
:103EA0008091130181500AC080912E0390912F03BD
:103EB0008750944034F0809113018F5F80931301F9
:103EC00001C01F5F80912C0390912D038C5F934064
:103ED00024F48091120181500AC080912C039091AA
:103EE0002D0387509440C4F0809112018F5F80931E
:103EF000120113C088E694E09F938F938EE296E1BF
:103F00009F938F93E091F404F091F50409950F903D
:103F10000F900F900F905FC01F5F82E180935C0352
:103F2000809156038E7F8093560385EA8093BC0070
:103F3000809114018A3040F480910D058160809356
:103F40000D058AE08093140180911401863F40F0B2
:103F500080910D05816080930D0585EF809314019C
:103F6000809113018A3040F480910D058260809326
:103F70000D058AE08093130180911301863F40F084
:103F800080910D05826080930D0585EF809313016C
:103F9000809112018A3040F480910D0584608093F5
:103FA0000D058AE08093120180911201863F40F056
:103FB00080910D05846080930D0585EF809312013B
:103FC00080915C03882339F0C7010E94351A882349
:103FD00009F090CFF5CF109211018FEC80937A0009
:103FE000809111018823E1F3CA3020F48AE090E047
:103FF0000E944E1AC15009F02DCF86E490E00E9435
:104000004E1ACF911F91FF90EF9008951F920F923B
:104010000FB60F921124EF92FF920F931F932F93DD
:104020003F934F935F936F937F938F939F93AF9340
:10403000BF93EF93FF9380913903282F33274427B1
:1040400055278F5F80933903F9012231310508F03C
:104050000BC5EA5BFF4F0C947299809178009091A8
:10406000790046C08091780090917900B8C1809124
:1040700078009091790090933D0380933C03E3C1D5
:1040800080910B0490910C0420917800309179007C
:10409000821B930B9093DD068093DC068091DC06F7
:1040A0009091DD069093470380934603EAC1809187
:1040B00078009091790020910D0430910E04821BBC
:1040C000930B9093E9068093E8068091E80690911F
:1040D000E9069093490380934803C8C48091400344
:1040E000909141032091780030917900820F931FC5
:1040F000909341038093400381E0B9C480913E03D3
:1041000090913F032091780030917900820F931FA6
:1041100090933F0380933E0384E0A9C48091AC0751
:1041200083FF1AC080911F01909120019C01220FF2
:10413000331F280F391F40917800509179008BE090
:1041400090E0489FB001499F700D589F700D112459
:10415000CB016EE170E00FC080911F0190912001B2
:104160009C01220F331F280F391F809178009091F6
:10417000790063E070E00E94D798260F371F3695CC
:104180002795369527953093200120931F0185E0D0
:104190006EC480917800909179009093DF068093AF
:1041A000DE068091DE069091DF0640910704509173
:1041B0000804841B950B60910604262F332727FDE6
:1041C0003095821B930B9093270380932603809155
:1041D0006703882309F071C080912603909127031B
:1041E00002977CF172E04E3E57070CF0A7C0209179
:1041F0003A0330913B032B5F3F4F30933B032093B7
:104200003A03255030408091700390917103845F90
:10421000914030F4215F3F4F30933B0320933A03AA
:1042200080913A0390913B03853691050CF486C04A
:104230004F5F5F4F509308044093070484569040AB
:1042400037C080912603909127038F5F9F4F0CF01A
:1042500075C082E0473258070CF470C020913A03D1
:1042600030913B032550304030933B0320933A0379
:104270002B5F3F4F8091700390917103845F914059
:1042800030F42F50304030933B0320933A03809119
:104290003A0390913B037FEF8C3997070CF04EC0A7
:1042A0004150504050930804409307048C599F4F4D
:1042B00090933B0380933A0341C08091FE08909114
:1042C000FF088F5C9F41D4F18091260390912703D2
:1042D0000297ACF020913A0330913B03C90101965B
:1042E00090933B0380933A03895893413CF16630A5
:1042F0001CF46F5F60930604275833411BC0809104
:104300002603909127038F5F9F4FC4F420913A03B7
:1043100030913B03C901019790933B0380933A038B
:1043200088579C4E5CF46B3F1CF061506093060410
:1043300029573C4E30933B0320933A038091260348
:10434000909127039C01442737FD4095542F80917D
:10435000C1039091C203A091C303B091C403820F23
:10436000931FA41FB51F8093C1039093C203A09312
:10437000C303B093C4032091C1033091C2034091A1
:10438000C3035091C40357FF04C021503C4F4F4F0B
:104390005F4F7AE055954795379527957A95D1F7F0
:1043A0008091C1039091C203A091C303B091C40353
:1043B000821B930BA40BB50B8093C1039093C20394
:1043C000A093C303B093C4032EC180913E03909188
:1043D0003F032091780030917900820F931F9093D2
:1043E0003F0380933E031092380343C38091010141
:1043F0008A3071F4809178009091790020913C038B
:1044000030913D03820F931F01969695879517C0B3
:1044100040913C0350913D03843158F02091780045
:1044200030917900240F351F8FEF97E0821B930B9B
:1044300006C08091780090917900840F951F909329
:104440002D0380932C0386E012C380910B0490917E
:104450000C042091780030917900821B930B90938B
:10446000DD068093DC068091DC069091DD062091CC
:10447000460330914703820F931F90932B03809341
:104480002A0387E0F4C2809178009091790020910E
:104490000D0430910E04821B930B9093E9068093D8
:1044A000E8068091E8069091E90620914803309152
:1044B0004903820F931F9093290380932803D6C248
:1044C00020914003309141038091780090917900D0
:1044D000280F391F3093410320934003809101013D
:1044E0008A3019F4220F331F04C0220F331F220F0A
:1044F000331F3093410320934003209140033091B8
:104500004103C90137FD079643E0959587954A9584
:10451000E1F79093310380933003809142039091AF
:104520004303820F931F97FD01969595879590936E
:104530004303809342032091170430911804821B97
:10454000930B90931E0180931D01209136033091AF
:10455000370380911D0190911E01280F391F37FFED
:1045600002C02F5F3F4F3595279530933703209337
:104570003603C2CD20913E0330913F0380917800F5
:1045800090917900280F391F30933F0320933E0309
:10459000809101018A3019F4220F331F04C0220FC9
:1045A000331F220F331F30933F0320933E0320918C
:1045B0003E0330913F03C90137FD0796B3E095955F
:1045C0008795BA95E1F790932F0380932E038091FE
:1045D000440390914503820F931F97FD0196959593
:1045E000879590934503809344032091150430915F
:1045F0001604821B930B90931C0180931B01209146
:1046000034033091350380911B0190911C01280FD8
:10461000391F37FF02C02F5F3F4F359527953093E5
:1046200035032093340383E022C2809167038823FB
:1046300009F180E00E949F929B01AC0120503F4F06
:104640004F4F5F4F57FF06C09B01AC0121503D4FBC
:104650004F4F5F4FE9E05595479537952795EA9578
:10466000D1F72093190330931A0340931B035093FF
:104670001C0310C08091A1039091A203A091A303F9
:10468000B091A4038093190390931A03A0931B0382
:10469000B0931C031092390381E080931101809143
:1046A0001D0390911E03019690931E0380931D039A
:1046B0008091780090917900909316018093150174
:1046C00080916703882309F47EC080911501909141
:1046D00016017C010027112780912103992787FD6E
:1046E0009095A92FB92FBC01CD012BE032E040E01D
:1046F00050E00E94AC98DC01CB01E81AF90A0A0BE1
:104700001B0BE0924A03F0924B0300934C0310936F
:104710004D032091170130911801409119015091DA
:104720001A0157FF04C0215F3F4F4F4F5F4F74E0A6
:1047300055954795379527957A95D1F7809117012B
:1047400090911801A0911901B0911A01821B930B4D
:10475000A40BB50B8093170190931801A093190136
:10476000B0931A018091170190911801A09119013D
:10477000B0911A018E0D9F1DA01FB11F80931701CC
:1047800090931801A0931901B0931A018091E0064B
:104790009091E106A091E206B091E3062091170105
:1047A000309118014091190150911A01821B930B0D
:1047B000A40BB50B8093A1039093A203A093A30332
:1047C000B093A40353C18091150190911601AA27BB
:1047D000BB2720914A0330914B0340914C035091E9
:1047E0004D03280F391F4A1F5B1F20934A03309344
:1047F0004B0340934C0350934D0380914E038F5FC6
:1048000080934E03803108F431C18091170190915B
:104810001801A0911901B0911A017C018D0163E08A
:10482000EE0CFF1C001F111F6A95D1F7E81AF90A58
:104830000A0B1B0BE20EF31E041F151F80912103B0
:10484000992787FD9095A92FB92FBC01CD0120EBA9
:1048500030E240E050E00E94AC98DC01CB01E81A65
:10486000F90A0A0B1B0BD801C7010496A11DB11D43
:10487000B7FF05C0D801C7010B96A11DB11D23E0EC
:10488000B595A795979587952A95D1F780931701A8
:1048900090931801A0931901B0931A01E090E006DB
:1048A000F090E1060091E2061091E3068091170175
:1048B00090911801A0911901B0911A01E81AF90A12
:1048C0000A0B1B0BE092A103F092A2030093A30337
:1048D0001093A403209122033091230340912403D9
:1048E0005091250357FF04C0215F3F4F4F4F5F4F4B
:1048F00084E055954795379527958A95D1F780910E
:10490000220390912303A0912403B0912503821BDD
:10491000930BA40BB50B8093220390932303A093D6
:104920002403B09325038091220390912303A09147
:104930002403B09125038E0D9F1DA01FB11F8093EE
:10494000220390932303A0932403B0932503809123
:10495000220390912303A0912403B0912503B7FF74
:1049600003C00F96A11DB11D14E0B595A7959795AD
:1049700087951A95D1F72091A1033091A203281BA6
:10498000390B64E0213036071CF020E034E006C02B
:104990007CEF2030370714F420E03CEF80911F03B8
:1049A0009091200380911F039091200397FF03C0F3
:1049B000909581959F4FA901F3E0440F551FFA95FB
:1049C000E1F78D5B9240C4F080911F03909120032A
:1049D0009C01E4E0220F331FEA95E1F7281B390B15
:1049E000240F351F37FF02C0215F3F4F74E035951C
:1049F00027957A95E1F717C080911F0390912003C6
:104A00009C0165E0220F331F6A95E1F7281B390BE3
:104A1000240F351F37FF02C0215E3F4F45E035951B
:104A200027954A95E1F73093200320931F03809147
:104A30004A0390914B03A0914C03B0914D03B7FFF3
:104A400003C00196A11DB11DB595A79597958795B2
:104A500080934A0390934B03A0934C03B0934D0370
:104A600088E080934E0302C01092390382E0809365
:104A700038038091380380937C0080913903882328
:104A800019F08FEC80937A00FF91EF91BF91AF9175
:104A90009F918F917F916F915F914F913F912F9156
:104AA0001F910F91FF90EF900F900FBE0F901F90EE
:104AB000189590E2EDEEF6E08FE49193815087FF38
:104AC000FCCF089590915103903540F4E92FFF27D2
:104AD000E351F94F80839F5F909351030895AF9204
:104AE000BF92CF92DF92FF920F931F93CF93DF93EA
:104AF00020914F0320FF0AC080915003882311F0BA
:104B0000815002C0809121018093500321FF0CC08D
:104B10009091500380912101981719F4109250033D
:104B200003C09F5F90935003822F992780FF04C09A
:104B300081FF02C0109250030E94592580915003BA
:104B4000282F332792E6C92E95E2D92EC091F4047E
:104B5000D091F5048A3098F481E1809351033F931A
:104B60002F938FE994E09F938F93DF92CF92FE0172
:104B700009952DB73EB72A5F3F4F2DBF11C080E189
:104B8000809351033F932F9384EA94E09F938F93F4
:104B9000DF92CF92FE0109958DB79EB706968DBF25
:104BA00020915003822F9927AA27BB27FC01419708
:104BB00010F00C94D72EE85AFF4F02E6C02E05E203
:104BC000D02EC091F404D091F5040C9472991092F7
:104BD000510389EA94E09F938F9302E615E2DF92F6
:104BE000CF92FE01099584E1809351030F900F90BD
:104BF0000F900F9087E690E09F938F938AE590E067
:104C00009F938F931F921F92809101016AE00E94EF
:104C1000CB98892F99279F938F93809101010E94B0
:104C2000CB9899279F938F9389EB94E09F938F93D1
:104C3000DF92CF92E091F404F091F504099588E2B7
:104C400080935103EDB7FEB73E96EDBF8CEB97E036
:104C50009F938F930E946E3299279F938F9381ED3C
:104C600094E09F938F93DF92CF92E091F404F091C0
:104C7000F504099580910E0599272DB73EB7285F59
:104C80003F4F2DBFEC01C071D07084FF06C08CE394
:104C9000809351038FED94E00AC19091850499238C
:104CA00059F18CE380935103892F99279F938F9318
:104CB0008CEE94E09F938F931F930F93E091F404F5
:104CC000F091F5040995DF93CF939091850481E1EC
:104CD000989FC0011124865A944F9F938F931F93DE
:104CE0000F93E091F404F091F50409958DB79EB708
:104CF0000C968DBF0C94E02E90910D05992351F0E8
:104D00008CE380935103892F99279F938F9384EF8E
:104D100094E044C190915703992371F08CE3809300
:104D20005103892F99279F938F938BE095E09F9351
:104D30008F931F930F93F3C48091360190913701A5
:104D4000069710F00C94E02E8CE38093510380E2E0
:104D500095E0BFC780912D0912E6C12E15E2D12E34
:104D6000C091F404D091F50480FF8EC010925103DD
:104D70008091A1039091A203A091A303B091A403F9
:104D8000BC01CD0125E030E040E050E00E942099D8
:104D90003F932F938DE295E09F938F93DF92CF9275
:104DA000FE01099584E1809351038DB79EB7069665
:104DB0008DBF80919D0390919E03A0919F03B09120
:104DC000A003BC01CD0125E030E040E050E00E94AE
:104DD00020993F932F938AE395E09F938F93DF92DF
:104DE000CF92E091F404F091F504099588E2809364
:104DF0005103EDB7FEB73696EDBF80911501909146
:104E000016019F938F9387E495E09F938F93DF9292
:104E1000CF92E091F404F091F50409958CE380932E
:104E200051032DB73EB72A5F3F4F2DBF87B5992756
:104E30009F938F9384E595E09F938F93DF92CF921A
:104E4000E091F404F091F50409958DB79EB70696AC
:104E50008DBF80916703882309F4B2C78DE48093E6
:104E6000510387B599279F938F9381E695E09F9390
:104E70008F93DF92CF92E091F404F091F5040995BD
:104E8000EDB7FEB73696D9C31092510385E695E08B
:104E90009F938F93DF92CF92FE01099584E18093D7
:104EA00051030F900F900F900F9084E795E09F9320
:104EB0008F93DF92CF9211C7109251038DE795E047
:104EC0009F938F9302E615E2DF92CF92FE01099540
:104ED00084E1809351030F900F900F900F90809179
:104EE000010490910204A0910304B0910404B7FF5F
:104EF00004C081509C4FAF4FBF4FCAE0B595A795F6
:104F000097958795CA95D1F7BF93AF939F938F934A
:104F10008AE895E09F938F931F930F93E091F40499
:104F2000F091F504099588E2809351032DB73EB7BF
:104F3000285F3F4F2DBF8091F9039091FA03A09114
:104F4000FB03B091FC03B7FF04C081509C4FAF4FEF
:104F5000BF4FFAE0B595A79597958795FA95D1F744
:104F6000BF93AF939F938F9389E995E09F938F931E
:104F70001F930F93E091F404F091F50409958CE3ED
:104F8000809351038DB79EB708968DBF8091E80836
:104F90009091E9089F938F9388EA95E09F938F9370
:104FA0001F930F9368CFE1E0FE2EC1E0D0E004E74D
:104FB00018E09F2D969584E1989FC001112480935D
:104FC0005103F801828193819F938F932196DF9300
:104FD000CF932197808191819F938F93DF93CF937C
:104FE00087EB95E09F938F9382E695E29F938F9353
:104FF000E091F404F091F50409952DB73EB7245FD4
:105000003F4F2DBF32E0F30E22960C5F1F4F88E01A
:105010008F1578F6D5C61092510380914007E82F7E
:10502000FF27EE0FFF1FEE58F74F808191819F936E
:105030008F9380913F07E82FFF27EE0FFF1FEE5859
:10504000F74F808191819F938F9389EC95E09F9397
:105050008F93DF92CF92FE01099584E180935103F3
:10506000EDB7FEB73896EDBF80914207E82FFF27D6
:10507000EE0FFF1FEE58F74F808191819F938F9322
:1050800080914107E82FFF27EE0FFF1FEE58F74FE3
:105090008081918181589F4F9F938F9389ED95E0F7
:1050A0009F938F93DF92CF92E091F404F091F504F7
:1050B000099588E2809351032DB73EB7285F3F4F93
:1050C0002DBF80914407E82FFF27EE0FFF1FEE58FA
:1050D000F74F8081918181589F4F9F938F9380914B
:1050E0004307E82FFF27EE0FFF1FEE58F74F808191
:1050F000918181589F4F9F938F9389EE95E09F9365
:105100008F93DF92CF92E091F404F091F50409952A
:105110008CE3809351038DB79EB708968DBF809125
:105120004607E82FFF27EE0FFF1FEE58F74F80814D
:10513000918181589F4F9F938F9380914507E82FCE
:10514000FF27EE0FFF1FEE58F74F808191818158A6
:105150009F4F9F938F9389EF95E063C21092510305
:1051600089E096E09F938F9302E615E2DF92CF925B
:10517000FE010995809101010F900F900F900F9003
:105180008A3009F09DC084E1809351038091170417
:10519000909118049C0197FF02C0295F3F4F287F20
:1051A000821B930B9F938F93809117049091180407
:1051B00097FD079673E0959587957A95E1F79F930C
:1051C0008F93209117043091180437FF02C0295F94
:1051D0003F4F63E0359527956A95E1F7809130035D
:1051E00090913103821B930B9F938F9387E196E0FD
:1051F0009F938F931F930F93E091F404F091F50424
:10520000099588E2809351032DB73EB7265F3F4F43
:105210002DBF80911504909116049C0197FF02C048
:10522000295F3F4F287F821B930B9F938F93809121
:1052300015049091160497FD079653E09595879570
:105240005A95E1F79F938F9320911504309116049E
:1052500037FF02C0295F3F4F43E0359527954A95B8
:10526000E1F780912E0390912F03821B930B9F9364
:105270008F9388E296E09F938F931F930F93E09113
:10528000F404F091F50409958CE3809351038DB7F4
:105290009EB70A968DBF80911304909114049F933A
:1052A0008F93809113049091140420912C033091DA
:1052B0002D03821B930B9F938F9389E396E0ADC0E0
:1052C0008B3019F0843108F4ADC084E18093510330
:1052D00080911704909118049C0197FF02C0215FF0
:1052E0003F4F207F821B930B97FD019695958795E5
:1052F0009F938F93809117049091180497FD0F96B8
:1053000024E0959587952A95E1F79F938F932091B7
:1053100017043091180437FF02C0295F3F4FC3E0E4
:1053200035952795CA95E1F7809130039091310327
:10533000821B930B9F938F9387E496E09F938F93A9
:105340001F930F93E091F404F091F504099588E21E
:10535000809351032DB73EB7265F3F4F2DBF8091FD
:105360001504909116049C0197FF02C0215F3F4FE6
:10537000207F821B930B97FD0196959587959F93B0
:105380008F93809115049091160497FD0F96A4E0D9
:1053900095958795AA95E1F79F938F932091150492
:1053A0003091160437FF02C0295F3F4FF3E0359577
:1053B0002795FA95E1F780912E0390912F03821B98
:1053C000930B9F938F9389E596E09F938F931F9301
:1053D0000F93E091F404F091F50409958CE3809328
:1053E00051038DB79EB70A968DBF8091130490919B
:1053F000140497FD0196959587959F938F938091BF
:1054000013049091140420912C0330912D03821BDE
:10541000930B9F938F938BE696E09F938F931F93AD
:105420000F9303C18D3009F0CBC484E18093510305
:105430008091140199279F938F93809117049091E5
:10544000180497FD0F9674E0959587957A95E1F786
:105450009F938F93209117043091180437FF02C057
:10546000295F3F4F63E0359527956A95E1F7809175
:10547000300390913103821B930B9F938F938AE7A4
:1054800096E09F938F931F930F93E091F404F09114
:10549000F504099588E2809351032DB73EB7265F46
:1054A0003F4F2DBF8091130199279F938F93809138
:1054B00015049091160497FD0F9654E095958795E5
:1054C0005A95E1F79F938F9320911504309116041C
:1054D00037FF02C0295F3F4F43E0359527954A9536
:1054E000E1F780912E0390912F03821B930B9F93E2
:1054F0008F938EE896E09F938F931F930F93E09185
:10550000F404F091F50409958CE3809351038DB771
:105510009EB70A968DBF8091120199279F938F9312
:10552000809113049091140497FD019695958795A9
:105530009F938F93809113049091140420912C03D6
:1055400030912D03821B930B9F938F9382EA96E0F9
:105550009F938F931F930F93E091F404F091F504C0
:105560000995EDB7FEB73A9668C01092510386EBE5
:1055700096E09F938F93DF92CF92FE01099584E18D
:10558000809351030F900F900F900F9080910D0416
:1055900090910E049F938F938091280390912903FB
:1055A0009F938F9383EC96E09F938F93DF92CF929C
:1055B000E091F404F091F504099588E28093510399
:1055C0002DB73EB7285F3F4F2DBF80910B049091C0
:1055D0000C049F938F9380912A0390912B039F93A8
:1055E0008F9382ED96E09F938F93DF92CF92E0911D
:1055F000F404F091F50409958CE3809351038DB781
:105600009EB708968DBF80910704909108049F93E0
:105610008F9380912603909127039F938F9381EE20
:1056200096E09F938F93DF92CF92E091F404F091F4
:10563000F5040995EDB7FEB73896EDBFC1C31092DA
:10564000510380911F01909120016AE070E00E9457
:10565000EB989F938F9380911F01909120016AE0B6
:1056600070E00E94EB987F936F9380EF96E09F939A
:105670008F93DF92CF92FE01099584E180935103CD
:105680002DB73EB7285F3F4F2DBF8091C209909143
:10569000C3096AE070E00E94D7989F938F9380912E
:1056A000C2099091C3096AE070E00E94D7987F9385
:1056B0006F9384E097E09F938F93DF92CF92E09176
:1056C000F404F091F504099588E2809351038DB7B5
:1056D0009EB708968DBF8091C4099091C5099F938C
:1056E0008F9388E197E09F938F93DF92CF92E09121
:1056F000F404F091F50409958CE380935103EDB720
:10570000FEB73696EDBF8091C6099091C7099F9369
:105710008F9388E297E09F938F93DF92CF92E091EF
:10572000F404F091F50409952DB73EB72A5F3F4F79
:105730004FC1109251038AE397E09F938F93DF92BA
:10574000CF92FE01099584E1809351030F900F9051
:105750000F900F9080917208909173089F938F9390
:1057600083E497E09F938F93DF92CF92E091F404CC
:10577000F091F504099588E2809351038DB79EB7A7
:1057800006968DBF8091A70399279F938F9383E5FA
:1057900097E09F938F93DF92CF92E091F404F09182
:1057A000F50409958CE380935103EDB7FEB7369667
:1057B000EDBF80917108992701979F938F9383E69E
:1057C00097E0A9CF1092510383E797E09F938F93BF
:1057D000DF92CF92FE01099584E1809351030F90EF
:1057E0000F900F900F9080918A0190918B019F9361
:1057F0008F938BE797E09F938F93DF92CF92E09107
:10580000F404F091F504099588E2809351038DB773
:105810009EB706968DBF8091E8089091E9089F9306
:105820008F9389E897E09F938F93DF92CF92E091D7
:10583000F404F091F50409958CE380935103EDB7DE
:10584000FEB73696EDBF8091BF039091C0039F9342
:105850008F9387E997E05FCFC8EACC2EC3E0DC2EB8
:1058600020E030E0E901B3E0FB2EC0935103F601E4
:1058700081916F0199279F938F9389010F5F1F4F2C
:105880001F930F9385EA97E09F938F9382E695E2AB
:105890009F938F93E091F404F091F50409952DB74F
:1058A0003EB7285F3F4F2DBFFA9464969801F7FEEC
:1058B000DCCF86C2ACEACA2EA3E0DA2EC0E0D0E08C
:1058C0008E01F3E0FF2E00935103F60181916F01E9
:1058D00099279F938F932596DF93CF9382EB97E041
:1058E0009F938F9382E695E29F938F93E091F404C8
:1058F000F091F50409952DB73EB7285F3F4F2DBFB6
:10590000FA940C5E1F4F2497F7FEDDCF59C2109218
:1059100051038FEB97E09F938F9302E615E2DF929E
:10592000CF92FE01099584E1809351030F900F906F
:105930000F900F908091690199279F938F9387EC27
:1059400097E09F938F93DF92CF92E091F404F091D0
:10595000F504099588E2809351038DB79EB70696AA
:105960008DBF809106039091070397FD039695954F
:105970008795959587959F938F9385ED97E09F9356
:105980008F931F930F93E091F404F091F504099520
:105990008CE380935103EDB7FEB73696EDBF80914F
:1059A0006E0799279F938F9380916D0799279F93F7
:1059B0008F9383EE97E09F938F931F930F93E091C4
:1059C000F404F091F50409952DB73EB7285F3F4FD9
:1059D0002DBFF6C11092510381EF97E09F938F93F3
:1059E00072E6A72E75E2B72EDF92CF92FE010995DF
:1059F0000F900F900F900F90C1E1D8E000E010E001
:105A000062E0F62E802F8C5E809351038B8D992758
:105A10008F7790709F938F938B8999278F77907052
:105A20009F938F938B8599278F7790709F938F93F8
:105A30008B8199278F7790709F938F9381E098E067
:105A40009F938F93BF92AF92E091F404F091F5048D
:105A500009958DB79EB70C968DBFFA940C5E1F4FBB
:105A6000A096F7FECFCFACC11092510382E198E02F
:105A70009F938F9352E6A52E55E2B52EDF92CF92DB
:105A8000FE0109950F900F900F900F90C1E1D8E0A3
:105A900000E010E042E0F42E802F8C5E80935103F2
:105AA0008F8D992787FD90959F938F938F89992745
:105AB00087FD90959F938F938F85992787FD90956C
:105AC0009F938F938F81992787FD90959F938F93B5
:105AD00081E298E09F938F93BF92AF92E091F4049C
:105AE000F091F5040995EDB7FEB73C96EDBFFA9439
:105AF0000C5E1F4FA096F7FECFCF62C110925103EC
:105B000082E398E09F938F9302E615E2DF92CF92B3
:105B1000FE01099584E1809351030F900F900F903F
:105B20000F9080912C08881F8827881F97E0899FF5
:105B3000C00111248D969F938F9380912408881F14
:105B40008827881F96E0899FC00111248D969F9316
:105B50008F9380911C08881F8827881F95E0899F54
:105B6000C00111248D969F938F9380911408881FF4
:105B70008827881F9927880F991F880F991F8D964E
:105B80009F938F9381E498E09F938F93DF92CF92BE
:105B9000E091F404F091F504099588E280935103B3
:105BA0002DB73EB7245F3F4F2DBF80914C08881F13
:105BB0008827881F9BE0899FC00111248D969F93A1
:105BC0008F9380914408881F8827881F9AE0899FB7
:105BD000C00111248D969F938F9380913C08881F5C
:105BE0008827881F99E0899FC00111248D969F9373
:105BF0008F9380913408881F8827881F992723E076
:105C0000880F991F2A95E1F78D969F938F9385E5CD
:105C100098E09F938F93DF92CF92E091F404F091FC
:105C2000F50409958CE3809351038DB79EB70C96CC
:105C30008DBF80915408881F8827881F9CE0899F0A
:105C4000C00111248D969F938F9389E698E09F93CE
:105C50008F93DF92CF92E091F404F091F5040995CF
:105C600080915C08EDB7FEB73696EDBF87FF12C096
:105C700080E4809351038AE798E09F938F93DF92AB
:105C8000CF92E091F404F091F50409950F900F90F4
:105C90000F900F908091640887FF12C084E4809376
:105CA00051038DE798E09F938F931F930F93E0919B
:105CB000F404F091F50409950F900F900F900F9058
:105CC00080916C0887FF7CC088E48093510380E852
:105CD00098E09F938F931F930F93E091F404F091BA
:105CE000F50409950F900F900F900F9069C01092D6
:105CF000510383E898E09F938F93DF92CF92FE0148
:105D0000099584E1809351030F900F900F900F90AD
:105D10008091DC029091DD029F938F9381E998E05E
:105D20009F938F93DF92CF92E091F404F091F5046A
:105D3000099588E2809351032DB73EB72A5F3F4F04
:105D40002DBF8091DE029091DF029F938F938EE9A9
:105D500098E09F938F93DF92CF92E091F404F091BB
:105D6000F504099589E4809351038DB79EB7069693
:105D70008DBF8BEA98E09F938F93DF92CF92E09153
:105D8000F404F091F504099580914F030F900F9062
:105D90000F900F9083FF14C01092DF021092DE026A
:105DA00060E070E08EE090E00E940B3109C08091CD
:105DB0002101281719F4215020932101109250033A
:105DC00010924F03DF91CF911F910F91FF90DF90C1
:105DD000CF90BF90AF900895F999FECF92BD81BD4D
:105DE000F89A80B599270895F999FECF1FBA92BD08
:105DF00081BD60BD0FB6F894FA9AF99A0FBE089566
:105E00004AEA20E030E02617370740F4FC01819190
:105E1000480F2F5F3F4F26173707C8F3842F992766
:105E20000895EAEA40E050E04617570778F49C01ED
:105E3000F999FECF32BD21BDF89A80B5E80F4F5FCA
:105E40005F4F2F5F3F4F4617570790F38E2F9927CD
:105E5000089581E08093410782E08093400783E0CA
:105E600080933F0784E08093420785E08093430757
:105E700086E08093440787E08093450788E080931D
:105E8000460789E0809347078AE0809348078BE0C4
:105E9000809349078CE080934A0708958DE58093AD
:105EA0003E078CE0EEEAF7E011928A95E9F78091DF
:105EB0000101843150F08AE080935E0710928207DE
:105EC0008BE180935A078EE40AC083E080935E07DB
:105ED00080E2809382078EE180935A0785E5809364
:105EE0007F078093800780E2809381071092AA0742
:105EF0008AE680934B0782E28093AC0790E490930C
:105F0000AD0786E0809365071092A20710929F0765
:105F100038E03093580786EE8093590790935B07DB
:105F20002EE120934C078FEF80934E0790916703EB
:105F3000992371F084E180934F0788E280934D07A5
:105F40002093510781E080935207109253070CC0B1
:105F50008FE080934F0720934D0790935107309324
:105F6000520784E180935307109254073FE0309327
:105F700050071092670710926807109269071092F5
:105F80006A07109284071092850710928607109274
:105F9000870790E890936B0722E320936C0782E0D9
:105FA0008093AB0730936D0786EE80936E0784E095
:105FB000809373073DE730937607309377073093EC
:105FC000780790936F0745E54093700786E48093C8
:105FD00071078CED809372078CE3809374071092A5
:105FE00075078FE58093880783EF80938A078AEA95
:105FF00080938C0780938D0788E280938907809334
:106000008B0710928E07209379079AE590937A0771
:1060100020937B078EEF80938F0784E68093900711
:106020009093910790939207909393078BE48093BA
:10603000940740939507809396071092970786E000
:106040008093980788E08093990790939A078AE253
:1060500080939B0785EF80939C078CE880939D0736
:1060600085E080939E071092A0071092A10781E21D
:106070008093620781E48093630790936407109292
:10608000A3071092A4071092A50786E98093A6079C
:1060900030937C0784E380937D071092A7071092CA
:1060A000A8071092A90708950E944E2F8AE08093B6
:1060B000550780E18093560726E0209357079AE51D
:1060C00090935C0788E780935D0790935F078093C8
:1060D00060072093610780E2809366078CE38093DA
:1060E0007E078BE48093830786E491E6A3E7B4E719
:1060F0008093AE079093AF07A093B007B093B1071A
:106100006CE770E08EE397E00E94002F8093BA075F
:106110000895CF93DF930E944E2F88E08093550718
:1061200030E13093560726E02093570794E690938A
:106130005C0788E780935D0790935F078093600713
:10614000209361073093660786E480937E078093EF
:106150008307AEEAB7E0E2E2F1E0ED0101900992D7
:106160002A95E1F76CE770E0CD01805790400E94DE
:10617000002F8093BA07DF91CF9108950E944E2F90
:1061800026E0209355078AE08093560784E08093A9
:10619000570794E690935C0788E780935D07909398
:1061A0005F07809360072093610780E18093660713
:1061B00086E480937E078093830785E491E6A3E7D6
:1061C000B9E78093AE079093AF07A093B007B09361
:1061D000B1076CE770E08EE397E00E94002F809398
:1061E000BA070895F999FECF92BD81BDF89A80B59E
:1061F00099270895F999FECF1FBA92BD81BD60BD60
:106200000FB6F894FA9AF99A0FBE08956CEE7EE2F2
:106210000E943A97089544EF5EE20E9474970895B1
:10622000EF92FF920F931F93CF93C82F8150853029
:1062300008F0C3E08DE7C89F8001112487EEE82EA7
:106240008FEFF82EE00EF11E6CE770E0C7010E94A0
:10625000112F682F98012D593F4F8FB39927AC010B
:106260004270507081FDF9CF32BD21BDF89A80B5E2
:10627000861711F0CA0123C08FB399279C012270A1
:10628000307081FDF9CFF2BCE1BCF89A80B58D3554
:1062900011F0C90114C08DE7C89FC00111244997AE
:1062A0002CEE3EE24DE750E0BC018EE397E00E9409
:1062B00015970E9470710E943A9181E090E0CF9111
:1062C0001F910F91FF90EF900895282F863010F0C6
:1062D00025E003C0882309F421E0F999FECF1FBA15
:1062E00082E090E092BD81BD20BD0FB6F894FA9A8D
:1062F000F99A0FBE0895CF93C82F80913E078D3530
:1063000009F051C0C63010F0C5E003C0CC2309F439
:106310004AC00E947E958091AD0782FF07C08091A0
:106320006307843618F080E5809363076CE770E0BC
:106330008EE397E00E94002F8093BA078DE7C89FF5
:10634000C001112424EF3EE24DE750E06EE377E018
:1063500049970E94529724EF3EE24CE050E06FE3F1
:1063600077E080E590E00E9452976CE070E08FE368
:1063700097E00E94002F282FF999FECF1FBA8CE5D5
:1063800090E092BD81BD20BD0FB6F894FA9AF99ABB
:106390000FBE8C2F0E9465310E9470710E943A914D
:1063A00081E090E002C080E090E0CF9108956DE43C
:1063B00070E088EE93E00E94112F482F8FB3992749
:1063C0009C012270307081FDF9CF85E394E092BD8D
:1063D00081BDF89A80B5841779F48FB399279C0111
:1063E0002270307081FDF9CF88EE93E092BD81BDBF
:1063F000F89A80B5813011F0C90108952CEE3EE283
:106400004EE450E068EE73E08BEB97E00E94159746
:1064100081E090E008958091BB078130A9F46DE49C
:1064200070E08BEB97E00E94002F8093080824EF28
:106430003EE24EE450E06BEB77E088EE93E00E94A2
:10644000529781E090E0089580E090E00895CF9326
:10645000DF9381E08093BB07EBEBF7E08FE01586DD
:1064600016861786108A8150349687FFF8CF80E40D
:106470008093C8078093C9071092CA078093CB07FF
:106480008093CC0790EC9093CD071092CE07809329
:10649000CF078093D0071092D1079093D2079093A3
:1064A000D3078093D4071092D5078093D607909393
:1064B000D707ACEBB7E08CE0E9E2F1E0ED01019049
:1064C00009928A95E1F76DE470E0CD0101970E9491
:1064D000002F80930808DF91CF910895F999FECF9E
:1064E00082E090E092BD81BDF89A80B5282F863079
:1064F00078F023E0322FF999FECF1FBA82E090E0C6
:1065000092BD81BD30BD0FB6F894FA9AF99A0FBECC
:10651000822F992708951F93CF93C82F162F863067
:1065200010F0C5E003C0882309F4C1E08C2F99273F
:106530008230910541F08330910544F4019731F4A4
:106540000E94543005C00E94893002C00E94BE30B3
:106550001123E1F06CE070E080E590E00E94112FE3
:10656000282FF999FECF8CE590E092BD81BDF89A75
:1065700080B5821759F42CEE3EE24CE050E060E525
:1065800070E08FE397E00E94159702C00E94292FC8
:106590008C2F0E947B31CF911F910895DF92EF9253
:1065A000FF920F931F93CF93FF24DF2CEF2C81E0FA
:1065B00090E00E94F2308B3211F031E0E32E6CE07B
:1065C00070E080E590E00E94112FC82FF999FECF6E
:1065D0008CE590E092BD81BDF89A80B58C1711F4DE
:1065E00021E0D22EC1E001E010E0EE2029F48C2F52
:1065F0000E9410318823C9F591E0F92E1F930F9363
:1066000083EB98E09F938F938EE296E19F938F9315
:10661000E091F404F091F50409952DB73EB72A5F97
:106620003F4F2DBF0230110549F0033011054CF4E6
:106630000130110531F40E94543005C00E948930A8
:1066400002C00E94BE30DD2059F02CEE3EE24CE04C
:1066500050E060E570E08FE397E00E94159702C07C
:106660000E94292F8C2F0E947B31CF5F0F5F1F4F1D
:10667000C63008F4BACFFF2019F083E00E946531DC
:106680000E946E32C82F0E9410318C2F99279F9341
:106690008F9389ED98E09F938F930EE216E11F93FD
:1066A0000F93E091F404F091F504099581E090E0F6
:1066B0000E94F2302DB73EB72A5F3F4F2DBF8F3F6C
:1066C00021F00E94D731882399F482EF98E09F93BC
:1066D0008F931F930F93E091F404F091F5040995C3
:1066E0000E9427320E940B320F900F900F900F9054
:1066F000EE2029F06BE281E090E00E94FA301092E7
:106700003D0790E0E8ECF7E0CFE080813496181682
:106710000CF49F5FC150C7FFF8CF90933D07892FBE
:1067200099279F938F938CEB97E09F938F9383E1AF
:1067300099E09F938F931F930F93E091F404F0914E
:10674000F50409950E94E6098DB79EB708968DBF9E
:10675000CF911F910F91FF90EF90DF900895982FA8
:106760002FB7F8943998389A88B1836088B98091A6
:10677000B9008C7F8093B9008AE28093B8001092B0
:106780005C0310925A0310925903992379F0E1E1C6
:10679000F8E08BE01082118212821382148215823B
:1067A000168217828150389687FFF4CF78942FBFD6
:1067B000089510925C0384E98093BC0080E8809384
:1067C000BC001092BD001092BA001092BB00109253
:1067D000B9001092B8001092580380E00E94AF33C5
:1067E0001092BB0085E88093BC00809156038260C4
:1067F0008093560308951F920F920FB60F921124A3
:106800002F933F934F935F938F939F93EF93FF93B8
:1068100080915C03282F3327442755278F5F80936F
:106820005C03F9012731310508F0C2C2E759FF4F77
:106830000C94729981E08093580309C080915A03A7
:106840008C3090F480915A038F5F80935A0380912B
:106850005A03E82FFF27EE0FFF1FEE0FFF1FE5542F
:10686000F84F8585181654F780915A038C3070F0D4
:10687000109255031092540310925A0385E08093AE
:106880005C0380915903880F8D5A04C080915A038C
:10689000880F8E5A8093BB0085E87FC280915A038F
:1068A000E82FFF2783E0EE0FFF1F8A95E1F7EF5EE9
:1068B000F74F81818093BB0085E88093BC00809175
:1068C0005A03E82FFF27EE0FFF1FEE0FFF1FEE0FFB
:1068D000FF1FEF5EF74F808180FF91C080915A03C8
:1068E000E82FFF27EE0FFF1FEE0FFF1FEE0FFF1F1A
:1068F000EF5EF74F8281882329F080913D07873032
:1069000008F46CC28091540390915503892B09F0CF
:1069100065C28091520390915303892B09F05EC2A6
:106920006EC080915A0321E030E002C0220F331F75
:106930008A95E2F7809152039091530328233923DB
:10694000232B79F080915A03E82FFF27EE0FFF1FCA
:10695000EE0FFF1FEE0FFF1FEF5EF74F80E1848306
:106960000DC080915A03E82FFF27EE0FFF1FEE0F97
:10697000FF1FEE0FFF1FEF5EF74F148280915A0347
:10698000E82FFF2753E0EE0FFF1F5A95E1F7EF5E68
:10699000F74F8481282F332743E0220F331F4A9576
:1069A000E1F780915A03E82FFF2793E0EE0FFF1FD6
:1069B0009A95E1F7EF5EF74F82818770822B809383
:1069C000BB0085E88093BC0020915A0381E090E0F1
:1069D00002C0880F991F2A95E2F720915403309145
:1069E000550382239323892B51F089E098E09093FB
:1069F000600380935F0388E080936103EFC184E0CC
:106A000089C1E0915F03F091600381918093BB00A5
:106A100085E88093BC00F0936003E0935F0380916E
:106A20006103815080936103882309F4D7C183E017
:106A300071C18091B900803351F580915D03882345
:106A400029F480915A038F5F80935D0380915A03EC
:106A5000E82FFF2783E0EE0FFF1F8A95E1F7EF5E37
:106A6000F74F838199278F7790708F3791057CF44A
:106A700080915A03E82FFF27EE0FFF1FEE0FFF1F35
:106A8000EE0FFF1FEF5EF74F83818F5F83831092BE
:106A90005C0384E98093BC008AE090E09093370126
:106AA0008093360180915A038F5F80935A0310922E
:106AB0005C036DC18091B9008034C9F180915903A4
:106AC000E82FFF27EE0FFF1FEE0FFF1FEE0FFF1F38
:106AD000EF5EF74F83818F778383809159038F5FB8
:106AE00080935903809159038C30A0F01092590380
:106AF000109253031092520380915E038F5F809334
:106B00005E038C3038F010925E03809156038D7FC7
:106B100080935603809156038160809356031092B0
:106B20005C0384E98093BC001092580373C0809189
:106B30005903E82FFF27EE0FFF1FEE0FFF1FEE0F89
:106B4000FF1FEF5EF74F8381806883838091590335
:106B5000E82FFF27EE0FFF1FEE0FFF1FEE0FFF1FA7
:106B6000EF5EF74F808180FF2FC080915903E82F9F
:106B7000FF2753E0EE0FFF1F5A95E1F7EF5EF74F47
:106B800084819927009751F04097D9F589E098E0E2
:106B90009093600380935F0388E031C08091590334
:106BA000992743E0880F991F4A95E1F78A5E974F2E
:106BB0009093600380935F039091590380915E03EB
:106BC0009817E1F483E01BC080915903992733E0C3
:106BD000880F991F3A95E1F78A5E974F909360036B
:106BE00080935F038091560381FD06C09091590305
:106BF00080915E03981711F482E001C081E08093D8
:106C0000610380916103813011F485E801C085EC56
:106C10008093BC0080915D038093570310925D03C5
:106C2000DDC0E0915F03F09160038091BB00808341
:106C300080915F039091600301969093600380932D
:106C40005F0380916103815080936103823010F073
:106C500085EC5DC0813011F485E859C08091560300
:106C600081FF2DC080916F0380FD1DC0809159036D
:106C7000E82FFF2723E0EE0FFF1F2A95E1F7EF5ED5
:106C8000F74F86818A3F79F480915903E82FFF27D7
:106C900093E0EE0FFF1F9A95E1F7EF5EF74F8081CB
:106CA000816080830CC080915903E82FFF2783E027
:106CB000EE0FFF1F8A95E1F7EF5EF74F108280918C
:106CC00059038F5F80935903809159038C30A0F052
:106CD00010925903109253031092520380915E0355
:106CE0008F5F80935E038C3038F010925E0380914A
:106CF00056038D7F8093560310925C0384E9809342
:106D0000BC008091560381608093560365C08093D8
:106D1000BC0086E080935C0361C088E9BBCD8091B4
:106D20005B03880F805FB6CD80915B03992781302C
:106D3000910561F0823091051CF4892B21F04EC041
:106D4000029739F04BC080911401A4CD80911301BA
:106D5000A1CD809112019ECD80E89CCD10925C0364
:106D600084E98093BC00109258038AE090E09093ED
:106D700037018093360180915B03823088F48091E3
:106D80005B038F5F80935B0382E180935C03809160
:106D900056038E7F8093560385EA8093BC001EC005
:106DA00010925B038091560381608093560316C056
:106DB00010925C0384E98093BC008091560381604B
:106DC000809356038AE090E09093370180933601D8
:106DD00010925A031092590310925803FF91EF91A9
:106DE0009F918F915F914F913F912F910F900FBE87
:106DF0000F901F9018951F93CF93DF93182F8091BA
:106E0000A603882321F48091EB02882319F081E006
:106E100090E097C01D3008F092C01123B1F0E12F2F
:106E2000FF2723E0EE0FFF1F2A95E1F7EF5EF74FF4
:106E300035978081359688230CF081C03897808102
:106E400080FD03C083E090E07CC08091090882301F
:106E500019F084E090E075C067E070E089E098E0A8
:106E60000E94002F90911008891719F085E090E09A
:106E700068C080ED97E00E942C1AEC0180915603C7
:106E800080FD05C0CE010E94351A8823B9F3112375
:106E900019F48FEF90E00BC0212F332721503040A1
:106EA00081E090E002C0880F991F2A95E2F7909345
:106EB000550380935403A1E0B0E0E1E1F8E040E045
:106EC00050E06BE0CD01042E02C0880F991F0A9498
:106ED000E2F7209154033091550382239323892BA9
:106EE00011F01182128261504F5F5F4F389667FF39
:106EF000E9CF10925A0310925C03809156038E7F63
:106F00008093560385EA8093BC008091560380FDF0
:106F100005C0CE010E94351A8823B9F3809154032D
:106F200090915503892B29F0CE010E94351A8823B0
:106F300011F38091540390915503009711F082E072
:106F400090E0DF91CF911F9108950F931F93CF93FE
:106F5000DF93982F8091A603882321F48091EB0280
:106F6000882319F081E090E092C09D30A0F499232D
:106F700019F486E090E08BC0C92FDD27FE0133E0D5
:106F8000EE0FFF1F3A95E1F7EF5EF74F35978081DF
:106F9000359687FD03C082E090E079C03897808104
:106FA00080FD03C083E090E072C080ED97E00E9416
:106FB0002C1A8C018091560380FD05C0C8010E94E7
:106FC000351A8823B9F3219721E030E0C90102C0C6
:106FD000880F991FCA95E2F7909353038093520349
:106FE000D901E1E1F8E040E050E06BE0CD01042E92
:106FF00002C0880F991F0A94E2F720915203309142
:10700000530382239323892B11F011821282615042
:107010004F5F5F4F389667FFE9CF10925903109288
:1070200009081092100810925C03809156038E7F1D
:107030008093560385EA8093BC008091560380FDBF
:1070400005C0C8010E94351A8823B9F38091520304
:1070500090915303892B29F0C8010E94351A882387
:1070600011F380910908823019F084E090E00FC09C
:1070700067E070E089E098E00E94002F909110088E
:10708000891719F085E090E002C080E090E0DF9180
:10709000CF911F910F910895CF93DF9380E021E866
:1070A0003FEFC6EAD8E0E2E7F8E0DF01853020F400
:1070B00011961C921E9202C031832083198218827D
:1070C00022968F5F129632968A3180F310921404C2
:1070D00010921304109216041092150410921804C2
:1070E00010921704DF91CF9108951F920F920FB65F
:1070F0000F9211240F931F932F933F934F935F93FE
:107100006F937F938F939F93AF93BF93CF93DF93AF
:10711000EF93FF9340918600509187008091630325
:1071200090916403481B590BCA0157FD0196AC01AD
:1071300055954795809186009091870090936403C0
:1071400080936303CA0189599840A0916503B09167
:107150006603875E954338F4149714F010923A0151
:1071600081E090E081C0AD30B1050CF081C0CA0172
:107170008B5F90408356944008F071C0425C53404E
:10718000FD01EA0FFB1FEE58F74F80819181FA0154
:10719000E81BF90BCF01F7FF03C0909581959F4F36
:1071A00006974CF48091A703883C28F48091A703AC
:1071B000865F8093A703FD01EA0FFB1FEE58F74F90
:1071C000808191819C01220F331F280F391F240FCA
:1071D000351F37FF02C02D5F3F4FE901D595C79599
:1071E000D595C795CA0101968C179D0714F4219770
:1071F00006C041505040C417D5070CF42196809129
:10720000A703833CD8F08D010A0F1B1FF801EE582D
:10721000F74F808191819E01281B390BC90163E0E2
:1072200070E00E94EB98CB01880F991F860F971F83
:107230000A55174FF8019183808307C0AA0FBB1F1F
:10724000AA55B74F11961C921E92E0916503F091DA
:107250006603EE0FFF1FEE58F74FD183C083809176
:10726000650390916603019690936603809365038E
:10727000FF91EF91DF91CF91BF91AF919F918F914E
:107280007F916F915F914F913F912F911F910F913E
:107290000F900FBE0F901F901895EF92FF920F93D3
:1072A0001F9380915A079927880F991F880F991F5C
:1072B0007C010027F7FC0095102F8091010490912C
:1072C0000204A0910304B0910404BC01CD01A80103
:1072D00097010E94209930939A06209399068091F5
:1072E000F9039091FA03A091FB03B091FC03BC0158
:1072F000CD01A80197010E94209930939C0620930C
:107300009B06809131099091320997FD03969595DE
:1073100087959595879590939E0680939D0680917D
:1073200041099091420997FD03969595879595950A
:1073300087959093A00680939F0680911304909167
:10734000140420912C0330912D03821B930B9093F6
:10735000A2068093A1068091A1039091A203A0911F
:10736000A303B091A403BC01CD012AE030E040E0CA
:1073700050E00E9420993093A4062093A3068091A8
:10738000DE069091DF069093A6068093A506809175
:107390008A0190918B019093AA068093A90680910F
:1073A0001F01909120019093AC068093AB068091D1
:1073B000A70399279093AE068093AD068091E808C5
:1073C0009091E9089093B0068093AF0680911208DF
:1073D00099279093B2068093B10680911A08992755
:1073E0009093B4068093B3068091220899279093D6
:1073F000B6068093B50680912A0899279093B8061F
:107400008093B70680910603909107039093C2067C
:107410008093C1068091C2099091C3099093C606DA
:107420008093C5068091C6099091C7099093C806BC
:107430008093C70680919D0390919E03A0919F0326
:10744000B091A003BC01CD012AE030E040E050E063
:107450000E9420993093CA062093C9068091BF03E9
:107460009091C0039093D0068093CF068091C80975
:1074700099279093D4068093D306809176049091B7
:1074800077049093D6068093D506809174049091EA
:1074900075049093D8068093D70680910D058823B4
:1074A00021F480910E05882321F080919806816057
:1074B00003C0809198068E7F809398061F910F914C
:1074C000FF90EF900895EF92FF921F93CF93DF9379
:1074D000182F7B018091A603882391F580910101EB
:1074E0008C3010F0873111F4299801C0299A11507D
:1074F0001F3FE9F0F0920D03E0920C03E701809149
:107500000C0390910D03892B11F4209781F3809146
:1075100010038823A1F31092100380910C03909123
:107520000D03892B09F421970E949495E8CF80914F
:1075300001018C3010F0873111F4299A01C029988B
:10754000DF91CF911F91FF90EF900895CF93DF933C
:10755000809101018D3011F40E941F1F10927A005A
:1075600080913003909131039093F4088093F30855
:1075700080912E0390912F039093E4088093E30869
:1075800080912C0390912D039093370980933609B5
:107590002091280330912903C901880F991F880F72
:1075A000991F820F931F820F931F9093320980932C
:1075B000310920912A0330912B03C901880F991FAB
:1075C000880F991F820F931F820F931F9093420978
:1075D000809341098FEC80937A00A8EAB3E0C3E47A
:1075E000D7E097E08991E82FFF27EE0FFF1FEE58B5
:1075F000F74F0190F081E02DE158FF4F1E161F0656
:107600001CF0E0E0F0E005C0EF3FF10514F0EFEF13
:10761000F0E08C91282F3327E217F30714F4815000
:1076200004C02E173F0714F48F5F8C93915011966E
:1076300097FFD8CF80917F079927AA27BB27BC0146
:10764000CD0124EC39E040E050E00E94AC98DC0130
:10765000CB018093820190938301A0938401B09326
:107660008501809180079927AA27BB27BC01CD01FE
:107670000E94AC98DC01CB0180937E0190937F0146
:10768000A0938001B0938101DF91CF910895A0E094
:10769000B0E0EDE4FBE30C943F99682EE1E07E2E30
:1076A00000E010E068015801E80110920D05109308
:1076B0000E0400930D0410930C0400930B0410931C
:1076C0000804009307041092060410931804009312
:1076D00017041093160400931504109314040093D8
:1076E00013041092640110926301109221030E940E
:1076F000A63A84E690E00E944E1A0E94A63A809133
:107700004B0780FF10C08091150190911601875B97
:10771000934038F480911501909116018E5E92404D
:1077200010F40E949D1E7FE1E72E8AE090E00E9407
:107730004E1A80912C0390912D03080F191F8091F0
:10774000300390913103C80ED91E80912E03909181
:107750002F03A80EB91E8091DE069091DF06C80F98
:10776000D91FEA94E7FEE1CF9601205F3F4F36959F
:107770002795369527953093180420931704C50153
:107780004096969587959695879590931604809345
:107790001504005F1F4F45E0169507954A95E1F7E0
:1077A00010931404009313046096B5E0D695C79522
:1077B000BA95E1F7D0930804C0930704909312049C
:1077C000809311043093100420930F0482E0681614
:1077D000C9F5809131099091320997FF03C09095C6
:1077E00081959F4F6CE070E00E94EB989B01709335
:1077F0000E0460930D04809141099091420997FF16
:1078000003C0909581959F4F6CE070E00E94EB98CB
:1078100070930C0460930B04B90184E090E00E9423
:107820000B3160910B0470910C0486E090E00E9493
:107830000B31609107047091080488E090E00E9489
:107840000B314FC084E090E00E94063190930E040B
:1078500080930D0486E090E00E9406319C01909395
:107860000C0480930B0480910D0490910E048150C0
:10787000984018F421503840A0F184E399E09F9398
:107880008F938EE296E19F938F93E091F404F091B1
:10789000F5040995809131099091320997FF03C051
:1078A000909581959F4F6CE070E00E94EB987093EB
:1078B0000E0460930D04809141099091420997FF55
:1078C00003C0909581959F4F6CE070E00E94EB980B
:1078D00070930C0460930B0477240F900F900F901B
:1078E0000F901092F4081092F3081092E40810928E
:1078F000E308109237091092360984E690E00E945E
:107900004E1A80912803909129039C01220F331F66
:10791000220F331F280F391F280F391F30933209C8
:107920002093310980912A0390912B038C01000F41
:10793000111F000F111F080F191F080F191F109397
:1079400042090093410980915A07C82EDD24EE2494
:10795000FF24442737FD4095542FC701B6010E94EC
:10796000AC984B015C016093010470930204809316
:107970000304909304049801442737FD4095542F45
:10798000C701B6010E94AC98DC01CB018093F903DA
:107990009093FA03A093FB03B093FC038092E1035E
:1079A0009092E203A092E303B092E4038093D903A0
:1079B0009093DA03A093DB03B093DC031092D1031E
:1079C0001092D2031092D3031092D4038091170126
:1079D00090911801A0911901B0911A018093E006CD
:1079E0009093E106A093E206B093E3061092200381
:1079F00010921F031092220310922303109224036B
:107A0000109225031092C1031092C2031092C30377
:107A10001092C40300918A0110918B011093C0034E
:107A20000093BF0384E690E09093870180938601E2
:107A300082E390E090930D0380930C0380917F0785
:107A40009927AA27BB27BC01CD0124EC39E040E0EF
:107A500050E00E94AC98DC01CB018856954CAF4FAA
:107A6000BF4F8093820190938301A0938401B093D0
:107A70008501809180079927AA27BB27BC01CD01EA
:107A80000E94AC98DC01CB018856954CAF4FBF4F9C
:107A900080937E0190937F01A0938001B093810138
:107AA0001092410110924001C801AA2797FDA095AC
:107AB000BA2F20913C0130913D0140913E015091FF
:107AC0003F01BC01CD010E94AC98DC01CB01809349
:107AD0003D0990933E09A0933F09B093400910924D
:107AE000BC031092BB030E94707180916F0384608D
:107AF00080936F038FEF8093BD091092BE0980E2DF
:107B00008093BF09C8EAD3E0A3E4B7E0E7E0EE2E34
:107B10008D91E82FFF27EE0FFF1FEE58F74F808162
:107B2000918181588993EA94E7FEF2CF84E68093AD
:107B3000A70380910A03882311F0579A06C080E0BA
:107B400091E1909308018093070180910104909145
:107B50000204A0910304B0910404E0903C01F09071
:107B60003D0100913E0110913F01BC01CD01A801F2
:107B700097010E94209959016A018091F90390911F
:107B8000FA03A091FB03B091FC03BC01CD01A80155
:107B900097010E942099B901C5010E94CC968C01E1
:107BA0000E94D7749C019093FF088093FE088091F7
:107BB000070490910804AA2797FDA095BA2F7DE0AD
:107BC000880F991FAA1FBB1F7A95D1F78050904F3D
:107BD000AF43B040442737FD4095542FBC01CD0141
:107BE0000E942099C90180509E4F90930804809371
:107BF0000704053111050CF07724662079F0809197
:107C00006703882359F0C90181599040C39730F028
:107C100080910D05806280930D0577248091170473
:107C20009091180480569940815C9B4228F0809185
:107C30000D05816080930D058091150490911604C7
:107C400080569940815C9B4228F080910D058260AE
:107C500080930D0580911304909114048C529140EF
:107C60008957954028F080910D05846080930D051B
:107C700080910D0490910E048C529140835C914050
:107C800028F080910D05886080930D0580910B048C
:107C900090910C048C529140835C914028F080912B
:107CA0000D05806180930D05809107049091080473
:107CB000805092408355914028F080910D0580625C
:107CC00080930D0580910D058111772486E48093C2
:107CD00079010E943A9182E00E949F92872D992714
:107CE000EEE0CDB7DEB70C945B99A3E1B0E0EBE733
:107CF000FEE30C943B99809113049091140420911D
:107D00002C0330912D03821B930B909337098093A2
:107D10003609809136039091370397FD07969C01B1
:107D200013E0359527951A95E1F73093F4082093E1
:107D3000F308809134039091350397FD0796B3E0E3
:107D400095958795BA95E1F79093E4088093E308B9
:107D500030930109209300099093F7088093F60867
:107D60008091310990913209AC01440F551F480FA1
:107D7000591F2091280330912903C901880F991FA9
:107D8000880F991F820F931F820F931F480F591F4F
:107D900057FF02C04D5F5F4F5595479555954795E5
:107DA00050933209409331098091410990914209E1
:107DB000AC01440F551F480F591F20912A033091E1
:107DC0002B03C901880F991F880F991F820F931FDA
:107DD000820F931F480F591F57FF02C04D5F5F4F1F
:107DE00055954795559547955093420940934109BC
:107DF0002091280330912903C901880F991F880F0A
:107E0000991F820F931F820F931F9C01442737FDF8
:107E10004095542F8091F1039091F203A091F303C8
:107E2000B091F403820F931FA41FB51F8093F10339
:107E30009093F203A093F303B093F40320912A03E9
:107E400030912B03C901880F991F880F991F820F4A
:107E5000931F820F931F9C01442737FD4095542F99
:107E60008091ED039091EE03A091EF03B091F003A8
:107E7000820F931FA41FB51F8093ED039093EE0311
:107E8000A093EF03B093F00380910A0990910B093E
:107E90002091280330912903820F931F90930B099F
:107EA00080930A098091390990913A0920912A0317
:107EB00030912B03820F931F90933A0980933909D5
:107EC0008091090490910A04019690930A0480938A
:107ED00009048091DE069091DF062091070430911D
:107EE0000804821B930B9C01442737FD4095542FB7
:107EF0008091E9039091EA03A091EB03B091EC0328
:107F0000820F931FA41FB51F8093E9039093EA0388
:107F1000A093EB03B093EC038FEC80937A00109264
:107F200011012091D9033091DA034091DB03509184
:107F3000DC0329873A874B875C8729543B464140BD
:107F400050402CF028E43BE641E050E00DC089852C
:107F50009A85AB85BC85885B9449AE4FBF4F4CF486
:107F600028EB34E94EEF5FEF2D833E834F83588734
:107F700008C089859A85AB85BC858D839E83AF8338
:107F8000B8872091E1033091E2034091E3035091DF
:107F9000E4032D873E874F87588B29543B46414049
:107FA00050402CF028E43BE641E050E00DC08D85C8
:107FB0009E85AF85B889885B9449AE4FBF4F4CF41E
:107FC00028EB34E94EEF5FEF29833A834B835C83E0
:107FD00008C08D859E85AF85B88989839A83AB83D8
:107FE000BC83A0913609B0913709BB8BAA8BFD01E8
:107FF000CF01AA2797FDA095BA2FA090D103B090EA
:10800000D203C090D303D090D403A80EB91ECA1EC9
:10801000DB1EA092D103B092D203C092D303D092C0
:10802000D403E0903D09F0903E0900913F09109182
:108030004009E80EF91E0A1F1B1FE0923D09F0924D
:108040003E0900933F0910934009F0918A03F98B90
:10805000FF2309F098C180918903882309F093C117
:1080600080912D0986FF8FC18091E3089091E408EB
:10807000AA2797FDA095BA2FBC01CD0129813A818D
:108080004B815C810E94AC989B01AC0197FF04C0BE
:108090002150384F4F4F5F4FBBE05595479537956F
:1080A0002795BA95D1F780916301682E77248824AB
:1080B0009924CA01B901A40193010E94AC98DC0182
:1080C000CB018093230490932404A0932504B093C0
:1080D0002604B7FF04C08150904FAF4FBF4F1C0123
:1080E0002D01ACE05594479437942794AA95D1F785
:1080F00020922304309224044092250450922604B6
:108100008091F3089091F408AA2797FDA095BA2FC3
:10811000BC01CD012D813E814F8158850E94AC98D4
:1081200097FF04C06150784F8F4F9F4FFBE09595AC
:10813000879577956795FA95D1F7A40193010E94E9
:10814000AC98DC01CB018093270490932804A09382
:108150002904B0932A04B7FF04C08150904FAF4F59
:10816000BF4F9C01AD01ECE055954795379527959C
:10817000EA95D1F7209327043093280440932904EB
:1081800050932A0480912304909124049093DB0857
:108190008093DA0880912704909128049093DF0857
:1081A0008093DE08221933094409550920932704D6
:1081B000309328044093290450932A04E20EF31EBE
:1081C000041F151FE0923D09F0923E0900933F09FC
:1081D00010934009809162018823B1F457FF04C0D5
:1081E0002F5F3F4F4F4F5F4F5595479537952795D9
:1081F000A21AB30AC40AD50AA092D103B092D2033C
:10820000C092D303D092D4032A893B8979010027F5
:10821000F7FC0095102F8091270490912804A091DD
:108220002904B0912A04E80EF91E0A1F1B1FC80179
:10823000B70129813A814B815C810E94AC989B01F6
:10824000AC0197FF04C02150384F4F4F5F4F6BE098
:1082500055954795379527956A95D1F78091640193
:10826000A82EBB24CC24DD24CA01B901A6019501A6
:108270000E94AC98DC01CB0180931B0490931C04FA
:10828000A0931D04B0931E04B7FF04C08150904F0B
:10829000AF4FBF4F3C014D013CE0959487947794DC
:1082A00067943A95D1F760921B0470921C048092F7
:1082B0001D0490921E04C801B7012D813E814F819B
:1082C00058850E94AC9897FF04C06150784F8F4F3B
:1082D0009F4F2BE095958795779567952A95D1F7D0
:1082E000A60195010E94AC98DC01CB0180931F048C
:1082F00090932004A0932104B0932204B7FF04C0FC
:108300008150904FAF4FBF4FAC01BD010CE0759550
:108310006795579547950A95D1F740931F04509359
:10832000200460932104709322042A893B8937FF3B
:1083300003C0309521953F4F21343105E4F1D4013C
:10834000C30197FE07C0B095A095909581959F4F6A
:10835000AF4FBF4F81389105A105B10584F4DB0112
:10836000CA0177FF07C0B095A095909581959F4F62
:10837000AF4FBF4F81389105A105B105E4F081E011
:108380008093BD0318C01092DF081092DE0810928F
:10839000DB081092DA0810921F0410922004109249
:1083A00021041092220410921B0410921C041092BB
:1083B0001D0410921E0480911F0490912004A0912E
:1083C0002104B0912204BC01CD0124E630E040E05C
:1083D00050E00E942099E0901B04F0901C04E21AE7
:1083E000F30AF092F208E092F10880911B04909158
:1083F0001C04A0911D04B0911E04BC01CD0124E613
:1084000030E040E050E00E942099DA01C90120915B
:108410001F04309120048C01021B130B1093E608FB
:108420000093E50880913C0190913D01A0913E01AF
:10843000B0913F01BC01CD0128E631E040E050E0C1
:108440000E94AC9820913D0930913E0940913F092E
:1084500050914009261737074807590764F0261B33
:10846000370B480B590B20933D0930933E0940933D
:108470003F095093400920913D0930913E094091B8
:108480003F095091400957FF0CC0260F371F481F66
:10849000591F20933D0930933E0940933F09509363
:1084A00040096091E3087091E4086E0D7F1D9B0107
:1084B000442737FD4095542F8091D5039091D603E2
:1084C000A091D703B091D803820F931FA41FB51FAB
:1084D0008093D5039093D603A093D703B093D8038A
:1084E00080918F0390919003681B790BCB01AA2791
:1084F00097FDA095BA2F29853A854B855C85820F1B
:10850000931FA41FB51F8093D9039093DA03A09300
:10851000DB03B093DC03C0907E01D0907F01E0903C
:108520008001F0908101C816D906EA06FB06C4F462
:1085300088EA91E6A0E0B0E08C199D09AE09BF0978
:108540008093D9039093DA03A093DB03B093DC0309
:108550008093D5039093D603A093D703B093D80309
:1085600022273327A9012C193D094E095F09809163
:10857000D9039091DA03A091DB03B091DC03821759
:108580009307A407B507B4F4D701C601885A9146EA
:10859000A040B0408093D9039093DA03A093DB030B
:1085A000B093DC038093D5039093D603A093D703B5
:1085B000B093D8036091F3087091F408600F711FB5
:1085C0009B01442737FD4095542F8091DD03909106
:1085D000DE03A091DF03B091E003820F931FA41F7D
:1085E000B51F8093DD039093DE03A093DF03B09368
:1085F000E00380918D0390918E03681B790BCB0172
:10860000AA2797FDA095BA2F2D853E854F855889BD
:10861000820F931FA41FB51F8093E1039093E20381
:10862000A093E303B093E403E0908201F090830110
:108630000091840110918501E816F9060A071B07CD
:10864000C4F488EA91E6A0E0B0E08E199F09A00B7F
:10865000B10B8093E1039093E203A093E303B09303
:10866000E4038093DD039093DE03A093DF03B093D4
:10867000E00322273327A9012E193F09400B510B94
:108680008091E1039091E203A091E303B091E403B0
:1086900082179307A407B507B4F4D801C701885A15
:1086A0009146A040B0408093E1039093E203A093F1
:1086B000E303B093E4038093DD039093DE03A09380
:1086C000DF03B093E0038091D1039091D203A09196
:1086D000D303B091D4038093E5039093E603A09372
:1086E000E703B093E8038091E1039091E203A09146
:1086F000E303B091E4038093010490930204A093F8
:108700000304B09304048091D9039091DA03A091FB
:10871000DB03B091DC038093F9039093FA03A093F9
:10872000FB03B093FC038091DD039091DE03A091E5
:10873000DF03B091E0038093FD039093FE03A093C9
:10874000FF03B09300048091D5039091D603A091CC
:10875000D703B091D8038093F5039093F603A093C9
:10876000F703B093F80380911D0190911E0197FDCE
:10877000079613E0959587951A95E1F79093F4087D
:108780008093F30880911B0190911C0197FD07963F
:10879000B3E095958795BA95E1F79093E4088093B7
:1087A000E30880913003909131030F9734F488E10E
:1087B0009CEF9093F4088093F3088091300390919C
:1087C0003103079734F480E398EF9093F408809393
:1087D000F308209101012A30A9F48091300390918F
:1087E0003103835F934034F088EE93E09093F40874
:1087F0008093F30880913003909131038A5F934016
:10880000DCF014C08091300390913103815D97407A
:1088100034F088EE93E09093F4088093F30880910D
:10882000300390913103805E974034F080ED97E003
:108830009093F4088093F30880912E0390912F0376
:108840000F9734F488E19CEF9093E4088093E30859
:1088500080912E0390912F03079734F480E398EFD3
:108860009093E4088093E3082A30A9F480912E03C2
:1088700090912F03835F934034F088EE93E09093C0
:10888000E4088093E30880912E0390912F038A5F80
:108890009340DCF014C080912E0390912F03815DF2
:1088A000974034F088EE93E09093E4088093E308D7
:1088B00080912E0390912F03805E974034F080EDDD
:1088C00097E09093E4088093E30860917001662339
:1088D00009F4AFC040911D0150911E0180912B04FD
:1088E00090912C04481B590B50933204409331044F
:1088F00020911D0130911E01280F391F37FF02C042
:108900002F5F3F4F3595279530932C0420932B04F0
:10891000413851051CF080E890E005C040585F4F99
:1089200034F480E89FEF90933204809331044091B7
:108930001B0150911C0180912D0490912E04481B25
:10894000590B5093300440932F0420911B01309118
:108950001C01280F391F37FF02C02F5F3F4F35958D
:10896000279530932E0420932D04413851051CF097
:1089700080E890E005C040585F4F34F480E89FEFF6
:108980009093300480932F04462F55278091310413
:1089900090913204849FB001859F700D949F700D5B
:1089A00011249B0177FF02C0215F3F4FE4E0359522
:1089B0002795EA95E1F78091F3089091F408820FEA
:1089C000931F9093F4088093F30880912F04909163
:1089D0003004849FD001859FB00D949FB00D112469
:1089E000AD019D01B7FF02C0215F3F4F94E0359577
:1089F00027959A95E1F78091E3089091E408820F1A
:108A0000931F9093E4088093E30880911D01909157
:108A10001E01860F971F90931E0180931D01809168
:108A20001B0190911C01840F951F90931C01809352
:108A30001B010091F6081091F7088091DA089091D7
:108A4000DB08101611065CF59C0197FF04C0222775
:108A50003327281B390BC901AA2797FDA095BA2FE8
:108A600020916201332744275527BC01CD010E9484
:108A7000AC989B01AC0197FF04C0215C3F4F4F4F66
:108A80005F4F86E055954795379527958A95D1F79D
:108A90008091F1089091F208820F931F27C097FFF1
:108AA00003C0909581959F4FAA2797FDA095BA2F57
:108AB00020916201332744275527BC01CD010E9434
:108AC000AC989B01AC0197FF04C0215C3F4F4F4F16
:108AD0005F4FB6E05595479537952795BA95D1F7ED
:108AE0008091F1089091F208821B930B9093F20809
:108AF0008093F108E0900009F09001098091DE0870
:108B00009091DF081E141F045CF59C0197FF04C0C0
:108B100022273327281B390BC901AA2797FDA095C7
:108B2000BA2F20916201332744275527BC01CD017C
:108B30000E94AC989B01AC0197FF04C0215C3F4FA1
:108B40004F4F5F4FA6E05595479537952795AA95C6
:108B5000D1F78091E5089091E608820F931F27C016
:108B600097FF03C0909581959F4FAA2797FDA095E9
:108B7000BA2F20916201332744275527BC01CD012C
:108B80000E94AC989B01AC0197FF04C0215C3F4F51
:108B90004F4F5F4FF6E05595479537952795FA95D6
:108BA000D1F78091E5089091E608821B930B909392
:108BB000E6088093E50880912D0987FF44C0B989B4
:108BC000BB2309F040C0809189038823E1F5E1E0EF
:108BD000EE16E1E0FE064CF08091F3089091F40867
:108BE0008E0D9F1D805091400DC0F0E0EF16FFEFFD
:108BF000FF0664F48091F3089091F4088E0D9F1D98
:108C000080509F4F9093F4088093F30821E0013047
:108C100012074CF08091E3089091E408800F911FB7
:108C2000805091400CC03FEF0030130764F48091F6
:108C3000E3089091E408800F911F80509F4F90931C
:108C4000E4088093E308E2E1CD5E0C9457998091AB
:108C5000A603882329F580916F038C7F80936F038F
:108C600080916E038F7D80936E03A2E1B5E0E1E118
:108C7000F8E09BE08091EB02882309F48C938D91BE
:108C8000818312829150389697FFF4CF8091EB0246
:108C9000882359F08091EB0281508093EB0205C04C
:108CA00080916F03816080936F03809158038823C4
:108CB00019F010925803089580935A0380935C032F
:108CC000809156038E7F8093560385EA8093BC0083
:108CD0000895CF93DF93A8EAB3E0C3E4D7E057E069
:108CE0009991E92FFF27EE0FFF1FEE58F74F0190E4
:108CF000F081E02DE158FF4FEF3FF10521F01CF02E
:108D0000EFEFF0E004C0F7FF02C0E0E0F0E09931DF
:108D100011F4EC931BC04C91242F3327E217F30777
:108D2000A9F0CF01821B930B97FD0396959587952C
:108D300095958795242F280F2C93822F9927E81734
:108D4000F90714F4215001C02F5F2C935150119654
:108D500057FFC6CF80914D07883F38F0EFEFF0E026
:108D6000E81BF109E855FC4F8081809376018091E2
:108D70007601882329F0843618F084E68093760102
:108D800080914F07883F38F0EFEFF0E0E81BF109E2
:108D9000E855FC4F80818093740180917401882391
:108DA00029F0843618F084E68093740180915C0782
:108DB000883F38F0EFEFF0E0E81BF109E855FC4F91
:108DC000808180936F0180916F018B3010F48AE075
:108DD00002C08F3F11F480936F0180918907883F13
:108DE00038F0EFEFF0E0E81BF109E855FC4F808127
:108DF00080930C0980910C09863010F485E002C044
:108E00008F3F11F480930C0980918B07883F38F0D5
:108E1000EFEFF0E0E81BF109E855FC4F808180930B
:108E2000340980913409863010F485E002C08F3F08
:108E300011F48093340980917607873F19F44299A1
:108E400005C006C0863F31F4439B02C08CE80BC0CE
:108E500086E409C0883F38F0EFEFF0E0E81BF10945
:108E6000E855FC4F80818093090980917707873FFF
:108E700019F4429905C006C0863F31F4439B02C0F5
:108E80008CE80BC086E409C0883F38F0EFEFF0E0D3
:108E9000E81BF109E855FC4F80818093E008809140
:108EA0007807883F38F0EFEFF0E0E81BF109E8556C
:108EB000FC4F80818093120980914E07883F38F0E3
:108EC000EFEFF0E0E81BF109E855FC4F808180935B
:108ED000750180915107883F38F0EFEFF0E0E81B13
:108EE000F109E855FC4F808180937301809153070D
:108EF000883F38F0EFEFF0E0E81BF109E855FC4F50
:108F000080818093710180915B07883F38F0EFEF9B
:108F1000F0E0E81BF109E855FC4F80818093720175
:108F200080915D07883F38F0EFEFF0E0E81BF10932
:108F3000E855FC4F808180936E0180915E07883FE9
:108F400038F0EFEFF0E0E81BF109E855FC4F8081C5
:108F50008093700180915F07883F38F0EFEFF0E079
:108F6000E81BF109E855FC4F808180936D018091E9
:108F70006007883F38F0EFEFF0E0E81BF109E855B3
:108F8000FC4F808180936C0180916607883F38F0A8
:108F9000EFEFF0E0E81BF109E855FC4F808180938A
:108FA0006A0180916707883F38F0EFEFF0E0E81B37
:108FB000F109E855FC4F8081809384038091680714
:108FC000883F38F0EFEFF0E0E81BF109E855FC4F7F
:108FD00080818093830380916907883F38F0EFEFA9
:108FE000F0E0E81BF109E855FC4F80818093820393
:108FF00080916A07883F38F0EFEFF0E0E81BF10955
:10900000E855FC4F80818093810380918407883FDD
:1090100038F0EFEFF0E0E81BF109E855FC4F8081F4
:109020008093800380918507883F38F0EFEFF0E070
:10903000E81BF109E855FC4F808180937F03809104
:109040008607883F38F0EFEFF0E0E81BF109E855BC
:10905000FC4F808180937E0380918707883F38F0A2
:10906000EFEFF0E0E81BF109E855FC4F80818093B9
:109070007D0380916B07883F38F0EFEFF0E0E81B4D
:10908000F109E855FC4F80818093690180916F0759
:10909000883F38F0EFEFF0E0E81BF109E855FC4FAE
:1090A00080818093680180916C07883F38F0EFEFF2
:1090B000F0E0E81BF109E855FC4F808180936701DF
:1090C00080917007883F38F0EFEFF0E0E81BF1097E
:1090D000E855FC4F80818093660180917907883F35
:1090E00038F0EFEFF0E0E81BF109E855FC4F808124
:1090F0008093650180917C07883F38F0EFEFF0E0C6
:10910000E81BF109E855FC4F808180936401809150
:109110007D07883F38F0EFEFF0E0E81BF109E855F4
:10912000FC4F80818093630180917E07883F38F0F7
:10913000EFEFF0E0E81BF109E855FC4F80818093E8
:1091400062018091A607883F38F0EFEFF0E0E81B5E
:10915000F109E855FC4F80818093EF0890918004DD
:10916000992321F08091EF08981720F08091EF0863
:10917000882311F49093EF0880914B0780932D0979
:109180008091AC078093110980918307883F38F064
:10919000EFEFF0E0E81BF109E855FC4F8081809388
:1091A000610180919F07883F38F0EFEFF0E0E81B06
:1091B000F109E855FC4F80818093440980916A0150
:1091C000282F33272F5F3F4F8CE398E2B9010E948D
:1091D000EB987093780160937701809159078093A1
:1091E0003509809158078093F8089091A10793332F
:1091F00008F44AC081E080937C03983F58F0EFEF79
:10920000F0E0E91BF109E855FC4F8081823310F44E
:1092100010927C038091790120917C03821721F1C7
:109220008330F8F43091A101222351F08CED95E0C8
:1092300090930D0380930C03332369F48EE209C0ED
:1092400088EC90E090930D0380930C03332319F482
:1092500087E18093A10185E08093910320937901B8
:1092600003C0815080937901809184099091850990
:1092700097FF0FC080917C03882359F080910D05E2
:10928000806880930D0505C010927C038AE080936E
:109290007901809184099091850997FF1DC0809183
:1092A000A6038823C9F080917C038823A9F08091CC
:1092B000090190910A018F5F9F4F71F488E99AE349
:1092C00090930D0380930C0380E094EA90930A013D
:1092D0008093090110927C0380917C03882369F0BC
:1092E00080916E03816080936E0380916401823D62
:1092F00048F4825E8093640105C080916E038E7F86
:1093000080936E03DF91CF910895A7E1B0E0EBE881
:10931000F9E40C943B990E94753E80916F03992764
:1093200084719070892B91F58091AD0782FF27C0E1
:1093300080918B0390918C030097F1F002E08835C7
:109340009007D4F49C0197FF02C02D5F3F4F3595E5
:10935000279535952795809163079927289FA00128
:10936000299F500D389F500D1124CA0164E670E00A
:109370000E94EB98CB0106C08DE290E003C0809183
:109380006307992790936D0380936C0320916A0380
:1093900030916B0355E72033350759F41092B2032F
:1093A0001092B1038091F808992790936D038093F0
:1093B0006C036091B1037091B2037A8369838091E9
:1093C000F80899270A966817790714F49A8389830D
:1093D0008091A703843608F06AC080916E0382FDF5
:1093E00066C08091470490914804009731F001973E
:1093F00090934804809347040BC01092A603909367
:1094000071038093700380916F038D7E80936F034F
:10941000809101018A3011F0843110F0289A01C046
:1094200028988091700390917103895E9340E0F1D8
:109430008091C8098536C0F180916C0390916D03CD
:109440009A83898380916F03806180936F038091F9
:109450003F07A82FBB27AA0FBB1FFD01EA55F74FF7
:109460001182108280914007282F3327220F331F4B
:10947000C9018A55974FFC0111821082AE58B74F2F
:1094800011961C921E922E58374FD90111961C929C
:109490001E9280914207E82FFF27EE0FFF1FEE5824
:1094A000F74F11821082C1C31092A603BEC38091F0
:1094B000A7038D3808F48FC380916F038F7E80934C
:1094C0006F039091640782E3989FC00111249093E9
:1094D000480480934704E981FA81B9978CF0809120
:1094E000A603882369F08091700390917103FFEFC8
:1094F0008F3F9F0729F0019690937103809370032B
:1095000020917003309171032F3F310509F030F540
:109510001092C9031092CA031092CB031092CC038D
:109520001092C5031092C6031092C7031092C8038D
:1095300010923304109234041092350410923604C1
:109540001092D1031092D2031092D3031092D4033D
:1095500080916E03806280936E0347C080916F0399
:10956000826080936F0380916E0385FF3EC080917F
:10957000A1039091A203A091A303B091A403825AE6
:109580009E4FAF4FBF4F855F9140A040B04020F449
:1095900080912D0980FD08C080916E038F7D80939E
:1095A0006E0380E38093A1011092C9031092CA0355
:1095B0001092CB031092CC031092C5031092C603F5
:1095C0001092C7031092C8031092D1031092D203D5
:1095D0001092D3031092D403295E334030F088EE0A
:1095E00093E0909371038093700380914107E82F7B
:1095F000FF27EE0FFF1FEE58F74F808191818135D5
:1096000091050CF44BC12091A603222309F046C119
:1096100080914207E82FFF27EE0FFF1FEE58F74F0C
:10962000808191818C3491050CF408C180914904AA
:109630008F5F80934904893C08F430C1209349042A
:10964000109271031092700330913F07E32FFF27B0
:10965000EE0FFF1FEE58F74F8081918187349105FF
:10966000B4F480914007E82FFF27EE0FFF1FEE585C
:10967000F74F808191810190F081E02DF7FF03C0C9
:10968000F095E195FF4FE734F1050CF478C041E027
:1096900020914007A22FBB27AA0FBB1FAE58B74F80
:1096A0008D919C9111978734910544F0E32FFF270A
:1096B000EE0FFF1FEE58F74F808191818D919C91A5
:1096C0008734910574F080913F07E82FFF27EE0F54
:1096D000FF1FEE58F74F80819181873491050CF080
:1096E00042E0E22FFF27EE0FFF1FEE58F74F808179
:1096F00091818634910574F480913F07E82FFF270C
:10970000EE0FFF1FEE58F74F80819181873491054E
:109710000CF043E0E22FFF27EE0FFF1FEE58F74F4C
:10972000808191818A5B9F4F74F480913F07E82F7D
:10973000FF27EE0FFF1FEE58F74F8081918187348E
:1097400091050CF044E0E22FFF27EE0FFF1FEE58CB
:10975000F74F808191818A5B9F4F74F480913F071E
:10976000E82FFF27EE0FFF1FEE58F74F8081918102
:10977000863491050CF445E0842F0E946531809178
:109780004007E82FFF27EE0FFF1FEE58F74F8081AD
:1097900091810190F081E02DF7FF03C0F095E195F4
:1097A000FF4F7E97CCF480913F07E82FFF27EE0F05
:1097B000FF1FEE58F74F808191818A5B9F4F64F4C1
:1097C00081E0809328051092920388EE93E09093B5
:1097D0000D0380930C0362C00E946E320E94103110
:1097E00080E00E94260A809165070E941394809170
:1097F0002D0980FF10C08091150190911601875BA3
:10980000934038F480911501909116018E5E92403C
:1098100010F40E949D1E81E00E94473B982F809388
:10982000920321E020930A03579A80910D05882323
:1098300019F5992339F52093A10127C080819181E1
:10984000855B9F4F4CF5809149048F5F809349045D
:10985000893C20F12093A6032093490410927103C0
:109860001092700382E00E94473B982F80939203EE
:1098700080910D05882311F087E005C0992311F42C
:1098800081E001C088E18093A1010E946E3268E707
:1098900070E00E94633A02C020934904809141071E
:1098A000E82FFF27EE0FFF1FEE58F74F80819181C1
:1098B0008B5A9F4F0CF088C12091A207E22FFF27FF
:1098C000EF77F070EE0FFF1FEA55F74F808191811F
:1098D000069714F084E606C0808191818B5F9F4FCC
:1098E0001CF48CE980934C048091A603E09142071C
:1098F000882309F014C1FF27EE0FFF1FEE58F74F22
:1099000080819181855B9F4F9CF48091AD0783FDA1
:109910000BC0E22FFF27EE0FFF1FEE58F74F80819D
:109920009181855B9F4FDCF08091A2078823B9F07D
:109930008091AD0783FFF0C08091A207E82FFF2739
:10994000EE0FFF1FEE58F74F80819181875F9F4F89
:109950000CF4E2C080914C04843609F0DDC0209103
:109960009203222329F080916F03886080936F0314
:109970008091170190911801A0911901B0911A01DD
:109980008093E0069093E106A093E206B093E3068D
:109990001092190310921A0310921B0310921C03C9
:1099A0001092A1031092A2031092A3031092A40399
:1099B0001092220310922303109224031092250385
:1099C00080914A048F5F80934A048E3F08F4EEC072
:1099D00010924A0480910D05882309F092C0222339
:1099E00009F48FC080918504882309F08AC081E042
:1099F00090E0909371038093700381E08093A603BD
:109A000010923304109234041092350410923604EC
:109A10001092D1031092D2031092D3031092D40368
:109A20001092CD031092CE031092CF031092D00368
:109A300080915A07E82EFF240027112780913109D1
:109A4000909132099C01442737FD4095542FC8015D
:109A5000B7010E94AC98DC01CB018093E1039093A5
:109A6000E203A093E303B093E40380914109909152
:109A700042099C01442737FD4095542FC801B70186
:109A80000E94AC98DC01CB018093D9039093DA0358
:109A9000A093DB03B093DC03809101049091020456
:109AA000A0910304B09104048093DD039093DE033E
:109AB000A093DF03B093E0038091F9039091FA0340
:109AC000A091FB03B091FC038093D5039093D60340
:109AD000A093D703B093D8031092C9031092CA037E
:109AE0001092CB031092CC031092C5031092C603C0
:109AF0001092C7031092C80384E68093910384E315
:109B000050C08CED95E090930D0380930C032223BD
:109B100009F04CC081E045C010924A0447C0FF27BD
:109B2000EE0FFF1FEE58F74F808191818C34910525
:109B30009CF08091AD0783FD0BC0E22FFF27EE0F55
:109B4000FF1FEE58F74F80819181855B9F4FCCF0CE
:109B50008091A2078823A9F08091AD0783FF24C0DC
:109B60008091A207E82FFF27EE0FFF1FEE58F74F57
:109B7000808191818E5C9F4FBCF480914C048C3924
:109B800099F480914B048F5F80934B048B3F70F06E
:109B90001092A60310924B0410927103109270035E
:109BA00086E28093A10102C010924B0480916A0367
:109BB00090916B0353E0883E9507B8F5019690931A
:109BC0006B0380936A0331C010924C0410926B03B4
:109BD00010926A032AC02E5E324038F180914C09FF
:109BE00090914D098059914000F58091A103909189
:109BF000A203A091A303B091A4038C5D9540A04063
:109C0000B0409CF480E395E790936B0380936A03E4
:109C100080917003909171038A5E934030F089EED9
:109C200093E0909371038093700380913A01815087
:109C300080933A0180913A018F3F21F080916F0328
:109C400084FFA9C30E946946B090550780915504CE
:109C5000909156049C01220F331F280F391FC0908A
:109C60003F07AC2DBB27AA0FBB1FFD01EE58F74FD6
:109C70004B2D552780819181849F7001859FF00C29
:109C8000949FF00C11242E0D3F1D37FF02C02D5F55
:109C90003F4FB9017595679575956795AA55B74F6B
:109CA00080915607082F11278D919C91809F9001DC
:109CB000819F300D909F300D1124620F731F7093A0
:109CC00056046093550480915704909158049C0168
:109CD000220F331F280F391FD0904007AD2DBB270F
:109CE000AA0FBB1FFD01EE58F74F80819181849F21
:109CF000F001859FF00D949FF00D11242E0F3F1F52
:109D000037FF02C02D5F3F4FA901559547955595E7
:109D10004795AA55B74F8D919C91809F7001819F67
:109D2000F00C909FF00C11244E0D5F1D50935804C1
:109D30004093570480917C03882309F448C0CB01E9
:109D400077FD0396DC01B595A795B595A795CA0152
:109D500057FD0396FC01F595E795F595E7958091FC
:109D60009A01682F772767FD70956A9F90016B9F16
:109D7000300D7A9F300D112480918704482F55278C
:109D800047FD50954E9FC0014F9F900D5E9F900DD7
:109D90001124280F391F37FF02C0295F3F4F93E07E
:109DA000359527959A95E1F73093B8032093B7033B
:109DB0006E9F90016F9F300D7E9F300D11244A9F42
:109DC000C0014B9F900D5A9F900D11243FC0809170
:109DD000A007E82FFF27EE5BFE4F868180939A0154
:109DE000908190938704A82FBB27A7FDB095A69FCD
:109DF0009001A79F300DB69F300D1124E92FFF274A
:109E0000E7FDF095E49FC001E59F900DF49F900D54
:109E10001124280F391F37FF02C0295F3F4F83E00D
:109E2000359527958A95E1F73093B8032093B703CA
:109E3000A49F9001A59F300DB49F300D1124E69F83
:109E4000C001E79F900DF69F900D1124281B390B40
:109E500037FF02C0295F3F4F03E0359527950A95EC
:109E6000E1F73093B6032093B50380914207E82FC2
:109E7000FF27EE0FFF1FEE58F74F808191819095DD
:109E800081959F4F9093B4038093B30385309105E0
:109E900014F0049705C00FEF8C3F900734F404963C
:109EA0009093B4038093B30304C01092B403109250
:109EB000B30380917304882309F43EC0282F33270D
:109EC0008091B7039091B80397FD079613E095959D
:109ED00087951A95E1F7289FA001299F500D389F7B
:109EE000500D1124CA0157FD0F96B4E09595879542
:109EF000BA95E1F79093B8038093B7038091B503C7
:109F00009091B60397FD0796A3E095958795AA953E
:109F1000E1F7289FB001299F700D389F700D112423
:109F2000CB0177FD0F96F4E095958795FA95E1F7CB
:109F30009093B6038093B5038090B7039090B803D5
:109F40008091760490917704881A990A9092B803C8
:109F50008092B7030091B5031091B6038091740409
:109F600090917504081B190B1093B6030093B50369
:109F700080914107E82FFF27EE0FFF1FEE58F74FA4
:109F8000E080F1808FE790E0E80EF91EF092B203D6
:109F9000E092B10380916F019927AA2797FDA095C0
:109FA000BA2FBC01CD010E942098DC01CB0120E03A
:109FB00030E040E251E4BC01CD010E948E97DC010B
:109FC000CB01BC01CD010E94F297DC01CB01809353
:109FD0003B0980916E018093130980916D0199274F
:109FE000AA2797FDA095BA2FBC01CD010E94209809
:109FF000DC01CB0120E030E040E251E4BC01CD01C6
:10A000000E948E97DC01CB01BC01CD010E94F2972A
:10A01000DC01CB018093EA0880916C0180930209F6
:10A020008091340580FF59C080914409813808F43B
:10A0300054C080912D05992787FD90952B2D3327AE
:10A04000829FD001839FB00D929FB00D11248A0E84
:10A050009B1E9092B8038092B70380912E0599279A
:10A0600087FD9095829FF001839FF00D929FF00DE8
:10A0700011240E0F1F1F1093B6030093B503809198
:10A080002F05282F332727FD30958091B30390911A
:10A09000B403820F931F9093B4038093B303809112
:10A0A0003105282F332727FD3095809150079927B8
:10A0B000289F8001299F100D389F100D11241093A7
:10A0C0004101009340018091300599278E159F052D
:10A0D00024F49093B2038093B1038091B1039091E3
:10A0E000B20397FF04C01092B2031092B1038091A3
:10A0F0002D0982FF02C0109213094091B7035091BD
:10A10000B803CA0157FD03969C01359527953595EF
:10A11000279537FF03C0309521953F4F80917403F9
:10A120009091750382179307B4F4CA0157FF03C0D7
:10A13000909581959F4F97FD039695958795959559
:10A14000879590937503809374038536910544F049
:10A1500084E690E001C001979093750380937403A7
:10A160004091B5035091B603CA0157FD03969C0177
:10A17000359527953595279537FF03C0309521955F
:10A180003F4F809172039091730382179307B4F449
:10A19000CA0157FF03C0909581959F4F97FD039685
:10A1A0009595879595958795909373038093720302
:10A1B0008536910544F084E690E001C001979093C4
:10A1C00073038093720380916F0384FF08C0109221
:10A1D0007503109274031092730310927203ED2DA5
:10A1E000FF27EE0FFF1FEE58F74F40917A07242FFD
:10A1F0003327808191812817390744F48091AA0779
:10A2000082FF04C081E08093880313C0ED2DFF27F7
:10A21000EE0FFF1FEE58F74F842F992720917B07F1
:10A22000821B9109208131812817390714F410927B
:10A23000880340914007E42FFF27EE0FFF1FEE58E1
:10A24000F74F50917A07852F992722273327281B0C
:10A25000390B808191818217930744F48091AA077A
:10A2600083FF04C081E08093870316C08091870339
:10A27000882391F0E42FFF27EE0FFF1FEE58F74FD2
:10A2800080917B079927851B910920813181821755
:10A29000930714F410928703EC2DFF27EE0FFF1F96
:10A2A000EE58F74F40917A07242F33278081918110
:10A2B0002817390744F48091AA0780FF04C081E081
:10A2C0008093850317C080918503882399F0EC2D36
:10A2D000FF27EE0FFF1FEE58F74F842F992720918D
:10A2E0007B07821B9109208131812817390714F4DB
:10A2F0001092850340913F07E42FFF27EE0FFF1FC9
:10A30000EE58F74F50917A07852F99272227332748
:10A31000281B390B808191818217930744F4809127
:10A32000AA0781FF04C081E08093860316C0809154
:10A330008603882391F0E42FFF27EE0FFF1FEE58CE
:10A34000F74F80917B079927851B910920813181E7
:10A350008217930714F41092860380918803882350
:10A3600019F480918703811181E0809389038091A2
:10A370008503882321F480918603882351F081E0AE
:10A3800080938A03109289031092880310928703A6
:10A3900002C080938A0380918903882321F48091ED
:10A3A0008A03882369F080917907992729813A8166
:10A3B0008217930714F49A83898381E08093BD0305
:10A3C00080916E0399279C012470307082FF2DC00C
:10A3D0008091760490917704909581959F4F90930A
:10A3E000B8038093B703809174049091750490959D
:10A3F00081959F4F9093B6038093B50380917C0124
:10A4000090917D019093B2038093B10380912D09C7
:10A410008B778B6680932D09809111098C7B8093BB
:10A42000110988EC809375011EC080916F0384FF31
:10A430001AC03093B4032093B3033093B80320932E
:10A44000B7033093B6032093B5039AE590933B0985
:10A4500088E7809313099093EA0880930209109289
:10A46000890310928A038091050990910609A091B1
:10A470000709B0910809209101043091020440912C
:10A48000030450910404820F931FA41FB51F8093EF
:10A49000050990930609A0930709B09308098091D4
:10A4A0000D0990910E09A0910F09B0911009E0904B
:10A4B000F903F090FA030091FB031091FC03EB8287
:10A4C000FC820D831E838E0D9F1DA01FB11F8093E4
:10A4D0000D0990930E09A0930F09B0931009809174
:10A4E000FA089091FB08A091FC08B091FD08E0905B
:10A4F000FD03F090FE030091FF0310910004EF8232
:10A50000F88609871A878E0D9F1DA01FB11F8093A3
:10A51000FA089093FB08A093FC08B093FD08809183
:10A52000EB089091EC08A091ED08B091EE08E09056
:10A53000F503F090F6030091F7031091F803EB8612
:10A54000FC860D871E878E0D9F1DA01FB11F809357
:10A55000EB089093EC08A093ED08B093EE08F09010
:10A560008A03FF86FF2029F480918903882309F458
:10A5700060C01092F1031092F2031092F303109254
:10A58000F4031092ED031092EE031092EF03109279
:10A59000F003109205091092060910920709109213
:10A5A000080910920D0910920E0910920F091092CD
:10A5B00010091092FA081092FB081092FC081092F1
:10A5C000FD081092EB081092EC081092ED08109222
:10A5D000EE088091E1039091E203A091E303B09132
:10A5E000E4038093DD039093DE03A093DF03B09335
:10A5F000E0038091D9039091DA03A091DB03B0913D
:10A60000DC038093D5039093D603A093D703B09334
:10A61000D80310921E0310921D0310928E03109205
:10A620008D031092900310928F030F85002309F081
:10A63000D0C180918903882309F0CBC18091DE06C7
:10A640009091DF06815092402CF48091A6038823DC
:10A6500009F4BFC19090BD09A0905A07209031091C
:10A6600030903209409041095090420919140CF081
:10A67000BBC0BB24CC24DD24CA01B901A6019501CD
:10A680000E94209979018A01809186099091870919
:10A69000281A390AC101AA2797FDA095BA2FE81AEE
:10A6A000F90A0A0B1B0B6B817C818D819E81A601AF
:10A6B00095010E94209959016A0180918809909121
:10A6C0008909481A590AC201AA2797FDA095BA2FED
:10A6D000A81AB90ACA0ADB0A292C332427FC3094A9
:10A6E000432C532CC801B701A20191010E94AC98E0
:10A6F00097FF04C061507E4F8F4F9F4F3B014C012D
:10A7000009E095948794779467940A95D1F7C601E8
:10A71000B501A20191010E94AC9897FF04C061505D
:10A720007E4F8F4F9F4F5B016C0119E0D594C7940A
:10A73000B794A7941A95D1F78091740390917503FB
:10A74000813491053CF480917203909173038134BC
:10A750009105D4F0D401C30197FE03C00196A11D59
:10A76000B11D3C014D019594879477946794D6016F
:10A77000C501D7FE03C00196A11DB11D5C016D018D
:10A78000D594C794B794A7948091BF09282F3327F5
:10A7900027FD3095432F532F2615370548055905BA
:10A7A00014F439014A01992787FD90959095819578
:10A7B0009F4FAA2797FDA095BA2F681679068A069B
:10A7C0009B0614F43C014D012A153B054C055D0523
:10A7D00014F459016A01A816B906CA06DB060CF082
:10A7E000D0C05C016D01CDC0EA2CFF2400271127E9
:10A7F000CA01B901A80197010E94209939014A01B3
:10A80000C101AA2797FDA095BA2F681A790A8A0A6A
:10A810009B0A6B817C818D819E81A80197010E949A
:10A82000209959016A01C201AA2797FDA095BA2F64
:10A83000A81AB90ACA0ADB0AD401C30197FE03C0E9
:10A840000F96A11DB11D3C014D01F4E09594879434
:10A8500077946794FA95D1F7D601C501D7FE03C066
:10A860000F96A11DB11D5C016D01E4E0D594C79464
:10A87000B794A794EA95D1F78091740390917503EA
:10A88000813491053CF4809172039091730381347B
:10A890009105A4F0C401B30123E030E040E050E0B2
:10A8A0000E94209939014A01C601B50123E030E038
:10A8B00040E050E00E94209959016A0180914207CE
:10A8C000E82FFF27EE0FFF1FEE58F74F8081918191
:10A8D0000190F081E02DF7FF03C0F095E195FF4F67
:10A8E0007A97A4F0C401B30123E030E040E050E0E7
:10A8F0000E94209939014A01C601B50123E030E0E8
:10A9000040E050E00E94209959016A0189E180935A
:10A91000880121E262167104810491042CF070E236
:10A92000672E712C812C912C30EE63163FEF73064D
:10A930003FEF83063FEF930644F460EE662E6FEF21
:10A94000762E6FEF862E6FEF962E41E2A416B1049D
:10A95000C104D1042CF050E2A52EB12CC12CD12C75
:10A9600050EEA5165FEFB5065FEFC5065FEFD506A3
:10A9700044F440EEA42E4FEFB42E4FEFC42E4FEF11
:10A98000D42E8091E1039091E203A091E303B09172
:10A99000E40386199709A809B9098093E103909304
:10A9A000E203A093E303B093E4038091D903909171
:10A9B000DA03A091DB03B091DC038A199B09AC098F
:10A9C000BD098093D9039093DA03A093DB03B0937E
:10A9D000DC0380911D0390911E038F3F910509F0C8
:10A9E00008F4C4C56F85662309F04EC580918903BC
:10A9F000882309F049C58091BD03882309F044C527
:10AA000070918207788B772309F43EC58091050900
:10AA100090910609A0910709B0910809B7FF04C0F9
:10AA200081509F4FAF4FBF4FE92EFA2E0B2F1127AA
:10AA300007FD1A95E0920509F092060900930709AF
:10AA40001093080980910D0990910E09A0910F09AA
:10AA5000B0911009B7FF04C081509F4FAF4FBF4F57
:10AA6000892F9A2FAB2FBB27A7FDBA95898B9A8B7D
:10AA7000AB8BBC8B80930D0990930E09A0930F09AB
:10AA8000B093100980915A07A82EBB24CC24DD2452
:10AA90002091F1033091F2034091F3035091F403BC
:10AAA000C601B5010E94AC9897FF04C061507F4F6A
:10AAB0008F4F9F4F672E782E892E992487FC9A946A
:10AAC0006092F1037092F2038092F3039092F40388
:10AAD0002091ED033091EE034091EF035091F0038C
:10AAE000C601B5010E94AC9897FF04C061507F4F2A
:10AAF0008F4F9F4F272E382E492E552447FC5A94AE
:10AB00002092ED033092EE034092EF035092F00357
:10AB10008091E9039091EA03A091EB03B091EC03DB
:10AB2000B7FF04C081509F4FAF4FBF4F892F9A2F5F
:10AB3000AB2FBB27A7FDBA958093E9039093EA0357
:10AB4000A093EB03B093EC03D801C70186199709D2
:10AB5000A809B90980933F0490934004A09341044D
:10AB6000B093420420918107E22EFF240027112791
:10AB7000BC01CD01A80197010E94209959016A01E9
:10AB800020934D0430934E0440934F04509350044F
:10AB900089899A89AB89BC8982199309A409B50965
:10ABA0008093430490934404A0934504B0934604D7
:10ABB000BC01CD01A80197010E9420992093510466
:10ABC000309352044093530450935404D601C5016A
:10ABD000D7FE04C081509F4FAF4FBF4F892F9A2F90
:10ABE000AB2FBB27A7FDBA9590938E0380938D035F
:10ABF00057FF04C021503F4F4F4F5F4FBB2757FDBA
:10AC0000BA95A52F942F832F9093900380938F0351
:10AC1000809174039091750381349105DCF48091E7
:10AC200072039091730381349105A4F480914207DB
:10AC3000E82FFF27EE0FFF1FEE58F74F808191811D
:10AC40000190F081E02DF7FF03C0F095E195FF4FF3
:10AC50007A97E4F08091BD098F3FC1F480918D0314
:10AC600090918E0397FD01969595879590938E030D
:10AC700080938D0380918F039091900397FD0196AF
:10AC8000959587959093900380938F038091FA0810
:10AC90009091FB08A091FC08B091FD08B7FF04C09B
:10ACA00081509F4FAF4FBF4F892F9A2FAB2FBB279C
:10ACB000A7FDBA958093FA089093FB08A093FC082F
:10ACC000B093FD088091EB089091EC08A091ED08FD
:10ACD000B091EE08B7FF04C081509F4FAF4FBF4FF8
:10ACE000892F9A2FAB2FBB27A7FDBA958093EB082E
:10ACF0009093EC08A093ED08B093EE0880910104C6
:10AD000090910204A0910304B09104042F8138852E
:10AD100049855A85281B390B4A0B5B0B2093370456
:10AD2000309338044093390450933A048091F903E6
:10AD30009091FA03A091FB03B091FC03EB84FC8497
:10AD40000D851E85E81AF90A0A0B1B0BE0923B04DD
:10AD5000F0923C0400933D0410933E0420933F0482
:10AD6000309340044093410450934204E0924304E2
:10AD7000F092440400934504109346048091DD034F
:10AD80009091DE03A091DF03B091E003821B930B4F
:10AD9000A40BB50B8093DD039093DE03A093DF0338
:10ADA000B093E0038091D5039091D603A091D7038F
:10ADB000B091D8038E199F09A00BB10B8093D503D6
:10ADC0009093D603A093D703B093D80388898823A0
:10ADD000E1F02091BB033091BC03213831054CF0E8
:10ADE000809113049091140401969093140480931D
:10ADF000130420583F4F4CF4809113049091140495
:10AE0000019790931404809313041092BC03109242
:10AE1000BB0381E090E090935A0480935904E09042
:10AE20003F04F09040040091410410914204D80185
:10AE3000C70117FF07C088279927DC018E199F09D2
:10AE4000A00BB10B81509240A040B04034F084E0A0
:10AE500090E090935A048093590480915F049091FC
:10AE60006004A0916104B0916204209105093091C1
:10AE700006094091070950910809821B930BA40B06
:10AE8000B50B815E914BAF4FBF4F8F539C49A04094
:10AE9000B04028F08091BE0989310CF4FFC021E058
:10AEA000E21620E1F20620E0020720E012070CF48F
:10AEB00073C080915B04882309F46AC0D801C7017C
:10AEC00017FF07C088279927DC018E199F09A00B5F
:10AED000B10B9C01AD01B7FF04C021503E4F4F4F55
:10AEE0005F4FF9E05595479537952795FA95D1F736
:10AEF0008091590490915A04820F931F90935A04A1
:10AF000080935904D801C70117FF03C00796A11DFC
:10AF1000B11DE3E0B595A79597958795EA95D1F78B
:10AF200080934D0490934E04A0934F04B09350042B
:10AF300089589341A040B04064F088E893E1A0E0D4
:10AF4000B0E080934D0490934E04A0934F04B093CF
:10AF5000500420914D0430914E0440914F04509183
:10AF6000500457FF04C021503F4F4F4F5F4F232FD6
:10AF7000342F452F552747FD5A9580918D03909189
:10AF80008E03820F931F90938E0380938D0306C0D0
:10AF900081E080935B0402C010925B0440E0E41601
:10AFA00040EFF4064FEF04074FEF14070CF073C0A7
:10AFB00080915C04882309F46AC0D801C70117FF97
:10AFC00007C088279927DC018E199F09A00BB10BB8
:10AFD0009C01AD01B7FF04C021503E4F4F4F5F4F62
:10AFE00069E055954795379527956A95D1F78091F2
:10AFF000590490915A04820F931F90935A0480939E
:10B000005904D801C70117FF03C00796A11DB11D40
:10B0100023E0B595A795979587952A95D1F78093C5
:10B020004D0490934E04A0934F04B093500488575E
:10B030009C4EAF4FBF4F64F488E79CEEAFEFBFEF7D
:10B0400080934D0490934E04A0934F04B09350040A
:10B0500020914D0430914E0440914F045091500482
:10B0600057FF04C021503F4F4F4F5F4F232F342FC6
:10B07000452F552747FD5A9580918D0390918E035A
:10B08000820F931F90938E0380938D0311C081E0F4
:10B0900080935C040DC010925C040AC010925A04A4
:10B0A0001092590484E690E0909387018093860182
:10B0B0006889262F33278091590490915A042817C4
:10B0C000390724F430935A04209359041091BE098F
:10B0D000112379F0212F332727FD309580915904D2
:10B0E00090915A042817390724F430935A04209376
:10B0F000590440913F045091400460914104709183
:10B100004204413851056105710574F080911704BE
:10B11000909118042091590430915A04820F931F82
:10B12000909318048093170440585F4F6F4F7F4FE0
:10B1300074F480911704909118042091590430916F
:10B140005A04821B930B909318048093170481E098
:10B1500090E090935A0480935904C0904304D09097
:10B160004404E0904504F0904604D701C601F7FE80
:10B1700007C088279927DC018C199D09AE09BF09F2
:10B1800081509240A040B04034F084E090E0909331
:10B190005A04809359048091630490916404A091AF
:10B1A0006504B091660420910D0930910E0940911B
:10B1B0000F0950911009821B930BA40BB50B815EF4
:10B1C000914BAF4FBF4F8F539C49A040B04018F0F8
:10B1D00019310CF4FFC001E0C01600E1D00600E018
:10B1E000E00600E0F0060CF473C080915D04882353
:10B1F00009F46AC0D701C601F7FE07C0882799275E
:10B20000DC018C199D09AE09BF099C01AD01B7FF96
:10B2100004C021503E4F4F4F5F4F09E05595479571
:10B22000379527950A95D1F78091590490915A0442
:10B23000820F931F90935A0480935904D701C6013B
:10B24000F7FE03C00796A11DB11D13E0B595A795A4
:10B25000979587951A95D1F780935104909352044E
:10B26000A0935304B093540489589341A040B04034
:10B2700064F088E893E1A0E0B0E0809351049093FB
:10B280005204A0935304B09354042091510430917C
:10B290005204409153045091540457FF04C021506C
:10B2A0003F4F4F4F5F4F232F342F452F552747FDDB
:10B2B0005A9580918F0390919003820F931F9093E2
:10B2C000900380938F0306C081E080935D0402C0E9
:10B2D00010925D0420E0C21620EFD2062FEFE206A6
:10B2E0002FEFF2060CF073C080915E04882309F4FE
:10B2F0006AC0D701C601F7FE07C088279927DC017D
:10B300008C199D09AE09BF099C01AD01B7FF04C0AE
:10B3100021503E4F4F4F5F4FE9E055954795379588
:10B320002795EA95D1F78091590490915A04820F9C
:10B33000931F90935A0480935904D701C601F7FED6
:10B3400003C00796A11DB11D73E0B595A79597950C
:10B3500087957A95D1F78093510490935204A093E6
:10B360005304B093540488579C4EAF4FBF4F64F4BE
:10B3700088E79CEEAFEFBFEF8093510490935204A7
:10B38000A0935304B093540420915104309152047B
:10B39000409153045091540457FF04C021503F4F33
:10B3A0004F4F5F4F232F342F452F552747FD5A9579
:10B3B00080918F0390919003820F931F909390033D
:10B3C00080938F0311C081E080935E040DC01092C2
:10B3D0005E040AC010925A041092590484E690E068
:10B3E00090938701809386014889242F3327809189
:10B3F000590490915A042817390724F430935A04B9
:10B40000209359048091BE09882379F0282F33278F
:10B4100027FD30958091590490915A0428173907D7
:10B4200024F430935A0420935904409143045091DA
:10B43000440460914504709146044138510561050A
:10B44000710574F0809115049091160420915904AF
:10B4500030915A04820F931F909316048093150421
:10B4600040585F4F6F4F7F4FCCF4809115049091FF
:10B4700016042091590430915A04821B930B909327
:10B480001604809315040AC01092900310928F0343
:10B4900010928E0310928D031092BD0380911309B8
:10B4A000882341F41092900310928F0310928E0320
:10B4B00010928D038091050990910609A0910709CA
:10B4C000B091080980935F0490936004A093610495
:10B4D000B093620480910D0990910E09A0910F091B
:10B4E000B09110098093630490936404A093650461
:10B4F000B09366041092F1031092F2031092F303DA
:10B500001092F4031092ED031092EE031092EF03E9
:10B510001092F0031092E9031092EA031092EB03E9
:10B520001092EC0310920509109206091092070977
:10B530001092080910920D0910920E0910920F092D
:10B54000109210091092FA081092FB081092FC0851
:10B550001092FD081092EB081092EC081092ED0882
:10B560001092EE0810921E0310921D03E090B30398
:10B57000F090B403C701F7FE04C0882799278E19FD
:10B580009F0904973CF080912D0984FD03C082E35C
:10B590008093910310915707A12EBB24CC24DD2466
:10B5A000B701882777FD8095982F9701F7FE04C093
:10B5B000222733272E193F09442737FD4095542F62
:10B5C0000E94AC989B01AC01C601B5010E94AC98E9
:10B5D00097FF04C061507E4F8F4F9F4F59E0959564
:10B5E0008795779567955A95D1F79B01812F992774
:10B5F0008E9DD0018F9DB00D9E9DB00D1124CD016B
:10B60000B7FD03969595879595958795280F391FD2
:10B6100080916A0390916B038150924010F020E07A
:10B6200030E08091930390919403280F391F4427B1
:10B6300037FD4095542F20933304309334044093C6
:10B640003504509336048091D1039091D203A09198
:10B65000D303B091D403821B930BA40BB50B80933F
:10B66000D1039093D203A093D303B093D403815515
:10B67000934CA040B04064F080E593ECA0E0B0E0D3
:10B680008093D1039093D203A093D303B093D403B8
:10B690008091D1039091D203A091D303B091D403B0
:10B6A000805B9C43AF4FBF4F64F480EB9CE3AFEFF4
:10B6B000BFEF8093D1039093D203A093D303B093B1
:10B6C000D40300918A0110918B0117FDFCC0809179
:10B6D0002D0983FFF8C080918901815080938901F1
:10B6E000882309F0F4C08DE08093890180910104E2
:10B6F00090910204A0910304B0910404B7FF04C028
:10B7000081509E4FAF4FBF4F39E0B595A7959795A4
:10B7100087953A95D1F77C0197FF04C0F094E194A6
:10B72000F108F3948091F9039091FA03A091FB033F
:10B73000B091FC03B7FF04C081509E4FAF4FBF4F85
:10B7400029E0B595A795979587952A95D1F79C01FE
:10B7500097FF03C0309521953F4FE216F3060CF496
:10B760007901B701F7FE02C0695F7F4F2B0183E0CB
:10B77000559447948A95E1F722E030E0420E531E3B
:10B7800060903D0970903E0980903F09909040097B
:10B7900020913C0130913D0140913E0150913F018B
:10B7A000C401B3010E94209959016A013093E9084C
:10B7B0002093E808021B130BC801845E9D4F68E6C6
:10B7C00071E00E94EB989C01245B304080918601DF
:10B7D00090918701009731F00197909387018093B2
:10B7E00086011BC049E1E416F104BCF48091BB035F
:10B7F0009091BC03820F931F9093BC038093BB0373
:10B8000080919103882349F081508093910388238C
:10B8100021F4B092C003A092BF0380918601909161
:10B820008701892BF9F4809188019927289FB0011D
:10B83000299F700D389F700D1124CB01B2010E9419
:10B84000EB98CB01AA2797FDA095BA2F680E791E19
:10B850008A1E9B1E60923D0970923E0980923F09AC
:10B860009092400980919103882369F58091BF03EC
:10B870009091C0032091E8083091E908821B930B56
:10B88000845E9D4F68E671E00E94EB989C01245B0A
:10B8900030408091720186959927289FD001299F79
:10B8A000B00D389FB00D11249D01B7FF02C0215F7C
:10B8B0003F4F04E0359527950A95E1F730939403BF
:10B8C0002093930304C010929403109293038091E9
:10B8D000BD03882381F01092C5031092C603109215
:10B8E000C7031092C8031092C9031092CA031092A2
:10B8F000CB031092CC03F0908A03FF20F1F48091E7
:10B900001309282F3327442755278091010490914C
:10B910000204A0910304B0910404BC01CD010E9473
:10B92000AC98DC01CB01BC01CD0128EF3AE240E04C
:10B9300050E00E942099390102C066247724E090EB
:10B940008903EE20F1F480911309282F332744272F
:10B9500055278091F9039091FA03A091FB03B091D0
:10B96000FC03BC01CD010E94AC98DC01CB01BC0101
:10B97000CD0128EF3AE240E050E00E9420992901F1
:10B9800002C0442455248091E5089091E608893C42
:10B9900091051CF088EC90E005C088539F4F34F46B
:10B9A00088E39FEF9093E6088093E5088091F10883
:10B9B0009091F208893C91051CF088EC90E005C05C
:10B9C00088539F4F34F488E39FEF9093F20880935D
:10B9D000F1088091F3089091F408AA2797FDA095AB
:10B9E000BA2F20913B09A22EBB24CC24DD24BC011C
:10B9F000CD01A60195010E94AC989B01AC018091FC
:10BA0000E5089091E608AA2797FDA095BA2F17E0C0
:10BA1000880F991FAA1FBB1F1A95D1F7280F391F2E
:10BA20004A1F5B1F57FF04C0215C3F4F4F4F5F4FC2
:10BA3000A6E05595479537952795AA95D1F78301A7
:10BA4000020F131F1093F4080093F3088091E3088A
:10BA50009091E408AA2797FDA095BA2FBC01CD01CB
:10BA6000A60195010E94AC989B01AC018091F10860
:10BA70009091F208AA2797FDA095BA2FF7E0880FBA
:10BA8000991FAA1FBB1FFA95D1F7280F391F4A1F0C
:10BA90005B1F57FF04C0215C3F4F4F4F5F4FE6E0F5
:10BAA0005595479537952795EA95D1F74201820E2E
:10BAB000931E9092E4088092E30880913609909159
:10BAC0003709880F991FAA2797FDA095BA2F2091B3
:10BAD000EA08332744275527BC01CD010E94AC98C2
:10BAE0005B016C0197FF08C02FE330E040E050E0BD
:10BAF000A20EB31EC41ED51E76E0D594C794B7948B
:10BB0000A7947A95D1F780910209282F33274427EB
:10BB100055278091E5039091E603A091E703B0914A
:10BB2000E803BC01CD010E94AC98DC01CB01BC0153
:10BB3000CD0120EF35E540E050E00E942099B501AD
:10BB4000620F731F709337096093360901501041DB
:10BB500034F080E090E19093F4088093F3088091B2
:10BB6000F3089091F4088050904F34F480E090EF07
:10BB70009093F4088093F30851E0851650E1950600
:10BB800034F080E090E19093E4088093E3088091A2
:10BB9000E3089091E4088050904F34F480E090EFF7
:10BBA0009093E4088093E3086150704134F080E0A2
:10BBB00090E19093370980933609809136099091EE
:10BBC00037098050904F34F480E090EF909337091C
:10BBD0008093360980910001482F552780911F01DD
:10BBE000909120014817590794F420911F0130913A
:10BBF000200109811A81049FC001059F900D149FA7
:10BC0000900D1124B9010E94D7987A836983298104
:10BC10003A81220F331F220F331F3A8329838091E9
:10BC20002D0980FD02C00C944E68EE2011F00C949A
:10BC30004E68FF2011F00C944E688824992480915E
:10BC40008B0390918C039093C4068093C3068091DC
:10BC5000190490911A04892BD9F5809115019091BE
:10BC600016018959934058F087B5803F20F48091A0
:10BC70002103815011C081E08093720455C08091EE
:10BC800015019091160184369105E8F487B580314D
:10BC9000B0F0809121038F5F809321039FE08902A0
:10BCA000900111248091EA06821B87BD8CE291E00D
:10BCB00090930D0380930C038EE591E031C081E0F9
:10BCC0008093710431C0F0927104F09272042CC020
:10BCD0009092200380921F0380916703882321F0B4
:10BCE00081E00E949F9217C08091A1039091A203CE
:10BCF000A091A303B091A40354E0880F991FAA1F39
:10BD0000BB1F5A95D1F78093220390932303A093EE
:10BD10002403B09325038091190490911A0401978C
:10BD200090931A048093190480912D092091750134
:10BD300081FF3CC0223348F580918C018150809373
:10BD40008C018F3F09F052C08091A101882339F402
:10BD50008091BE03882319F088E28093A10110929C
:10BD6000BE038091A1039091A203A091A303B0917F
:10BD7000A40380939D0390939E03A0939F03B0938D
:10BD8000A00381E080938C0131C0273478F1809149
:10BD9000A101882339F48091BE03882319F487E236
:10BDA0008093A10188EC80938C011DC0809140019B
:10BDB00090914101820F911D209150073327829F5E
:10BDC000A001839F500D929F500D1124CA01AA27F4
:10BDD00097FDA095BA2F80939D0390939E03A09307
:10BDE0009F03B093A00381E08093BE038091010480
:10BDF00090910204A0910304B0910404E0903C01EE
:10BE0000F0903D0100913E0110913F01BC01CD0138
:10BE1000A80197010E94209959016A018091F903B4
:10BE20009091FA03A091FB03B091FC03BC01CD01FA
:10BE3000A80197010E942099B901C5010E94CC96E2
:10BE40009093FF088093FE08CC9734F08CE390E049
:10BE50009093FF088093FE088091FE089091FF0860
:10BE60000E94D7749093FF088093FE0880E280932D
:10BE70003B0110929C0310929B038091BE03882388
:10BE800009F470C780916F0399279C01207130706D
:10BE900084FD68C780916E03826080936E03709109
:10BEA0001109872F992741E0C42ED12CC822D9220D
:10BEB00080FD04C080912D0981FD10C0E980FA80C9
:10BEC000309368042093670430939C0320939B0372
:10BED00080916F03806C80936F03DFC280916F034A
:10BEE00081FFAEC200917C0110917D01C8010F96C7
:10BEF000A090B103B090B2038A159B050CF06EC000
:10BF000080917104882309F069C08091690490913F
:10BF10006A04459784F08091190390911A03A091C7
:10BF20001B03B0911C0380939D0390939E03A093E9
:10BF30009F03B093A00380916F0387FF15C080918A
:10BF40006F038F7780936F038091190390911A0389
:10BF5000A0911B03B0911C0380939D0390939E03BB
:10BF6000A0939F03B093A00380916F03806480939C
:10BF70006F03E090EF08EE20F1F080919D03909127
:10BF80009E03A0919F03B091A003BC01CD0124E6C4
:10BF900030E040E050E00E9420998E2D9927AA279A
:10BFA000BB2782179307A407B5072CF4D0929C03F4
:10BFB000C0929B0310C0C501801B910B0F9797FF88
:10BFC00003C0909581959F4F90939C0380939B0312
:10BFD0008BE280933B011092950334C1C8010F9707
:10BFE000A816B906C4F5209172042223A1F5809108
:10BFF0006F0386FF15C080916F038F7B80936F0363
:10C000008091190390911A03A0911B03B0911C0316
:10C0100080939D0390939E03A0939F03B093A003EE
:10C0200080916F03806880936F03C501801B910B23
:10C030000F9697FF03C0909581959F4F909581959E
:10C040009F4F90939C0380939B038DE280933B01D1
:10C0500020939503F7C08DE380933B016091960395
:10C06000662371F1209197033091980340919903D1
:10C0700050919A0380919D0390919E03A0919F03FC
:10C08000B091A00382179307A407B507CCF4809161
:10C090006F03806480936F03862F992790939C038E
:10C0A00080939B038AE0809395038EE580933B0108
:10C0B00080916F0387FFC6C080916F038F7733C075
:10C0C000662309F443C0209197033091980340916F
:10C0D000990350919A0380919D0390919E03A091A2
:10C0E0009F03B091A003281739074A075B0774F52F
:10C0F00080916F03806880936F03862F99279095B6
:10C1000081959F4F90939C0380939B0386EF809330
:10C11000950386E780933B0180916F0386FF92C071
:10C1200080916F038F7B80936F03809119039091AF
:10C130001A03A0911B03B0911C0380939D0390935D
:10C140009E03A0939F03B093A0037CC080916F03D4
:10C15000807C09F477C080919503882309F04CC056
:10C160008091190390911A03A0911B03B0911C03B5
:10C17000885C9040A040B04020919D0330919E0388
:10C1800040919F035091A00382179307A407B5071E
:10C190006CF08091190390911A03A0911B03B09148
:10C1A0001C03885C9040A040B0401DC080911903E2
:10C1B00090911A03A0911B03B0911C0388539F4FC9
:10C1C000AF4FBF4F281739074A075B07BCF0809174
:10C1D000190390911A03A0911B03B0911C0388537B
:10C1E0009F4FAF4FBF4F80939D0390939E03A093AB
:10C1F0009F03B093A00302C01092950380916F0338
:10C200008F7380936F03109268041092670471FF1C
:10C2100006C084EF91E090930D0380930C0380910E
:10C22000A503882379F48091A1039091A203A091A2
:10C23000A303B091A403C397A105B1051CF081E04D
:10C240008093A503609167047091680480919B03BB
:10C2500090919C03680F791F709368046093670442
:10C26000CB0177FF04C088279927861B970B855F32
:10C2700091400CF4CEC040919503442389F1809104
:10C2800097039091980320919D0330919E03821B08
:10C29000930B0996439748F48091970390919803E4
:10C2A000A0919903B0919A0312C0242F332727FD40
:10C2B0003095432F532F80919D0390919E03A09121
:10C2C0009F03B091A003820F931FA41FB51F8093FB
:10C2D0009D0390939E03A0939F03B093A00324C05B
:10C2E0008091500720919D0330919E0340919F03C0
:10C2F0005091A0031616170644F463E00E94CB98F1
:10C30000280F311D411D511D07C063E00E94CB98CD
:10C31000281B31094109510920939D0330939E0345
:10C3200040939F035093A0031092680410926704F7
:10C33000E090A103F090A2030091A3031091A40345
:10C34000D801C70180509440A040B04020919D0387
:10C3500030919E0340919F035091A0038217930751
:10C36000A407B5075CF4D801C70180509C4FAF4FBC
:10C37000BF4F281739074A075B0744F080939D0396
:10C3800090939E03A0939F03B093A0038091110903
:10C3900081FF06C084E690E090930D0380930C0328
:10C3A000809154078823A9F580919603882389F505
:10C3B00040918B0350918C0357FF02C04D5F5F4F3C
:10C3C000559547955595479580911F01909120016E
:10C3D000209100013327489FB001499F700D589F5D
:10C3E000700D1124CB01B9010E94EB9870937D016F
:10C3F00060937C01663471051CF486E490E005C00E
:10C400006739710534F086E990E090937D0180935F
:10C410007C018091190490911A04892BD1F18091AB
:10C42000190390911A03A0911B03B0911C038093F0
:10C430009D0390939E03A0939F03B093A00329C0F4
:10C440008091A1039091A203A091A303B091A403B2
:10C4500080599140A040B04080939D0390939E03EB
:10C46000A0939F03B093A00380915407882311F0F9
:10C47000992702C088E790E090937D0180937C012A
:10C4800089819A8190938C0380938B038EE28093B1
:10C490003B01E0908B03F0908C0380911903909105
:10C4A0001A03A0911B03B0911C0320919D033091AE
:10C4B0009E0340919F035091A003281739074A0714
:10C4C0005B0724F08091110980FD98C48091670377
:10C4D0006091190470911A04882309F07CC2672BBB
:10C4E00049F0E0908B03F0908C0310926A04109254
:10C4F0006904E1C08091190390911A03A0911B0374
:10C50000B0911C03821B930BA40BB50B80933704D3
:10C5100090933804A0933904B0933A048230E0E851
:10C520009E07EFEFAE07EFEFBE072CF481E090E837
:10C53000AFEFBFEF09C08F5F9F47A040B04064F0EE
:10C540008FEF9FE7A0E0B0E080933704909338042A
:10C55000A0933904B0933A04809137049091380441
:10C5600090936A048093690480917401282F332783
:10C57000442755278091370490913804A0913904BD
:10C58000B0913A04BC01CD010E94AC9897FF04C061
:10C59000615E7F4F8F4F9F4F25E0959587957795EB
:10C5A00067952A95D1F76093370470933804809388
:10C5B000390490933A0465300EEF70070FEF80074F
:10C5C0000FEF90072CF484E09EEFAFEFBFEF09C0B0
:10C5D000605074408040904064F080E094E0A0E0BF
:10C5E000B0E08093370490933804A0933904B0935B
:10C5F0003A04809037049090380420911F033091C2
:10C60000200337FF02C0295F3F4F03E03595279590
:10C610000A95E1F74FEF223834071CF421E83FEF89
:10C6200005C02038310514F020E830E0C901AA2700
:10C6300097FDA095BA2F20917601332744275527DF
:10C64000BC01CD010E94AC9897FF04C06D5F7F4F85
:10C650008F4F9F4F12E095958795779567951A951F
:10C66000D1F79B015FEF613075071CF420E03FEFCD
:10C6700006C06F3F710519F014F020E031E08091A1
:10C680006F03807C49F0C90137FD03969C01359505
:10C690002795359527950DC08091110980FF09C018
:10C6A000C90137FD07969C01A3E035952795AA950A
:10C6B000E1F7820E931E20917301222309F454C0E6
:10C6C0006091C1037091C2038091C3039091C40330
:10C6D00097FF04C061587F4F8F4F9F4FF7E09595AC
:10C6E000879577956795FA95D1F73327442755278E
:10C6F0000E94AC9897FF04C0615E7F4F8F4F9F4FA1
:10C70000E5E09595879577956795EA95D1F76093DC
:10C710003704709338048093390490933A04613855
:10C72000AFEF7A07AFEF8A07AFEF9A072CF480E8F4
:10C730009FEFAFEFBFEF0AC06F3F71058105910515
:10C7400069F064F080E091E0A0E0B0E0809337040D
:10C7500090933804A0933904B0933A04809137043D
:10C7600090913804880E991E80917101282F3327EB
:10C770008091C109992787FD9095289FF001299FF5
:10C78000F00D389FF00D11249F01F7FF02C02158D2
:10C790003F4F220F232F221F330BFFEF21383F077C
:10C7A0001CF420E83FEF06C02F3F310519F014F0CC
:10C7B00020E031E0820E931EC401AA2797FDA095C8
:10C7C000BA2F00918B0310918C039801442737FDF9
:10C7D0004095542FBC01CD010E94AC9897FF04C036
:10C7E00061507E4F8F4F9F4F59E095958795779574
:10C7F00067955A95D1F7E61AF70A80919B039091B5
:10C800009C03892B09F064C0101611060CF060C05F
:10C810002091690430916A04C90137FF03C0309543
:10C8200021953F4F2D33310540F48091B90390910C
:10C83000BA038E159F0574F526C02C53304045E091
:10C84000369527954A95E1F72031310510F02FE014
:10C8500030E04091B9035091BA0318161906E4F478
:10C8600080E190E0821B930B489F9001499F300D1F
:10C87000589F300D1124B4E036952795BA95E1F70D
:10C880002E153F0520F580917A0190917B01E816E5
:10C89000F906F4F07C011CC0205F3F4F80917A01C3
:10C8A00090917B01829FB001839F700D929F700DCC
:10C8B00011249B01A4E036952795AA95E1F74E1522
:10C8C0005F0514F07A0104C0E216F30608F079015E
:10C8D000C701AA2797FDA095BA2FFDE0880F991FE1
:10C8E000AA1FBB1FFA95D1F72091FE083091FF08CF
:10C8F000442737FD4095542FBC01CD010E9420995B
:10C9000020933B0430933C0440933D0450933E04F9
:10C91000E0903B04F0903C0480916B0490916C0497
:10C920009C01220F331F280F391F2E0D3F1D37FF8B
:10C9300002C02D5F3F4FA9015595479555954795E5
:10C9400050936C0440936B0480914C07282F33273D
:10C95000220F331F220F331F241735076CF48091E9
:10C960003509282F3327220F331F220F331F20555D
:10C9700030404217530724F030936C0420936B042B
:10C980008091110980FF14C080916B0490916C0418
:10C99000A981BA818A179B0724F0B0936C04A093F5
:10C9A0006B04E0916B04F0916C04FA83E98326C276
:10C9B00029813A81201B310B37FF02C02D5F3F4F89
:10C9C0003595279535952795E0906B04F0906C048C
:10C9D000E20EF31EC1C1672B49F0E0908B03F0908B
:10C9E0008C0310926A041092690438C18091190373
:10C9F00090911A03A0911B03B0911C03821B930B0F
:10CA0000A40BB50B8093370490933804A09339049A
:10CA1000B0933A04823000E890070FEFA0070FEFC1
:10CA2000B0072CF481E090E8AFEFBFEF09C08F5F53
:10CA30009F47A040B04064F08FEF9FE7A0E0B0E0D8
:10CA40008093370490933804A0933904B0933A0448
:10CA5000809137049091380490936A04809369041C
:10CA600080917401282F332744275527809137045C
:10CA700090913804A0913904B0913A04BC01CD01E1
:10CA80000E94AC9897FF04C0615E7F4F8F4F9F4F0D
:10CA900005E095958795779567950A95D1F7609309
:10CAA0003704709338048093390490933A046530C6
:10CAB00028EF72072FEF82072FEF92072CF484E004
:10CAC00098EFAFEFBFEF09C06050784080409040D2
:10CAD00064F080E098E0A0E0B0E0809337049093A9
:10CAE0003804A0933904B0933A04809037049090AE
:10CAF000380480917301282F332780912603909169
:10CB00002703829FA001839F500D929F500D1124F7
:10CB10009A0157FF02C021503F4F232F330F330B91
:10CB200080911F0390912003820F931FAA2797FDE6
:10CB3000A095BA2F8093370490933804A0933904BA
:10CB4000B0933A048091950320919B0330919C030C
:10CB5000882331F0B3E0220F331FBA95E1F71BC0F1
:10CB6000809150079927289FB001299F700D389F09
:10CB7000700D11249B01A3E0220F331FAA95E1F74A
:10CB8000260F371F37FF02C0215E3F4FF5E0359576
:10CB90002795FA95E1F73093690320936803809114
:10CBA0006803909169039C01442737FD4095542FF9
:10CBB0008091370490913804A0913904B0913A04DF
:10CBC000821B930BA40BB50B80933704909338040E
:10CBD000A0933904B0933A04209176013327442777
:10CBE0005527BC01CD010E94AC9897FF04C0615E3F
:10CBF0007F4F8F4F9F4FE5E0959587957795679588
:10CC0000EA95D1F760933704709338048093390420
:10CC100090933A046530A8EF7A07AFEF8A07AFEF39
:10CC20009A072CF484E098EFAFEFBFEF09C0605093
:10CC300078408040904064F080E098E0A0E0B0E070
:10CC40008093370490933804A0933904B0933A0446
:10CC50008091370490913804880E991EE818F908DD
:10CC60008091B9039091BA038E159F053CF4809191
:10CC70007A0190917B01E816F9060CF07C01C7015E
:10CC8000AA2797FDA095BA2F5DE0880F991FAA1FCC
:10CC9000BB1F5A95D1F72091FE083091FF08442719
:10CCA00037FD4095542FBC01CD010E94209920935F
:10CCB0003B0430933C0440933D0450933E04E09089
:10CCC0003B04F0903C0480916B0490916C049C01B7
:10CCD000220F331F280F391F2E0D3F1D37FF02C0B3
:10CCE0002D5F3F4FA9015595479555954795509311
:10CCF0006C0440936B0480914C07282F3327220F3C
:10CD0000331F220F331F241735076CF48091350928
:10CD1000282F3327220F331F220F331F2055304077
:10CD20004217530724F030936C0420936B048091D6
:10CD3000110920916B0430916C0480FF10C0E981CF
:10CD4000FA812E173F0724F0F0936C04E0936B04F4
:10CD5000E0906B04F0906C04FA82E9824FC03A8351
:10CD600029834CC080915407882301F560918B037F
:10CD700070918C0377FF02C06D5F7F4F759567954B
:10CD80007595679540911F01509120018091000198
:10CD9000282F3327649FC001659F900D749F900DCD
:10CDA0001124B9010E94EB98CB0101C099279093FF
:10CDB0007D0180937C0180917C0190917D0187347D
:10CDC00091051CF486E490E005C08639910534F0A5
:10CDD00086E990E090937D0180937C0109811A811E
:10CDE00010936C0400936B0480916F03806C8093AC
:10CDF0006F0380916E038D7F80936E0380916F032C
:10CE000099279C012270307081FF39C180916D0497
:10CE100090916E04A0916F04B09170040097A105E9
:10CE2000B10521F08091A5038130B9F480918B0385
:10CE300090918C03AA2797FDA095BA2F1EE0880F2A
:10CE4000991FAA1FBB1F1A95D1F780936D04909369
:10CE50006E04A0936F04B09370048091A503813099
:10CE600019F482E08093A50329813A817901002792
:10CE7000F7FC0095102F8091FE089091FF089C010F
:10CE8000442737FD4095542FC801B7010E94AC9844
:10CE9000DC01CB0180933B0490933C04A0933D04C0
:10CEA000B0933E04B7FF04C08150904EAF4FBF4FC8
:10CEB0007C018D01ADE015950795F794E794AA954F
:10CEC000D1F7E0923B04F0923C0400933D041093B0
:10CED0003E0460917003709171033FE0603A730704
:10CEE00050F580916D0490916E04A0916F04B09103
:10CEF00070049C01AD01FAE056954795379527954A
:10CF0000FA95D1F7821B930BA40BB50BA8019701DF
:10CF1000E4E0220F331F441F551FEA95D1F7820F1B
:10CF2000931FA41FB51F80936D0490936E04A0936C
:10CF30006F04B093700460547F4118F580916D04C4
:10CF400090916E04A0916F04B09170049C01AD01AA
:10CF50006CE056954795379527956A95D1F7821BD2
:10CF6000930BA40BB50BA8019701F2E0220F331F1E
:10CF7000441F551FFA95D1F7820F931FA41FB51FA9
:10CF800041C080911F039091200380911F039091D5
:10CF9000200397FF03C0909581959F4F843691059C
:10CFA000CCF58091190390911A03A0911B03B091C5
:10CFB0001C039C0180919D0390919E03281B390BBB
:10CFC00037FF03C0309521953F4F2F3F310509F0C2
:10CFD0000CF580916D0490916E04A0916F04B09156
:10CFE00070049C01AD01EEE0569547953795279565
:10CFF000EA95D1F7821B930BA40BB50B8E0D9F1DE9
:10D00000A01FB11F80936D0490936E04A0936F04D2
:10D01000B093700480916D0490916E04A0916F04A0
:10D02000B09170047EE0B695A795979587957A950F
:10D03000D1F790938C0380938B0340915207442344
:10D0400099F055279C01BA010E94EB98C901861BF3
:10D05000970B9093BA038093B903260F371F309331
:10D060007B0120937A011FC01092BA031092B9037A
:10D070008FEF93E090937B0180937A0114C010921C
:10D08000A50310926D0410926E0410926F0410921A
:10D09000700430938C0320938B0305C080916F0341
:10D0A000806C80936F038091810481FF37C08981F8
:10D0B0009A8197FD039695958795959587952091EB
:10D0C0006C0330916D032817390760F480918B034E
:10D0D00090918C03892B31F0220F331F220F331FC5
:10D0E0003A8329838091190390911A03A0911B031D
:10D0F000B0911C0380939D0390939E03A0939F0384
:10D10000B093A00388E99AE390930D0380930C03F6
:10D1100080E09EE090930A01809309012091F80835
:10D12000822F9927880F991F880F991F88966981E8
:10D130007A818617970714F09A838983709135094D
:10D140007D8B872F9927880F991F880F991F8055EE
:10D150009040A981BA818A179B0714F49A83898326
:10D1600080915703882341F48091C8098F3F21F4AF
:10D17000809185048823E9F0809170039091710378
:10D180000297C097B0F4E981FA811E161F068CF44D
:10D1900081E090E09093710380937003E22EFF246E
:10D1A000EE0CFF1CEE0CFF1C8701085D1F4F1A835D
:10D1B000098329813A813093A8062093A70680919C
:10D1C000330490913404A0913504B091360412E0F8
:10D1D000880F991FAA1FBB1F1A95D1F70091360916
:10D1E00010913709081B190B213A31058CF0C90140
:10D1F00037FD019695958795801791070CF48C0162
:10D20000909581959F4F081719076CF48C010BC0FE
:10D210000135110514F000E510E03FEF003B130766
:10D2200014F400EB1FEF4D89242F3327220F331FF7
:10D23000220F331FC90169817A81861B970B8017E2
:10D2400091070CF48C0189819A81821B930B08173A
:10D2500019070CF48C018091F3089091F408609107
:10D26000B7037091B803861B970B909304098093C2
:10D270000309D09013092091C9033091CA0340914A
:10D28000CB035091CC03DD2041F0661A770AC3012D
:10D29000AA2797FDA095BA2F04C0AA2797FDA095AD
:10D2A000BA2F280F391F4A1F5B1F2093C9033093E1
:10D2B000CA034093CB035093CC038091C903909150
:10D2C000CA03A091CB03B091CC0381509A4FA040E8
:10D2D000B04064F080E09AEFA0E0B0E08093C90332
:10D2E0009093CA03A093CB03B093CC038091C9035E
:10D2F0009091CA03A091CB03B091CC03805096408B
:10D30000AF4FBF4F64F480E096E0AFEFBFEF809384
:10D31000C9039093CA03A093CB03B093CC03C090EE
:10D320006107209103093091040978E0E72EEC149D
:10D3300098F08C2D9927829FA001839F500D929F7A
:10D34000500D1124CA0157FD07967C0163E0F59446
:10D35000E7946A95E1F712C08C2D86959927829FF4
:10D36000B001839F700D929F700D1124CB0177FD4A
:10D3700003967C01F594E794F594E794A0907701E7
:10D38000B09078019501442737FD4095542F809146
:10D39000C9039091CA03A091CB03B091CC03BC0107
:10D3A000CD010E942099E20EF31E90906101692D3B
:10D3B000772788279927980117FF04C0222733274A
:10D3C000201B310B37FF02C02F5F3F4F359527954C
:10D3D000A981BA812A0F3B1F442737FD4095542F5E
:10D3E0000E94AC9897FF04C0615C7F4F8F4F9F4FA6
:10D3F00026E095958795779567952A95D1F79B01B6
:10D400006E157F050CF47B01309521953F4FE21698
:10D41000F3060CF479018091E3089091E40860919F
:10D42000B5037091B603861B970B9093E208809327
:10D43000E1082091C5033091C6034091C703509184
:10D44000C803DD2041F0461A570AC201AA2797FDFA
:10D45000A095BA2F04C0AA2797FDA095BA2F280F30
:10D46000391F4A1F5B1F2093C5033093C6034093A7
:10D47000C7035093C8038091C5039091C603A09140
:10D48000C703B091C80381509A4FA040B04064F0E8
:10D4900080E09AEFA0E0B0E08093C5039093C603CC
:10D4A000A093C703B093C8038091C5039091C603AE
:10D4B000A091C703B091C80380509640AF4FBF4FB3
:10D4C00064F480E096E0AFEFBFEF8093C5039093E4
:10D4D000C603A093C703B093C8032091E10830911D
:10D4E000E20848E04C1598F08C2D9927829FB001F6
:10D4F000839F700D929F700D1124CB0177FD0796CD
:10D500006C01B3E0D594C794BA95E1F712C0C69404
:10D510008C2D9927829FD001839FB00D929FB00DD3
:10D520001124CD01B7FD03966C01D594C794D59411
:10D53000C7949501442737FD4095542F8091C5032A
:10D540009091C603A091C703B091C803BC01CD015F
:10D550000E942099C20ED31E692D7727882799270C
:10D56000980117FF04C022273327201B310B37FFF8
:10D5700002C02F5F3F4F35952795E981FA812E0F25
:10D580003F1F442737FD4095542F0E94AC9897FFCA
:10D5900004C0615C7F4F8F4F9F4FE6E09595879564
:10D5A00077956795EA95D1F79B016C157D050CF48D
:10D5B0006B01309521953F4FC216D3060CF46901DB
:10D5C0008091F808282E33245090A30761E1862E1D
:10D5D00068E0962E58ECA52E57E0B52E4BE0442E71
:10D5E00034E1632E39E0732ED5012C9112160CF024
:10D5F00029C1203429F4E981FA81FF8BEE8B1FC009
:10D6000049815A81CA01AA2797FDA095BA2F3327CD
:10D6100027FD3095432F532FBC01CD010E94AC98BC
:10D6200097FF04C0615C7F4F8F4F9F4F26E0959519
:10D630008795779567952A95D1F77F8B6E8BF50146
:10D640002181203439F42E893F892E0D3F1D3F8BD7
:10D650002E8B2AC0203C39F44E895F894E195F0910
:10D660005F8B4E8B21C0C701AA2797FDA095BA2FCB
:10D67000332727FD3095432F532FBC01CD010E9446
:10D68000AC9897FF04C0615C7F4F8F4F9F4FB6E00F
:10D690009595879577956795BA95D1F7AE89BF89A6
:10D6A000A60FB71FBF8BAE8BF5012281203439F452
:10D6B0002E893F892C0D3D1D3F8B2E8B2AC0203C8F
:10D6C00039F44E895F894C195D095F8B4E8B21C0FF
:10D6D000C601AA2797FDA095BA2F332727FD3095BD
:10D6E000432F532FBC01CD010E94AC9897FF04C07B
:10D6F000615C7F4F8F4F9F4FA6E0959587957795FB
:10D700006795AA95D1F7AE89BF89A60FB71FBF8BC2
:10D71000AE8BF5012381203439F42E893F89200F07
:10D72000311F3F8B2E8B2AC0203C39F44E895F89F4
:10D73000401B510B5F8B4E8B21C0C801AA2797FD60
:10D74000A095BA2F332727FD3095432F532FBC01C7
:10D75000CD010E94AC9897FF04C0615C7F4F8F4F52
:10D760009F4FF6E09595879577956795FA95D1F750
:10D77000AE89BF89A60FB71FBF8BAE8BF301808127
:10D7800091812E893F898217930764F4B901680F4C
:10D79000791F77FF02C06F5F7F4F759567957F8B0D
:10D7A0006E8B1DC0552049F44E895F89440F551F6B
:10D7B000481B590B5F8B4E8B12C051E0551578F406
:10D7C000252D33276E897F89861B970BB9010E940F
:10D7D000EB98AE89BF89A60FB71FBF8BAE8BC10177
:10D7E000880F991F880F991FEE89FF898E179F0751
:10D7F00064F4FD898F2F9927880F991F880F991F2F
:10D800002E893F892817390714F09F8B8E8B8E89BC
:10D810009F8997FD03969595879595958795F40132
:10D820008183880F991F880F991F2E893F89281B94
:10D83000390BC901880F8283EE89FF89D301ED93EB
:10D84000FC9303C0F401118212824A9422E030E07A
:10D85000620E731E44E050E0A40EB51E68E070E056
:10D86000860E971E47FEC0CEE2E1C95E0C94579922
:10D8700084B1806A84B93D9A82E58CBD1DBC459A0D
:10D8800081E0809347098AEA8093580983E880936E
:10D8900059098AE080935A0910925C0910925B0939
:10D8A00010925E0910925D091092C00910927C09D5
:10D8B000089530914709332309F085C00DB407FE60
:10D8C00082C084E080930B03459A2EB58091880432
:10D8D00099278130910589F0823091051CF4892BBC
:10D8E00021F03EC00297B9F03BC030937B092093F2
:10D8F00089042138A9F581E008C0253549F48091D3
:10D900008904820F8093890482E08093880428C070
:10D910003093880425C080917B09E82FFF27E356C8
:10D92000F64F20838F5F80937B099091890480322A
:10D93000A0F0291769F480E2ADE9B9E0EDE7F9E07C
:10D940000D9001928A95E1F781E080937C0902C0F5
:10D9500030937C091092880403C0920F909389043D
:10D9600020915709223208F028C045980000000095
:10D9700000000000000000000000000000000000A7
:10D980000000000000000000000000000000000097
:10D99000000000000000000000000000E0915009BD
:10D9A000F0915109E20FF11D80818EBD80917909BE
:10D9B0009081890F8093790903C081E080934709A2
:10D9C0002F5F209357090895EF92FF920F931F93B3
:10D9D00080915A079927880F991F880F991F7C01FA
:10D9E0000027F7FC0095102F80910104909102040C
:10D9F000A0910304B0910404BC01CD01A8019701DA
:10DA00000E94209930935C0920935B098091F9036F
:10DA10009091FA03A091FB03B091FC03BC01CD01EE
:10DA2000A80197010E94209930935E0920935D0917
:10DA300020913D0930913E0940913F0950914009A4
:10DA4000DA01C90163E0880F991FAA1FBB1F6A95FD
:10DA5000D1F7820F931FA41FB51F820F931FA41F1E
:10DA6000B51F20913C0130913D0140913E01509104
:10DA70003F01BC01CD010E9420993093640920939D
:10DA80006309809113049091140420912C03309128
:10DA90002D03821B930B90936A0980936909E0918F
:10DAA0000904F0910A0480910A0990910B09BF01C1
:10DAB0000E94EB989B01220F331F220F331F260F6A
:10DAC000371F260F371F37FF02C02D5F3F4F359599
:10DAD0002795359527953093600920935F098091AC
:10DAE000390990913A09BF010E94EB989B01220FDE
:10DAF000331F220F331F260F371F260F371F37FF05
:10DB000002C02D5F3F4F359527953595279530936A
:10DB100062092093610910920A041092090410927C
:10DB20000B0910920A0910923A0910923909809152
:10DB30005A099927AA27BB27FC013A97E830F10533
:10DB400008F0FEC1E058FF4F0C9472998091840355
:10DB500080936D098091830380936E098091820385
:10DB600080936F0980918103809370098091800375
:10DB70008093710980917F038093720980917E0365
:10DB80008093730980917D038093740980916F0362
:10DB90008093750980916F03837F80936F030E9448
:10DBA0006E32809376098091A407809377098091E3
:10DBB0006E03C4C18091C2099091C30990936E090C
:10DBC00080936D098091C6099091C709909370095F
:10DBD00080936F0980911F019091200180937109BA
:10DBE000809100018093720980913B0180937309B9
:10DBF00090918A0490937409E92FFF27A3E0EE0F18
:10DC0000FF1FAA95E1F7EF5EF74F868180937509B4
:10DC100083818093760987818093770985818093BA
:10DC20007809892F8F5F6CE00E94CB9890938A04CB
:10DC300087C180918F0780936D09809190078093B1
:10DC40006E098091910780936F098091920780936C
:10DC50007009809193078093710980919707809351
:10DC60007209809198078093730980919907809336
:10DC7000740980919C078093750980919A0780931D
:10DC8000760980919B078093770980919D0756C103
:10DC900080918E0780936D0980916507863081F0B1
:10DCA0008091D802823451F00E946E79E82FFF27CC
:10DCB000EF53FE4E84918093D80202C00E946E7989
:10DCC0008091AF0480936E093BC1F8948091410725
:10DCD000E82FFF27EE0FFF1FEE58F74F0190F0815E
:10DCE000E02DE038F1051CF0EFE7F0E006C02FEF83
:10DCF000E138F20714F4E1E8FFEFE0936D09809159
:10DD00004207E82FFF27EE0FFF1FEE58F74F019055
:10DD1000F081E02DE038F1051CF0EFE7F0E006C0FF
:10DD20007FEFE138F70714F4E1E8FFEFE0936E09C5
:10DD300080914007E82FFF27EE0FFF1FEE58F74FA7
:10DD40000190F081E02DE038F1051CF0EFE7F0E004
:10DD500006C08FEFE138F80714F4E1E8FFEFE09335
:10DD60006F0980913F07E82FFF27EE0FFF1FEE5846
:10DD7000F74F0190F081E02DE038F1051CF0EFE75E
:10DD8000F0E006C02FEFE138F20714F4E1E8FFEF0E
:10DD90007894E09370098091A80380937109809131
:10DDA000A903809372098091AA03809373098091DB
:10DDB000AB03809374098091AC03809375098091C3
:10DDC000AD03809376098091AE03809377098091AB
:10DDD000AF03B4C080912805863018F01092280552
:10DDE00085E080936D0980919E0780936E098091F4
:10DDF000A1039091A203A091A303B091A403BC013D
:10DE0000CD0125E030E040E050E00E9420993093C1
:10DE1000700920936F0980919D0390919E03A091BA
:10DE20009F03B091A003BC01CD0125E030E040E0AC
:10DE300050E00E94209930937209209371098091DB
:10DE4000940780937309809195078093740980915A
:10DE50009607809375098091A70380937609809136
:10DE6000720890917308809377098091A70690912A
:10DE7000A80697FD039695958795959587955EC01D
:10DE800010926D098AE580936E0986E080936F0990
:10DE900085E38093700980910101809371098091DD
:10DEA0000D058093720990910E05909373098F77F9
:10DEB00080930D05907190930E0580910F058093CE
:10DEC000740980912D0980937509809111098093BF
:10DED00076098091A007809377098091AD072EC0C5
:10DEE0008091730780936D098091AB0780936E09D1
:10DEF0008091690180936F0980916C07809370090C
:10DF000080916D078093710980916E0780937209EB
:10DF100080916801809373098091700780937409E0
:10DF200080917107809375098091720780937609BB
:10DF30008091C809809377098091D10680937809F0
:10DF400080917C09882309F47DC160917D098091CD
:10DF50009B01681719F08AEF8093990160939B01E8
:10DF600081E08093890140917E0950917F09CA0127
:10DF700081509E4F8F5F9340B0F420918009309183
:10DF80008109C90181509E4F8F5F934060F4809159
:10DF90004B0785FF08C05093770440937604309375
:10DFA000750420937404809184099091850921E07F
:10DFB0008936920724F490938B0180938A012091F3
:10DFC0008E0930918F0980910C0390910D03821777
:10DFD000930740F48091E002882321F430930D03ED
:10DFE00020930C03862F99278936910509F4A5C043
:10DFF0008A36910544F48736910571F0883691058B
:10E0000009F462C027C18A36910509F414C18B3620
:10E01000910509F4E2C01EC1809190098093BD0969
:10E02000809191098093BF09809192098093BE09E4
:10E030008091930980938801809194098093C1090C
:10E040008091950980939A01809196098093870425
:10E05000809197098093730480917C038823F9F061
:10E06000209198093091990937FD19C03093C00368
:10E070002093BF0390917507992389F08FE0989FB3
:10E08000C0011124281B390BC90188599E4F68E62D
:10E0900071E00E94EB989093C0038093BF0320919E
:10E0A0007E0430917F0480919A0990919B09280FFA
:10E0B000391F37FF02C02F5F3F4F359527953093AB
:10E0C0007F0420937E04C6C08091900980935209FA
:10E0D000809191098093530980919209809354090A
:10E0E00080919309809355098091940980935609F2
:10E0F0008091970690919509892B8093970690912E
:10E1000098069370809196098C70982B909398063E
:10E1100080919709809385048091980980938D015F
:10E12000809199098093C00980919A098093810414
:10E1300080919B09809380048DC080919009809389
:10E1400048098091910980934909809192098093AF
:10E150004A098091930980934B0980919409909189
:10E16000950990934D0980934C098091960990915F
:10E17000970990934F0980934E09809198099927A8
:10E1800087FD90959093A5088093A40880919909A4
:10E190008093960380919A0990919B099C01442752
:10E1A00037FD4095542FDA01C90163E0880F991FAC
:10E1B000AA1FBB1F6A95D1F7820F931FA41FB51F1B
:10E1C000820F931FA41FB51F80939703909398030A
:10E1D000A0939903B0939A033DC0809190098093D6
:10E1E00084048091910980938304809192098093A3
:10E1F000820490919309992349F08091A101882389
:10E2000019F08151833010F49093A1018091940909
:10E210008093B404809195098093B304809196090A
:10E22000909197099093B1048093B00480919809DC
:10E230008093B2040FC080916507863059F40E9424
:10E24000C77908C010927704109276041092750472
:10E25000109274041F910F91FF90EF900895809198
:10E260004709882309F43BC0459888E599E09093D5
:10E2700051098093500990918604E92FFF27E257B6
:10E28000FE4F9F5F90938604808180935A099B3054
:10E2900010F010928604109247090E94E46C81E00D
:10E2A00080935709000000000000000000000000FB
:10E2B000000000000000000000000000000000005E
:10E2C000000000000000000000000000000000004E
:10E2D0000000000080915809809379098EBD08954F
:10E2E00087B18C6087B94298439810928C0480E87B
:10E2F00080939D0110928B0480939C0108958091DE
:10E3000091048150809391048F3F09F055C189E0B9
:10E31000809391048091A4089091A50881589F4F03
:10E3200039F08091A4089091A508815880939604B3
:10E3300080916F03992780739070892B21F48091CD
:10E340000E0580FF1DC080918C07882351F08091BD
:10E350009404882319F484E080938C0481E08093F2
:10E36000940480918D078823B9F0809195048823C7
:10E3700019F484E080938B0481E0809395040CC0B1
:10E3800010929404109295048091880780939204CF
:10E3900080918A078093930480919404882309F0E4
:10E3A00073C08091AA07282F332724FF07C08091CC
:10E3B000A603882319F425FD80C081C090918907A8
:10E3C000983F48F080910C098D3D28F0809192048F
:10E3D00088236CF00AC0983F68F080910C09853062
:10E3E00049F48091920487FF02C0429801C0429A8A
:10E3F00081E032C080918C04815080938C048F3FE7
:10E4000009F05EC08091AD0785FF29C09091960408
:10E41000892F869580938C04992351F480919204DE
:10E4200087FF02C0429801C0429A10929D0148C0E5
:10E4300080919D0190919204882341F480939604E9
:10E4400080E880939D019923D4F137C0982311F07F
:10E45000429A01C04298869580939D0131C0809177
:10E460000C09869580938C0480919D01813021F464
:10E470001092960480E801C0869580939D0180915A
:10E480009D019091920417C080918C0481508093DB
:10E490008C048F3FA9F489E080938C0480919D01C6
:10E4A000813011F480E801C0869580939D018091B0
:10E4B0009D0190918C07892311F0429A01C04298E6
:10E4C00080919504882309F043C09091AA0797FF93
:10E4D00007C08091A603882319F496FD52C053C04B
:10E4E00090918B07983F48F0809134098D3D28F03A
:10E4F0008091930488236CF00AC0983F78F0809153
:10E500003409853059F48091930487FF02C0439801
:10E5100001C0439A81E080939C0136C080918B04B6
:10E52000815080938B048F3F79F5809134098695D3
:10E5300080938B0480919C01813011F480E801C0AC
:10E54000869580939C0180919C019091930417C0C3
:10E5500080918B04815080938B048F3FA9F489E0D4
:10E5600080938B0480919C01813011F480E801C07C
:10E57000869580939C0180919C0190918D078923C1
:10E5800011F0439A01C04398429B04C080916E03EE
:10E59000886003C080916E03877F80936E03439BE6
:10E5A00006C080916E03806180936E030895809110
:10E5B0006E038F7E80936E0308954FB724E130E0A1
:10E5C000F8948091C9008F778093C9008091C90029
:10E5D0008F7B8093C9008091C9008F7D8093C90093
:10E5E000832F99278093CD002093CC008091C80081
:10E5F00082608093C80080E18093C9008091CA0046
:10E600008F778093CA008091CA008F7B8093CA0065
:10E610008091CA008F7D8093CA008091CA008F7E4E
:10E620008093CA008091CA00877F8093CA0080913E
:10E63000C9008B7F8093C9008091CA008460809359
:10E64000CA008091CA0082608093CA008091C8008D
:10E6500087FF03C08091CE00F9CF8091C900806808
:10E660008093C9004FBF0895EF92FF920F931F93BD
:10E67000CF93DF93482F00E010E080919E0181301E
:10E6800061F410929E0184E480939704109299049F
:10E690001092980410929A0439C1809197048823AB
:10E6A00019F421E030E001C0980190919804992379
:10E6B00071F4232B11F081E010C084E4809397045F
:10E6C000909399049093980490939A0408C1913080
:10E6D00069F4232B09F0F9C082E0809398048091BB
:10E6E00099048F5F8093990483E0F7C09230D1F44E
:10E6F000232B09F0EAC083E08093970440939A04A7
:10E7000090919904923039F410929B0447FF03C012
:10E7100081E080939B0483E0809398049F5F9093B3
:10E720009904DDC0933009F0D0C0232B09F0CDC08F
:10E730009093970482E080939804809199048F5F6E
:10E740008093990420919A04822F9927782F662725
:10E75000842F9927682B792B80916507813049F4A4
:10E760007370CB018050924063E070E00E94EB98A0
:10E7700017C0823061F47770CB018050944066E01E
:10E7800070E00E94EB982695269526950BC0737035
:10E7900068567140CB0177FD0196BC017595679570
:10E7A00026952695022F11270F7010700F5F1F4FAF
:10E7B0000D30110508F082C07801E00EF11EF7015E
:10E7C000EE58F74F808191819B01281B390BC901BD
:10E7D00037FF03C0909581959F4F069704F5E09110
:10E7E000A707EE2351F0FF27EE0FFF1FEE58F74F5C
:10E7F000808191818436910594F48091A703883CAF
:10E8000030F48091A703865F8093A70308C088EC4B
:10E810008093A70380916F008F7D80936F00F70135
:10E82000EE58F74F808191819C01220F331F280FF2
:10E83000391F260F371F37FF02C02D5F3F4FE901F9
:10E84000D595C795D595C795CB0101968C179D0792
:10E8500014F4219706C061507040C617D7070CF416
:10E8600021968091A703843BD0F0F701EE58F74F33
:10E8700080819181FE01E81BF90BCF0163E070E01C
:10E880000E94EB98CB01880F991F860F971F26EAED
:10E8900038E0E20EF31EF7019183808307C026EA79
:10E8A00038E0E20EF31EF70111821082000F111FF3
:10E8B0000E58174FF801D183C08311C002311105E2
:10E8C00070F081E080939E010AC081E080939E01F8
:10E8D0001092990410929B0484E480939704809191
:10E8E0009904803198F080919B04882331F48091C1
:10E8F0009E01882311F480933A011092990410929A
:10E900009B041092980484E480939704E6E0CDB7CA
:10E91000DEB70C946399CF93FC0197FF05C0CFEF4E
:10E92000F095E195FF4F01C0C1E028E631E0CF014D
:10E93000B9010E94EB98FC018B35910554F08B5581
:10E9400090408A35910538F484EB90E08E1B9F0B44
:10E95000FC0141E00DC0CF01855B90408A359105F7
:10E9600018F4E45BF04003C02E1B3F0BF9014FEF9E
:10E97000EE0FFF1FE45BF64F259134918C2F992702
:10E9800087FD9095289FB001299F700D389F700DCD
:10E990001124842F992787FD9095689FA001699F76
:10E9A000500D789F500D1124CA01CF9108952AE58A
:10E9B00030E0281B390BC9010E948B740895CF9356
:10E9C000DF9380E00E948C8B80911F019091200149
:10E9D0006AE070E00E94EB989F938F9380911F01F3
:10E9E000909120016AE070E00E94EB987F936F9312
:10E9F00080E29AE09F938F93CFE7DBE8DF93CF939A
:10EA0000E091F404F091F50409952DB73EB7285F25
:10EA10003F4F2DBF80919901882361F186E00E94CC
:10EA20008C8B80918D0199279F938F9380914C09B6
:10EA300090914D096AE070E00E94D7987F936F93A0
:10EA40008FED90E09F938F938091E8089091E90873
:10EA50009F938F9389E29AE09F938F93DF93CF9355
:10EA6000E091F404F091F50409958DB79EB70C96EA
:10EA70008DBF12C086E00E948C8B87E39AE09F9343
:10EA80008F93DF93CF93E091F404F091F50409950F
:10EA90000F900F900F900F9080918504882309F4B8
:10EAA00058C080919C0490919D040E94351A88233F
:10EAB00091F080919F01882319F010929F0103C06B
:10EAC00081E080939F018CED95E00E942C1A909339
:10EAD0009D0480939C0480919F018823E1F080E055
:10EAE0000E948C8B1F921F929091850481E1989FC8
:10EAF000C0011124865A944F9F938F93DF93CF9335
:10EB0000E091F404F091F50409952DB73EB72A5F22
:10EB10003F4F2DBF1EC086E00E948C8B80918504E4
:10EB200099279F938F938EE39AE09F938F93DF9320
:10EB3000CF93E091F404F091F50409958DB79EB759
:10EB400006968DBF8091A603882319F08FE48093E9
:10EB5000D80280E10E948C8B8091DA029091DB02D6
:10EB60006CE370E00E94D7989F938F938091DA02B4
:10EB70009091DB026CE370E00E94D7987F936F93D3
:10EB80008091C6099091C7099F938F938AE49AE078
:10EB90009F938F93CFE7DBE8DF93CF93E091F4046B
:10EBA000F091F504099580912D092DB73EB7265FA8
:10EBB0003F4F2DBF80FF29C08AE10E948C8B80913E
:10EBC0003B0199279F938F938091A1039091A2037A
:10EBD000A091A303B091A403BC01CD0124E630E0D1
:10EBE00040E050E00E9420993F932F9387E59AE000
:10EBF0009F938F93DF93CF93E091F404F091F5040A
:10EC000009958DB79EB708968DBFDF91CF91089576
:10EC1000CF93DF9380E00E948C8B809130089927FE
:10EC200087FD90959F938F9380912808992787FD62
:10EC300090959F938F9380912008992787FD9095B9
:10EC40009F938F9380911808992787FD90959F93A4
:10EC50008F938EE59AE09F938F93CFE7DBE8DF9366
:10EC6000CF93E091F404F091F504099580E10E94BE
:10EC70008C8B2DB73EB7245F3F4F2DBF809150083E
:10EC8000992787FD90959F938F93809148089927A6
:10EC900087FD90959F938F9380914008992787FDDA
:10ECA00090959F938F9380913808992787FD909531
:10ECB0009F938F938EE69AE09F938F93DF93CF93EA
:10ECC000E091F404F091F504099580913D072DB78A
:10ECD0003EB7245F3F4F2DBF853098F480E10E94FE
:10ECE0008C8B8EE79AE09F938F93DF93CF93E09185
:10ECF000F404F091F50409950F900F900F900F9088
:10ED000018C08730B0F488E10E948C8B8FED90E0C2
:10ED10009F938F938FE89AE09F938F93DF93CF9386
:10ED2000E091F404F091F50409958DB79EB706962D
:10ED30008DBFDF91CF9108950F931F9380E00E94C4
:10ED40008C8B2AE030E08091C2099091C309B9010F
:10ED50000E94D7989F938F938091C2099091C30985
:10ED6000B9010E94D7987F936F9380911F01909172
:10ED70002001B9010E94EB989F938F9380911F010E
:10ED800090912001B9010E94EB987F936F9388E9DD
:10ED90009AE09F938F930FE71BE81F930F93E091E7
:10EDA000F404F091F504099580E10E948C8B8DB7F5
:10EDB0009EB70C968DBF8091C6099091C7099F930D
:10EDC0008F938091C4099091C5099F938F938AEA8C
:10EDD0009AE09F938F931F930F93E091F404F09127
:10EDE000F50409958DB79EB708968DBF1F910F91B9
:10EDF0000895EF92FF920F931F9380E00E948C8BF7
:10EE00008FEDE82EF12CFF92EF9280918A01909184
:10EE10008B019F938F938091840499279F938F9365
:10EE200086EB9AE09F938F930FE71BE81F930F9356
:10EE3000E091F404F091F504099580E10E948C8B37
:10EE40008DB79EB70A968DBF8091820499279F93B4
:10EE50008F93FF92EF928091830499279F938F93D2
:10EE600089EC9AE09F938F931F930F93E091F404A2
:10EE7000F091F50409958DB79EB70A968DBF1F9145
:10EE80000F91FF90EF9008950F931F93CF93DF930F
:10EE900080919901CFE7DBE8882309F47DC080E009
:10EEA0000E948C8B8091490999279F938F93809121
:10EEB0004B0999279F938F938CED9AE09F938F93A3
:10EEC0008E01DF93CF93E091F404F091F50409955E
:10EED0008DB79EB708968DBF80914A09833031F473
:10EEE0008CE00E948C8B8BEE9AE005C08CE00E9437
:10EEF0008C8B80EF9AE09F938F93DF93CF93E09179
:10EF0000F404F091F50409950F900F900F900F9075
:10EF10008091480981FF12C08CE00E948C8B85EFA4
:10EF20009AE09F938F931F930F93E091F404F091D5
:10EF3000F50409950F900F900F900F9080E10E94BB
:10EF40008C8B80918D0199279F938F938FED90E00B
:10EF50009F938F9380914E0990914F099F938F9328
:10EF600080914C0990914D096AE070E00E94D79819
:10EF70007F936F938AEF9AE09F938F938FE79BE83D
:10EF80009F938F93E091F404F091F50409958DB768
:10EF90009EB70C968DBF12C082E00E948C8B8DE0D4
:10EFA0009BE09F938F93DF93CF93E091F404F091D4
:10EFB000F50409950F900F900F900F90DF91CF916E
:10EFC0001F910F910895CF93C82F20919E042093F5
:10EFD0009F0499278F329105E1F0803391051CF44D
:10EFE0004F9779F027C08F349105D9F08F3891056C
:10EFF00009F586E0289FF0011124EE5FF54F84911A
:10F0000017C086E0289FF0011124ED5FF54F849131
:10F010000FC086E0289FF0011124EC5FF54F84912A
:10F0200007C086E0289FF0011124EB5FF54F849123
:10F0300080939E0490919E0480919F049813C0E059
:10F040008091A001282F33278F5F8093A00120FF9C
:10F050000FC00E94928B90919E0486E0989FF001D1
:10F060001124EA5FF54F259134918C2FF901099510
:10F0700080E090E0CF9108951092C3091092C209E8
:10F080001092C7091092C6091092C5091092C409BE
:10F090001092C8098AE090E00E942C1A9093A10473
:10F0A0008093A0040895CF93DF938091A004909162
:10F0B000A1040E94351A882309F4AFC08091A004EE
:10F0C0009091A1040A969093A1048093A004E0E09B
:10F0D000F0E09F0190E05FEFA1E1B8E04BE0ED01CF
:10F0E0008B8187FF0BC09F5F8D81E80FF11D8981A8
:10F0F000280F311D8E81851708F4582F415018961E
:10F1000047FFEDCF5093C809232B41F52091A6046A
:10F110003091A7044091A8045091A904BB27A52FC2
:10F12000942F832F9093A5048093A404AA27BB2730
:10F13000281B390B4A0B5B0BCF01AA27BB27280FD3
:10F14000391F4A1F5B1F2093A6043093A7044093E6
:10F15000A8045093A904E5E0F0E013C02091A404B2
:10F160003091A5042E173F0718F4E21BF30B02C0E1
:10F17000E0E0F0E0892F9927880F991FE80FF91F29
:10F180003596F093C309E093C209EF3FF10578F497
:10F1900080911F01909120018E9F90018F9F300DD3
:10F1A0009E9F300D1124C90164E670E013C0CF01A9
:10F1B000969587959695879520911F01309120010E
:10F1C000289FA001299F500D389F500D1124CA017E
:10F1D00069E170E00E94D7987093C5096093C409F3
:10F1E0002091A2043091A3042E0F3F1F3093A3045B
:10F1F0002093A2045EE02131350778F08091C609A2
:10F200009091C70901969093C7098093C609205130
:10F210003E403093A3042093A204DF91CF91089540
:10F220003091B504E32FFF2783E0EE0FFF1F8A958F
:10F23000E1F7EF5EF74F2781422F552747FD5095A5
:10F240008091B6049927841795072CF42093B6046F
:10F250003093B8040AC0222341F08091B704992763
:10F260004817590714F42093B704832F8F5F8093B6
:10F27000B5048D30D0F01092B5048091B7048F3F63
:10F2800019F08093AB0402C01092AB048091B604D5
:10F290008093AC048091B8048093AA048FEF80938C
:10F2A000B7041092B6041092B804089595E1899FAE
:10F2B000802D11240E94359186EA9DE09F938F93C3
:10F2C00087E091E99F938F93E091F404F091F50426
:10F2D00009950F900F900F900F900895CF93C0E075
:10F2E0002091A1012093AF0480916F0385FF02C09C
:10F2F000C0E123C0909185049923B1F08091A603C9
:10F30000882349F4E92FFF27EE0FFF1FE55EF44F36
:10F310008491882349F4E92FFF27EE0FFF1FE65E53
:10F32000F44FC491CC2349F48091AD0786FD03C00E
:10F330001092A10104C0C22F02C0C093AF048091FB
:10F34000B9048C1771F48091BA049091BB040E94A7
:10F35000351A882319F480E090E017C088E893E11B
:10F3600002C080ED97E00E942C1A9093BB0480931A
:10F37000BA04CC2331F08091A101C81711F4109286
:10F38000A101C093B9048C2F9927CF91089540E033
:10F3900050E030E080919B0999278A38910589F0E7
:10F3A0008B38910524F48938910541F013C08D38CC
:10F3B000910569F08E38910539F00CC041E25AE0B0
:10F3C00008C049EF5AE005C049EC59E002C045EFDA
:10F3D00059E03CE29091900920E080919109281732
:10F3E00070F4931760F4DA01A90FB11DE22FFF2723
:10F3F000E358F64F85898C939F5F2F5FEECF08957A
:10F4000020E335E780913B018B3211F08D32F9F426
:10F4100080915007282F332780919B0390919C0364
:10F42000829FA001839F500D929F500D1124CA010D
:10F4300063E070E00E94EB98CB019B01205D3A48AD
:10F44000C196C19708F03FC02EEF34E73CC0803230
:10F4500029F580916F0381FF36C02091AD04309172
:10F46000AE04205D3A4855E72133350748F085E77B
:10F470002439380718F420E335E702C02456304019
:10F4800045E720333407F8F454E72D3C350718F0EE
:10F4900020E335E718C02C593F4F15C08E3549F48D
:10F4A000909196038AE0989F90011124205D3A483C
:10F4B0000AC0863741F4909196038AE0989FC00174
:10F4C0001124281B390BC9010895EF92FF920F9365
:10F4D0001F9399278A38910509F444C18B38910507
:10F4E00024F48938910551F0DEC28D38910509F474
:10F4F00024C28E38910509F486C1D5C28091A1033A
:10F500009091A203A091A303B091A403BC01CD01EB
:10F5100024E630E040E050E00E942099DA01C90181
:10F520008C509E4F9093270A8093260A0E94007A5F
:10F5300090932D0A80932C0A90932F0A80932E0A81
:10F540009093310A8093300A2091260A3091270A3D
:10F5500080912A0A90912B0A2817390724F43093B6
:10F560002B0A20932A0A8091280A9091290A82174F
:10F57000930724F43093290A2093280A1092230A2F
:10F5800081E29AE09093CC048093CB0480913B017C
:10F590008093470A80916E0380FF02C083E401C01C
:10F5A00080E28093480A20918504222309F1822F6A
:10F5B0006AE00E94CB98805D8093320A822F0E947D
:10F5C000CB98892F805D8093330A8AE38093340A35
:10F5D00081E1289FF0011124A5E3BAE0E65AF44F37
:10F5E0009FE084918D939150319697FFFACF58C246
:10F5F00080916F0385FF0CC0A2E3BAE0EAE7FDE06B
:10F6000094E184918D939150319697FFFACF48C23F
:10F610003091B304332309F499C087E58093320A0B
:10F6200080E58093330A40E24093340A2091B40489
:10F63000822F6AE00E94CB98805D8093350A822FEA
:10F640000E94CB98892F805D8093360A8FE2809349
:10F65000370A832F0E94CB98805D8093380A832FCE
:10F660000E94CB98892F805D8093390A40933A0A93
:10F670002091B0043091B10483E0293E380780F036
:10F68000C90168EE73E00E94D798CB01805D80933A
:10F690003B0AC90168EE73E00E94D7989C0102C042
:10F6A00040933B0A2536310580F0C90164E670E0DD
:10F6B0000E94D798CB01805D80933C0AC90164E623
:10F6C00070E00E94D7989C0103C080E280933C0ABE
:10F6D000C9016AE070E00E94D798CB01805D8093F9
:10F6E0003D0AC9016AE070E00E94D798805D80936E
:10F6F0003E0A8DE680933F0A80E28093400A209183
:10F70000B204253660F0822F64E60E94CB98805DBB
:10F710008093410A822F0E94CB98292F02C08093A8
:10F72000410A822F6AE00E94CB98805D8093420A52
:10F73000822F0E94CB98892F805D8093430A83E7B4
:10F740008093440A80E28093450AAAC1A2E3BAE00A
:10F75000E0E9FDE094E184918D939150319697FF1B
:10F76000FACF9EC18091A1039091A203A091A3031F
:10F77000B091A403BC01CD0124E630E040E050E0AC
:10F780000E942099DA01C9018C509E4F90930F0B73
:10F7900080930E0B0E94007A9093110B8093100BB4
:10F7A00088E78093120B809149098093130B0E9484
:10F7B0006E798093FB0A8091480981FF02C084E43E
:10F7C00007C080914A09833011F480E201C081E2D0
:10F7D0008093140B89EF9AE09093CC048093CB0430
:10F7E00080918D018093200B8091140B8093220BCC
:10F7F00080914E0990914F0997FD019695958795B7
:10F800008093150B4DC10E9410798091A1039091B6
:10F81000A203A091A303B091A403BC01CD0124E6EF
:10F8200030E040E050E00E942099DA01C9018C509C
:10F830009E4F9093E4098093E30980911F0190917A
:10F8400020019093DE098093DD0980911F01909142
:10F8500020019093E0098093DF098091E80890915E
:10F86000E90897FD0196959587958093CF09809338
:10F87000D60920914E0930914F0937FF02C02F5F02
:10F880003F4F359527952093D40980914C0990914D
:10F890004D0964E170E00E94D7986093D5092093E8
:10F8A000DB096093DC090E94007A9093EC09809355
:10F8B000EB0988E78093ED0980911F019091200169
:10F8C0009093E8098093E7098091AB048C5E809364
:10F8D000E1098091AC048C5E8093E2098091C609B5
:10F8E0009091C7096AE070E00E94D7987093EA0986
:10F8F0006093E9091092CB098091C2099091C309E4
:10F900009093E6098093E50989EC99E09093CC0403
:10F910008093CB042091DA023091DB02C9016CE3C1
:10F9200070E00E94D7986093F009C9016CE370E021
:10F930000E94D7988093F109B3C00E9410798091FA
:10F940004C0990914D0964E670E00E94D79870933D
:10F950000B0A60930A0A8091E8089091E90897FDE4
:10F960000196959587958093FB0980914E0990911A
:10F970004F0997FD0196959587958093000A809190
:10F980000001482F55279A012B5F3F4F80911F019F
:10F99000909120012817390784F480911F019091DC
:10F9A0002001841B950B9C01220F331F280F391F48
:10F9B000822F82518093070A02C01092070AE090BA
:10F9C000A103F090A2030091A3031091A403C80126
:10F9D000B70124E630E040E050E00E9420993093E7
:10F9E000090A2093080A37FF04C01092090A1092EE
:10F9F000080AC801B70124E630E040E050E00E9468
:10FA00002099DA01C9018C509E4F90930D0A809382
:10FA10000C0A80911F01909120019093020A80931B
:10FA2000010A80911F01909120019093040A809314
:10FA3000030A0E94007A90930F0A80930E0A88E7C7
:10FA40008093100A80911F01909120019093140AD5
:10FA50008093130A8091AB048C5E8093050A809199
:10FA6000AC048C5E8093060A8091C6099091C70908
:10FA70006AE070E00E94D7987093160A6093150AA6
:10FA80001092F7098091C2099091C3099093120ACC
:10FA90008093110A85EF99E09093CC048093CB0476
:10FAA0002CE230E002C020E030E0C9011F910F914C
:10FAB000FF90EF900895EF92FF920F931F93CF93D3
:10FAC000DF938091AD049091AE049C0153E0220F2E
:10FAD000331F5A95E1F7281B390B80911F03909132
:10FAE0002003280F391F37FF02C0295F3F4F43E033
:10FAF000359527954A95E1F73093AE042093AD04F0
:10FB00009091BD04992309F020C38091BC04282F53
:10FB10003327442755278F5F8093BC04F901213197
:10FB2000310508F00FC3E857FF4F0C94729980918C
:10FB30006F0385FF2AC080E00E94359180911F01EC
:10FB4000909120016AE070E00E94EB989F938F9360
:10FB500080911F01909120016AE070E00E94EB9873
:10FB60007F936F938CEB9DE09F938F9388E291E955
:10FB70009F938F93E091F404F091F50409952DB7CC
:10FB80003EB7285F3F4F2DBF28C080E00E943591CF
:10FB900080911F01909120016AE070E00E94EB9833
:10FBA0009F938F9380911F01909120016AE070E0F4
:10FBB0000E94EB987F936F9389EC9DE09F938F93C6
:10FBC00087E091E99F938F93E091F404F091F5041D
:10FBD00009958DB79EB708968DBF80912D0980FF3E
:10FBE00039C08091BE038823E9F08AE00E943591F4
:10FBF00080913B0199279F938F938091A1039091CE
:10FC0000A203A091A303B091A403BC01CD0124E6FB
:10FC100030E040E050E00E9420993F932F9386ED22
:10FC20009DE099C68AE00E9435918091A103909150
:10FC3000A203A091A303B091A403BC01CD0124E6CB
:10FC400030E040E050E00E9420993F932F9382EEF5
:10FC50009DE0ADC78AE00E9435918DEE9DE09F93B7
:10FC60008F9387E091E90C94088780916F0385FF5B
:10FC70002AC085E10E9435918091DA029091DB02E1
:10FC80006CE370E00E94D7989F938F938091DA0283
:10FC90009091DB026CE370E00E94D7987F936F93A2
:10FCA00087EF9DE09F938F9388E291E99F938F93D5
:10FCB000E091F404F091F50409952DB73EB7285F63
:10FCC0003F4F2DBF28C085E10E9435918091DA0217
:10FCD0009091DB026CE370E00E94D7989F938F9322
:10FCE0008091DA029091DB026CE370E00E94D79879
:10FCF0007F936F9384E09EE09F938F9387E091E9D9
:10FD00009F938F93E091F404F091F50409958DB7DA
:10FD10009EB708968DBF8FE10E94359180E690E0F6
:10FD20009F938F938091E8089091E9089F938F9318
:10FD300081E19EE09F938F93C7E0D1E9DF93CF935A
:10FD4000E091F404F091F504099580916E032DB7CC
:10FD50003EB7285F3F4F2DBF80FF06C089E20E945B
:10FD600035918CE19EE073C389E20E9435918EE16A
:10FD70009EE0B9C680916F0385FF1BC08AE20E9496
:10FD800035918091C6099091C7099F938F9380E226
:10FD90009EE09F938F9388E291E99F938F93E091E8
:10FDA000F404F091F50409958DB79EB706968DBFC2
:10FDB0001BC08AE20E9435918091C6099091C709C3
:10FDC0009F938F9388E29EE09F938F9387E091E9C2
:10FDD0009F938F93E091F404F091F50409952DB76A
:10FDE0003EB72A5F3F4F2DBF86E30E943591809139
:10FDF000C2099091C3096AE070E00E94D7989F936E
:10FE00008F938091C2099091C3096AE070E00E94CB
:10FE1000D7987F936F9380E39EE09F938F9387E0C3
:10FE200091E99F938F93E091F404F091F504099583
:10FE30008DB79EB70896C9C689E00E9435918CE3BC
:10FE40009EE09F938F9307E011E91F930F93E0913A
:10FE5000F404F091F50409958EE10E9435910F901C
:10FE60000F900F900F908EE39EE09F938F931F93C0
:10FE70000F93E091F404F091F504099583E30E9457
:10FE800035910F900F900F900F9080E49EE09F931C
:10FE90008F931F930F93E091F404F091F50409956B
:10FEA0008FE30E9435910F900F900F900F9082E496
:10FEB0009EE09F938F931F930F93E091F404F09132
:10FEC000F50409958EE70E9435910F900F900F90E1
:10FED0000F9088E59EE09F938F931F930F939AC78F
:10FEE00080919901882309F462C08DE50E943591C3
:10FEF0008EE69EE09F938F93C7E0D1E9DF93CF9387
:10FF0000E091F404F091F504099584E50E9435919F
:10FF10000F900F900F900F908091490999279F9310
:10FF20008F9380E79EE09F938F93DF93CF93E09131
:10FF3000F404F091F50409958EE50E9435912DB7F2
:10FF40003EB72A5F3F4F2DBF80914C0990914D09DC
:10FF50006AE070E00E94D7987F936F9389E79EE0F4
:10FF60009F938F93DF93CF93E091F404F091F50486
:10FF700009958DB79EB706968DBF80914A0983304B
:10FF800081F48091480981FF06C08BE50E9435917C
:10FF900083E89EE0A8C58BE50E94359186E89EE047
:10FFA000A2C58BE50E94359189E89EE02DC784E0CB
:10FFB000D3C380919901882309F47AC08091BF044A
:10FFC00097E0E92E91E9F92E882309F44BC089E6E0
:10FFD0000E9435918091840499279F938F938CE898
:10FFE0009EE09F938F93FF92EF92E091F404F09143
:10FFF000F504099585E70E9435912DB73EB72A5F34
:020000021000EC
:100000003F4F2DBF80918D0199279F938F9300E6DD
:1000100010E01F930F9380914E0990914F099F9389
:100020008F9387E99EE09F938F93FF92EF92E091E9
:10003000F404F091F504099582E70E9435918DB79B
:100040009EB70A968DBF8091820499279F938F93C4
:100050001F930F938091830499279F938F9383EA33
:100060009EE073C689E60E94359180918D019927A3
:100070009F938F9380E690E09F938F9380914E099A
:1000800090914F099F938F9380914B0999279F934C
:100090008F9383EB9EE09F938F93FF92EF92E0917B
:1000A000F404F091F50409958DB79EB70C968DC5B3
:1000B00085E052C3909185049923D1F08091C804C2
:1000C000882381F0903270F487E00E94567983E9AA
:1000D0000E9435918091850499279F938F938CEC92
:1000E0009EE0A4C383E90E94359187ED9EE0B3C3EF
:1000F00080916F0307E0E02E01E9F02E85FF06C036
:1001000084E90E9435918DED9EE0DAC383E90E9477
:10011000359180EF9EE0D4C380915E0B863059F418
:100120008091BF04882319F01092BF049AC681E021
:100130008093BF0496C6883009F093C60E943A9116
:1001400081E0DBC39093BC0494C6913009F0E0C316
:100150008091BC04282F3327442755278F5F809335
:10016000BC04F9012131310508F07EC6E756FF4F86
:100170000C94729980916F0385FF43C080E00E94C8
:1001800035918091C6099091C7099F938F93809173
:100190001F01909120016AE070E00E94EB989F930C
:1001A0008F9380911F01909120016AE070E00E947E
:1001B000EB987F936F938091DA029091DB026CE36E
:1001C00070E00E94D7989F938F938091DA0290916C
:1001D000DB026CE370E00E94D7987F936F9386E018
:1001E0009FE09F938F9388E291E99F938F93E09193
:1001F000F404F091F50409952DB73EB7225F3F4F07
:10020000B1C580E00E9435918091C6099091C709DF
:100210009F938F9380911F01909120016AE070E07D
:100220000E94EB989F938F9380911F0190912001E2
:100230006AE070E00E94EB987F936F938091DA02FE
:100240009091DB026CE370E00E94D7989F938F93AC
:100250008091DA029091DB026CE370E00E94D79803
:100260007F936F9381E29FE0C2C285E10E94359146
:1002700080E690E09F938F9380918A0190918B010B
:100280009F938F938CE39FE09F938F93C7E0D1E977
:10029000DF93CF93E091F404F091F50409958091F8
:1002A0002D092DB73EB7285F3F4F2DBF80FF51C0AE
:1002B0008091BE03882339F18FE10E9435918091AE
:1002C000A1039091A203A091A303B091A403BC0148
:1002D000CD0124E630E040E050E00E9420993F93B9
:1002E0002F9386E49FE09F938F9387E191E99F93FB
:1002F0008F93E091F404F091F50409958DB79EB7C2
:1003000006968DBF38C08FE10E9435918091A10380
:100310009091A203A091A303B091A403BC01CD01CD
:1003200024E630E040E050E00E9420993F932F9374
:100330008FE49FE09F938F93DF93CF93E091F4043A
:10034000F091F50409952DB73EB72A5F3F4F2DBFB9
:1003500012C08FE10E94359188E59FE09F938F93B3
:10036000DF93CF93E091F404F091F50409950F9099
:100370000F900F900F9089E20E94359180913B0180
:1003800099279F938F9382E69FE09F938F93DF93AC
:10039000CF9313C4809199018823F9F08BE20E94D6
:1003A000359180918D0199279F938F9380914C096E
:1003B00090914D096AE070E00E94D7987F936F9307
:1003C00080E690E09F938F9380914E0990914F0922
:1003D0009F938F9385E69FE058C182E0BDC18FE374
:1003E0000E9435918091C4099091C5099F938F9384
:1003F0008091C2099091C3096AE070E00E94D79889
:100400009F938F938091C2099091C3096AE070E035
:100410000E94D7987F936F938CE79FE09F938F9371
:10042000C7E0D1E9DF93CF93E091F404F091F504B4
:10043000099580916E032DB73EB7265F3F4F2DBFC4
:1004400080FF0AC082E50E94359180E99FE09F937A
:100450008F9387E191E9DCC482E50E94359183E9BD
:100460009FE041C38091990117E0E12E11E9F12E3F
:10047000882309F449C084E50E9435918091490997
:1004800099279F938F9380914B0999279F938F93DF
:1004900086E99FE09F938F93E701FF92EF92E091AF
:1004A000F404F091F50409958DB79EB708968DBFB9
:1004B00080914A09833051F484E60E94359189EA9B
:1004C0009FE09F938F93FF92EF920BC084E60E9470
:1004D00035918FEA9FE09F938F9388E291E99F93F4
:1004E0008F93E091F404F091F50409950F900F902B
:1004F0000F900F908091480981FFBBC484E60E9451
:10050000359185EB9FE0EFC284E50E9435918BEB3E
:100510009FE0D6C18091BE04C7E0EC2EC1E9FC2E5D
:10052000882309F450C089E60E94359180912E08F5
:100530006AE00E94CB98892F99279F938F9380918F
:100540002E080E94CB9899279F938F93809126081D
:100550000E94CB98892F99279F938F93809126088B
:100560000E94CB9899279F938F9380911E080E9499
:10057000CB98892F99279F938F9380911E080E9473
:10058000CB9899279F938F93809116080E94CB98C0
:10059000892F99279F938F93809116080E94CB985B
:1005A00099279F938F9381ED9FE09F938F93FF9265
:1005B000EF92E091F404F091F50409952DB73EB760
:1005C0002C5E3F4FCFC389E60E94359180E690E0D4
:1005D0009F938F9380913008992787FD90959F93E3
:1005E0008F9380912808992787FD90959F938F93EB
:1005F00080912008992787FD90959F938F938091F4
:100600001808992787FD90959F938F938EEE9FE012
:100610009F938F93FF92EF92E091F404F091F50491
:1006200009958DB79EB70E96D0C28091BE04909169
:100630003D07882309F48DC0943009F48CC09630AE
:10064000A1F58EE70E94359180913E086AE00E94F4
:10065000CB98892F99279F938F9380913E080E9472
:10066000CB9899279F938F93809136080E94CB98BF
:10067000892F99279F938F93809136080E94CB985A
:1006800099279F938F9381E090E19F938F9387E0C9
:1006900091E99F938F93E091F404F091F50409950B
:1006A0002DB73EB7245F3F4F5DC3973008F4E1C3D9
:1006B0008EE70E94359180914E086AE00E94CB98A7
:1006C000892F99279F938F9380914E080E94CB98F2
:1006D00099279F938F93809146080E94CB98892FEA
:1006E00099279F938F93809146080E94CB989927D2
:1006F0009F938F9380913E080E94CB98892F9927D2
:100700009F938F9380913E080E94CB9899279F9347
:100710008F93809136080E94CB98892F99279F93B9
:100720008F93809136080E94CB9899279F938F933F
:1007300080E190E19F938F9387E091E99F938F935E
:10074000E091F404F091F50409958DB79EB74496B5
:100750003CC2943021F486E00E9456798AC39630D8
:10076000F1F48EE70E94359180E690E09F938F939D
:1007700080914008992787FD90959F938F93809152
:100780003808992787FD90959F938F938DE290E18C
:100790009F938F9387E091E99F938F93DAC297306D
:1007A00008F467C38EE70E94359180E690E09F933E
:1007B0008F9380915008992787FD90959F938F93F1
:1007C00080914808992787FD90959F938F938091FA
:1007D0004008992787FD90959F938F9380913808C3
:1007E000992787FD90959F938F9380E490E19F9345
:1007F0008F9387E091E99F938F930ECF909185041B
:10080000992309F44AC08091C8048823F9F09032F2
:10081000E8F487E00E94567983E90E94359180913F
:10082000850499279F938F9383E590E19F938F93FE
:1008300087E191E99F938F93E091F404F091F5049F
:1008400009952DB73EB72A5F3F4F8CC283E90E94BE
:1008500035918EE590E19F938F9307E011E91F9307
:100860000F93E091F404F091F50409951F921F9203
:100870009091850481E1989FC0011124865A944F7C
:100880009F938F931F930F93E091F404F091F504DD
:1008900009958DB79EB70A9698C180916F03B7E00E
:1008A000EB2EB1E9FB2E85FF06C084E90E9435914D
:1008B00084E690E105C083E90E94359187E790E1E5
:1008C0009F938F93FF92EF92A5C280915E0B86302B
:1008D00079F48091BE04882319F01092BE0403C0FD
:1008E00081E08093BE0485E00E94567986E0AEC226
:1008F000883031F40E943A9182E08093BD04AFC207
:10090000813009F0AEC20E943A911092BD04A7C294
:10091000923009F0ACC28091BC04282F33274427C1
:1009200055278F5F8093BC04F9012131310508F010
:100930009BC2E655FF4F0C94729980E00E9435915E
:100940008EEA97E09F938F930E946E3299279F9330
:100950008F938DE890E19F938F9387E191E99F9327
:100960008F93E091F404F091F50409952DB73EB70B
:10097000285F3F4FF7C185E10E9435918CEB97E0EE
:100980009F938F93809100016AE00E94CB98892FFA
:1009900099279F938F93809100010E94CB9899276C
:1009A0009F938F938CE990E19F938F9387E091E9D8
:1009B0009F938F93E091F404F091F504099569CF2A
:1009C0008AE20E9435918DEA90E19F938F93C7E070
:1009D000D1E9DF93CF93E091F404F091F504099508
:1009E00080912D090F900F900F900F9080FF41C0C4
:1009F00080914B079091750181FD0BC0892F99273C
:100A00009F938F9382EB90E19F938F93DF93CF938C
:100A100013CFE091F404F091F504933318F08CEBCC
:100A200090E102C083EC90E19F938F93DF93CF938B
:100A300009950F900F900F900F9080911109E09100
:100A4000F404F091F5049091750180FF0BC0892F9B
:100A500099279F938F938AEC90E19F938F93DF93D5
:100A6000CF93AFC0892F99279F938F9380ED90E10B
:100A7000CFC086ED90E137C08FE30E9435918FEDB6
:100A800090E19F938F93C7E0D1E9DF93CF93E091FB
:100A9000F404F091F50409950F900F900F900F90CA
:100AA0008091A107882319F483EE90E11CC0809106
:100AB0007C03E091F404F091F504882319F08CEEA6
:100AC00090E102C083EF90E19F938F93DF93CF93E8
:100AD00009950F900F900F900F908091AC0786FFB3
:100AE000C8C18AEF90E19F938F93DF93CF9392C118
:100AF00084E50E94359181E091E19F938F93C7E057
:100B0000D1E9DF93CF93E091F404F091F5040995D6
:100B100080912D090F900F900F900F9085FD03C0CD
:100B200086E091E111C080918F07883F10F4E82F93
:100B300007C0EFEFF0E0E81BF109E855FC4FE0815A
:100B4000E23358F48FE091E19F938F93DF93CF933B
:100B5000E091F404F091F50416C0E43B18F086E14E
:100B600091E1F2CF8091AC07E091F404F091F504AB
:100B700085FF03C08DE191E102C084E291E19F9382
:100B80008F93DF93CF9309950F900F900F900F9055
:100B90008091A507882309F46CC18EE50E943591E8
:100BA0008091A50799279F938F938BE291E19F9363
:100BB0008F9387E091E99F938F93E091F404F091F4
:100BC000F50409958DB79EB706968DBF52C189E68B
:100BD0000E94359186E391E19F938F93C7E0D1E91D
:100BE000DF93CF93E091F404F091F50409950F9011
:100BF0000F900F900F908091A407E091F404F09172
:100C0000F504882351F099279F938F9380E491E115
:100C10009F938F93DF93CF9313CE84E491E19F93BF
:100C20008F93DF93CF93FAC08091C004A7E0EA2EA0
:100C3000A1E9FA2E882309F053C08EE70E9435916E
:100C40008091690199279F938F9380914007E82FA6
:100C5000FF27EE0FFF1FEE58F74F808191819F9382
:100C60008F9380913F07E82FFF27EE0FFF1FEE586D
:100C7000F74F808191819F938F938AE491E19F93B5
:100C80008F93FF92EF92E091F404F091F5040995AF
:100C900083E90E9435918DB79EB70A968DBF8091EA
:100CA0004207E82FFF27EE0FFF1FEE58F74F808116
:100CB00091819F938F9380914107E82FFF27EE0F3B
:100CC000FF1FEE58F74F8081918181589F4F9F936E
:100CD0008F938EE591E19F938F93FF92EF9241CE98
:100CE0008EE70E9435918091AA0399279F938F9355
:100CF0008091A90399279F938F938091A8039927A7
:100D00009F938F938DE691E19F938F93FF92EF9244
:100D1000E091F404F091F504099583E90E9435917E
:100D20008DB79EB70A968DBF8091AD0399279F938B
:100D30008F938091AC0399279F938F938091AB03FE
:100D400099279F938F9381E891E19F938F93FF92CF
:100D5000EF92E091F404F091F50409952DB73EB7B8
:100D6000265F3F4F2DBF85C08091C804882309F4BA
:100D700080C08EE70E94359180912D0986FD11C0BB
:100D800085E991E19F938F9388E291E99F938F93F7
:100D9000E091F404F091F50409950F900F900F90F5
:100DA0000F908091AA0799278F709070892B89F0F6
:100DB00084EA91E19F938F9388E291E99F938F93C7
:100DC000E091F404F091F50409950F900F900F90C5
:100DD0000F9080912D0982FF11C08EEA91E19F93BF
:100DE0008F9388E291E99F938F93E091F404F091BF
:100DF000F50409950F900F900F900F9080912D0999
:100E000083FD37C083EB91E19F938F9388E291E953
:100E10009F938F93E091F404F091F50409950F905E
:100E20000F900F900F9025C000915E0B063089F453
:100E30008091C004882319F01092C00403C081E09F
:100E40008093C00486E00E94567987E00E9456791C
:100E500008C0013031F40E943A910093BD04109211
:100E6000BC0410925E0B05C01092BC0402C010922C
:100E7000BD04E6E0CDB7DEB70C9463994FB728E127
:100E800030E0F8948091C9008F778093C9008091F9
:100E9000C9008F7B8093C9008091C9008F7D8093AA
:100EA000C900832F99278093CD002093CC00809197
:100EB000C80082608093C80080E18093C90080915F
:100EC000CA008F778093CA008091CA008F7B80937D
:100ED000CA008091CA008091CA008F7E8093CA00A8
:100EE0008091CA0088608093CA008091C9008B7F7E
:100EF0008093C9008091CA0084608093CA00809169
:100F0000CA0082608093CA008091C80087FF03C036
:100F10008091CE00F9CF8091C90080688093C9008C
:100F200080913C0B846080933C0B4FBF089590915F
:100F30009704992341F48F3031F49093C20480E5F3
:100F4000809397040895E091C204EF5FE093C20498
:100F5000E83121F481E08093C1040895E93120F063
:100F600089E18093C2040895FF27EB5DF44F8083ED
:100F70000895A0E0B0E0EFEBF7E80C94439991E01E
:100F8000D92E82E0A82EBD2CE12C01E0F02E80911C
:100F90003C0B82FDB5C080916F008F7D80936F0008
:100FA000E091A707EE2351F0FF27EE0FFF1FEE5849
:100FB000F74F80819181843691055CF48091A7037D
:100FC000883C20F48091A7038C5E01C088EC80935C
:100FD000A7038091260B682F77278091C304815047
:100FE0008093C3048F3F31F41CE7C12E82E08093CD
:100FF000C30402C0C4E2CC2E40E04C1508F07EC011
:10100000EA2DFF27EB5DF44F80818D2111F06E29D1
:101010007F298D2D9927880F991FD82E882319F4A1
:10102000B1E0DB2EAD0CEE0CFF1C20E0E21628E058
:10103000F20609F061C0A1E0EA2EF12CCB0180504C
:10104000944065E070E00E94EB98AB2DBB27FD015A
:10105000EA0FFB1FEE58F74F808191819C01220F10
:10106000331F280F391F260F371F37FF02C02D5F90
:101070003F4FE901D595C795D595C795CB01019609
:101080008C179D0714F4219706C061507040C61755
:10109000D7070CF421968091A703833CD8F08D01EB
:1010A0000A0F1B1FF801EE58F74F80819181FE0156
:1010B000E81BF90BCF0163E070E00E94EB98CB01D5
:1010C000880F991F860F971F0A55174FF8019183B4
:1010D000808307C0AA0FBB1FAA55B74F11961C9259
:1010E0001E92EB2DFF27EE0FFF1FEE58F74FD18317
:1010F000C08360E070E0B3944F5F7FCF10923A01FD
:101100001092C104EAE0CDB7DEB70C945F99089560
:10111000089540E050E08091C4049091C5049C0182
:10112000220F331F280F391F80911F039091200336
:10113000280F391F37FF02C02D5F3F4F3595279588
:10114000359527953093C5042093C40480913B01C5
:101150008B32D9F480915007282F332780919B033D
:1011600090919C03829FA001839F500D929F500DF0
:101170001124CA0157FD4F96AC0125E055954795BE
:101180002A95E1F74B5F5F4F3DC08D32D9F48091D6
:101190005007282F332780919B0390919C03829FB7
:1011A000A001839F500D929F500D1124CA0157FD3D
:1011B0004F96AC0195E0559547959A95E1F74550C6
:1011C000504020C0803271F480916F0381FF1AC0BB
:1011D000C90137FD4F96AC0185E0559547958A9535
:1011E000E1F710C08E3529F480919603482F5527DA
:1011F00009C0863739F480919603992744275527EB
:10120000481B590BCA01AA2797FDA095BA2F8093B6
:10121000940290939502A0939602B093970208953A
:101220000F931F930E94107980911F0190912001CC
:10123000AA2797FDA095BA2F8093C3019093C4016C
:10124000A093C501B093C6018091C2099091C309D2
:10125000AA27BB278093D6019093D701A093D801EA
:10126000B093D9010AE010E08091C6099091C709B6
:10127000B8010E94D798CB01AA27BB278093E90128
:101280009093EA01A093EB01B093EC018091A1034C
:101290009091A203A091A303B091A403BC01CD013E
:1012A00024E630E040E050E00E9420992093FC01C9
:1012B0003093FD014093FE015093FF0180918A011C
:1012C00090918B01AA2797FDA095BA2F80930F02CA
:1012D00090931002A0931102B093120280914909D9
:1012E0009927AA27BB278093220290932302A093D9
:1012F0002402B093250280914B099927AA27BB2786
:101300008093350290933602A0933702B09338024F
:1013100080914C0990914D09B8010E94D798CB015A
:10132000AA27BB278093480290934902A0934A02C0
:10133000B0934B0280914E0990914F09AA2797FDD7
:10134000A095BA2F80935B0290935C02A0935D02FC
:10135000B0935E028091AC049927AA27BB278093A3
:101360006E0290936F02A0937002B093710280910D
:1013700084049927AA27BB27809381029093820235
:10138000A0938302B0938402809185049927AA27B1
:10139000BB278093A7029093A802A093A902B093C1
:1013A000AA021F910F9108954FB720E430E0F894FE
:1013B0008091C9008F778093C9008091C9008F7B8D
:1013C0008093C9008091C9008F7D8093C900832FCD
:1013D00099278093CD002093CC008091C800826033
:1013E0008093C80088E18093C9008091CA008F77FC
:1013F0008093CA008091CA008F7B8093CA0080913D
:10140000CA008F7D8093CA008091CA008F7E80932E
:10141000CA008091CA00877F8093CA008091C9006A
:101420008B7F8093C9008091CA0084608093CA003A
:101430008091CA0082608093CA008091C80087FFB3
:1014400003C08091CE00F9CF8091C900806880935D
:10145000C9004FBF08950F931F93CF93DF93482F79
:101460004F5F893108F08BC080917108841720F498
:101470004F5F409371084150CB0183539B4268E119
:1014800070E00E94EB98A42FBB27FD01EA0FFB1F21
:10149000EE58F74F808191819B01281B390BC901C0
:1014A00037FF03C0909581959F4F069794F48091E4
:1014B000A703883C30F48091A703865F8093A7033D
:1014C00008C088EC8093A70380916F008F7D809384
:1014D0006F00FD01EA0FFB1FEE58F74F80819181ED
:1014E0009C01220F331F280F391F260F371F37FF8C
:1014F00002C02D5F3F4FE901D595C795D595C7959A
:10150000CB0101968C179D0714F4219706C06150FA
:101510007040C617D7070CF421968091A703843B2F
:10152000D8F08D010A0F1B1FF801EE58F74F80818C
:101530009181FE01E81BF90BCF0163E070E00E948E
:10154000EB98CB01880F991F860F971F0A55174FED
:10155000F8019183808307C0AA0FBB1FAA55B74F1C
:1015600011961C921E92E42FFF27EE0FFF1FEE58DC
:10157000F74FD183C083443011F410923A01DF91C8
:10158000CF911F910F910895CF93DF9320915F0B1F
:10159000822F9927807F9070409709F06CC02F317F
:1015A00009F046C08091600B8093CF042091620BBC
:1015B0002093D1048091630B8093D004822F9927CC
:1015C0009093730880937208222309F054C080918D
:1015D0003F07282F3327220F331FF901EA55F74F12
:1015E0001182108280914007A82FBB27AA0FBB1F32
:1015F000FD01EA55F74F1182108280914207E82FD2
:10160000FF27EE0FFF1FCF018A55974FEC0119827C
:1016100018822E58374FE90119821882AE58B74FF9
:1016200011961C921E92EE58F74F1182108223C021
:10163000C22FCF70CA30F8F48091600B80938B0B6F
:101640008091610B80938A0B8091620B80938D0B4C
:101650008091630B80938C0B60918A0B70918B0B44
:101660008C2F0E942B8A60918C0B70918D0B8C2F8C
:101670008F5F0E942B8ADF91CF910895CF93C82F5F
:101680008F3F49F48091D2048F3F29F41092D40403
:101690001092D30432C02091D404222339F4CF31E4
:1016A00011F485E001C084E08093D5048091D504D5
:1016B0009091D3048217A0F4892F80958093D3044E
:1016C0008F3F19F48EEF8093D3048091D304C81711
:1016D00011F40E94C48A1092D4041092D3040BC057
:1016E000E22FFF27E15AF44FC0832F5F2093D404E9
:1016F0009C0F9093D304C093D204CF9108959091FE
:10170000CE04933240F4E92FFF27E959F44F808348
:101710009F5F9093CE040895833218F48D5F809379
:10172000CE04089590E2EAE6FBE08FE191938150C8
:1017300087FFFCCF0895CF93CFB723E031E0F89433
:101740008091C9008F778093C9008091C9008F7BF9
:101750008093C9008091C9008F7D8093C900832F39
:1017600099278093CD002093CC008091C80082609F
:101770008093C80088E18093C9008091CA008F7768
:101780008093CA008091CA008F7B8093CA008091A9
:10179000CA0080628093CA008091CA0080618093F1
:1017A000CA008091CA0088608093CA008091C900F5
:1017B00084608093C9008091CA0084608093CA00CD
:1017C0008091CA0082608093CA008091C80087FF20
:1017D00003C08091CE00F9CF8091C90080688093CA
:1017E000C9008091C90080648093C9000E94928BD7
:1017F000CFBFCF910895282F99278F709070892B94
:1018000031F420958091CD04822B8093CD040895EE
:101810001F920F920FB60F9211248F93EF93FF93A5
:101820008091D402882309F068C0E091D704EE23A8
:1018300089F48091D604882369F48091670B88230A
:1018400021F081E08093D80405C08091C9008160B7
:101850008093C9008091D804882379F4EF5FE093E6
:10186000D70480913E0B8E1720F481E08093D8043A
:101870001CC0FF27E25CF44F3CC08091D604882353
:1018800061F48091670B882311F483E003C08139F0
:1018900099F481E08093D6040FC0833099F480914D
:1018A000670B882349F01092670B8091C9008E7FE7
:1018B0008093C9008EEF1EC08091C9008160809323
:1018C000C9000EC0833261F48091C9008E7F80937D
:1018D000C9008FEF8093CE0081E08093D40218C0BE
:1018E0008091D604E82FFF27E959F44F8F5F80934A
:1018F000D60480818093CE000BC01092D604109243
:10190000D7041092D8048091C90080618093C900E7
:10191000FF91EF918F910F900FBE0F901F90189530
:10192000682727E0322F67FF06C0862F9927880F88
:10193000991F832702C0862F880F682F215027FF09
:10194000F2CF992708950F931F93CF93DF93062F1C
:1019500060E0162F601740F4EC0189910E94908C92
:10196000682F1F5F1017C8F3862F9927DF91CF913B
:101970001F910F910895DC0190E0961758F48C9117
:10198000803241F09F5F961728F4FD01E90FF11DA9
:101990008081F6CF892F99270895A0E0B0E0E3ED8C
:1019A000FCE80C9444998FE980933F0B80E180938D
:1019B000410B84EA8093420B85E58093430B8DE5D0
:1019C0008093440B1092450B8091DA04882309F030
:1019D0006AC08091D90413E1819FC001112463E0A2
:1019E00084559E4F0E94BB8C082F8091D904819F03
:1019F000C00111246AE08E559E4F0E94BB8C982F27
:101A0000800F865F80933E0B4EEFB42EB80EB092DF
:101A1000400B2091D9042093460BE92EFF24C701E7
:101A200033E0880F991F3A95E1F7802B8093470B9D
:101A3000822F992723E1C22ED12C8C9D90018D9D60
:101A4000300D9C9D300D1124C9018E559E4FA7016C
:101A5000BC0188E49BE00E940C9711278091D90477
:101A600099278C9DE0018D9DD00D9C9DD00D11245A
:101A7000CE0184559E4FA801BC01C701885B944FDD
:101A80000E940C97025C144F0E0D1F1D6B2D80E4FD
:101A90009BE00E94A38CF80182878091DA048F5F1B
:101AA0008093DA0470C01091450B0E941089409118
:101AB000D5024031C8F563E170E0812F9927DC0140
:101AC000AA0FBB1FA80FB91FA25CB44F842F992780
:101AD000869FF001879FF00D969FF00D1124EE5523
:101AE000FE4F2585C4E0880F991FCA95E1F7282B82
:101AF000ED012887268537853F7982899927982F98
:101B000088279295990F907E282B392B2987832F30
:101B100099278A87842F8F5F1F5F163018F4482F0C
:101B2000803158F28093D50283E0189F90011124F0
:101B3000822F885F80933E0B825C8093400B812FC5
:101B400099278C01000F111F080F191F025C144FF9
:101B5000822F8A5F682F80E49BE00E94A38CF801AB
:101B600080878091D502803170F081E08093D5022A
:101B70001092DA048091D9048F5F8093D904803168
:101B800010F01092D904E9E0CDB7DEB70C9460995B
:101B90008091D402882309F447C080916F0385FDAA
:101BA00004C08091D802882381F082E98093670B7A
:101BB00083E28093680B8091D802882309F485E53D
:101BC0008093690B1092D80202C08093670B8091BA
:101BD000D6028F3071F48091CD040E94E377882380
:101BE00041F081E98093670B8093680B81E38093D8
:101BF000690B1092D4028091C80085FFFCCF8091C0
:101C0000C9008F7E8093C9008091C9008E7F809328
